:10000000407B0020D93C000051AE0100AD3C000017
:10001000AD3C0000AD3C0000AD3C00000000000025
:10002000000000000000000000000000B5390000E2
:10003000AD3C00000000000061390000AD3C000054
:10004000653A000069050100653A0000653A000064
:10005000653A0000653A0000653A0000653A000024
:10006000653A0000653A0000653A0000653A000014
:10007000653A0000653A0000653A0000653A000004
:10008000653A0000653A0000653A0000653A0000F4
:10009000653A0000653A0000653A0000653A0000E4
:1000A000653A0000653A0000653A0000653A0000D4
:1000B000653A0000653A0000653A0000653A0000C4
:1000C000653A0000653A0000653A0000653A0000B4
:1000D000653A0000653A0000653A0000653A0000A4
:1000E000653A0000653A0000653A0000653A000094
:1000F000653A0000653A0000653A0000653A000084
:1001000053B94AB9002908BF00281CBF4FF0FF317E
:100110004FF0FF3000F00CB8ADF1080C6DE904CEE3
:1001200000F008F8DDF804E0DDE9022304B07047D0
:10013000704700BF2DE9F04F07468C460846099EE0
:1001400015463C461946002B40F0C6808242B2FA62
:1001500082F746D94FB1C7F1200E24FA0EFE00FAFD
:1001600007F3BD404EEA030CBC404FEA15481FFAA6
:1001700085FEBCFBF8F9220C08FB19C309FB0EFA3B
:1001800042EA03439A4528D9EB1809F1FF3004D21B
:100190009A4502D9A9F102002B44A3EB0A03A4B2A9
:1001A000B3FBF8F208FB123302FB0EFE44EA0344F1
:1001B000A64514D92C1902F1FF3303D2A64501D963
:1001C000931E2C44A4EB0E0443EA00401EB1FC40F5
:1001D000002334607360BDE8F08F4846DDE71346C6
:1001E000F0E702B9FFDE87BB831A01214FEA154E03
:1001F000AAB2B3FBFEFC200C0EFB1C330CFB02F876
:1002000040EA0343984563D9EB180CF1FF3004D260
:10021000984502D9ACF102002B44A3EB0803A4B229
:10022000B3FBFEFC0EFB1C330CFB02F244EA03445E
:10023000A2424FD92C190CF1FF3304D2A24202D9A9
:10024000ACF102032C44A41ABEE7C7F1200C20FA3B
:100250000CF800FA07F324FA0CFCBD404CEA030248
:100260004FEA154EABB2B8FBFEFC110C0EFB1C8026
:100270000CFB03F941EA0040814504FA07F423D955
:1002800028180CF1FF3104D2814502D9ACF10201EA
:100290002844A0EB090092B2B0FBFEFC0EFB1C0050
:1002A0000CFB03F842EA004398450FD9EB180CF118
:1002B000FF3204D2984502D9ACF102022B44A3EBE1
:1002C000080342EA014191E76146E2E76246F6E748
:1002D0006046A2E76346B6E7834205D90EB1C6E998
:1002E00000700021084676E7B3FA83F181B98342B2
:1002F00001D3BA420AD8BC1A60EB030301209C4622
:10030000002E68D0C6E9004C002164E70846F7E7F4
:10031000C1F1200C8B4022FA0CF41C4302FA01F5C7
:1003200000FA01F327FA0CF220FA0CFB4FEA144909
:100330001343BBFBF9F81FFA84FE09FB18BB1A0C28
:1003400008FB0EFA42EA0B42924507FA01F73ED942
:10035000A21808F1FF3004D2924502D9A8F1020098
:100360002244A2EB0A029BB2B2FBF9F809FB182265
:1003700008FB0EFE43EA024296452AD9A21808F16C
:10038000FF3304D2964502D9A8F10203224443EA7E
:100390000040A0FB0593A2EB0E029A42CE4698467F
:1003A00002D306D14F4504D2B9EB050E63EB040826
:1003B000013886B1B7EB0E0362EB080707FA0CFCB5
:1003C000CB404CEA0303CF40C6E900379CE74046E8
:1003D000C7E74346DBE73146FDE6000000000000CA
:1003E0002DE9F041D0E90B35866A5C193034A6421C
:1003F0008846174618D81C4DA3FB050118A3D3E95E
:100400000023FFF77DFEA41B20F07F40C8F800000A
:1004100013A3D3E90023A4FB0501FFF771FE20F02D
:100420007F403860BDE8F0810F4C0DA3D3E9002375
:10043000A6FB0401FFF764FE05F1300120F07F40C8
:10044000C8F8000006A3D3E90023A1FB0401FFF7CD
:1004500057FE20F07F403860BDE8F081AFF30080A8
:100460008D49FD1A0700000000CA9A3B00000000F9
:1004700000284FD02DE9F04F6B4C94F86A5015F0DE
:10048000010591B040F0BF8094F82500FF2300F0F3
:10049000030084F826300FF07BFC94F86A004207D2
:1004A00029D494F8292094F8353004EB820204EB27
:1004B0008303D76AD3F8389087B15B48394609F08F
:1004C00087F83B785B0605D5062103F039FF002845
:1004D00000F004825448494609F07AF83B7813F05A
:1004E0000E0F19D1236A002B00F0AA800C25284694
:1004F00011B0BDE8F08F2A4604F16B01C0F3C000D3
:100500000FF0C0FDFF2884F82600CAD028460FF05F
:1005100085FCC6E708F0C8BD94F824300121C3F378
:1005200042030CA88DF8303004F096F800286FD004
:1005300099F801100246384608F046FE3B49B4F8E7
:10054000689031230026A360A0FB010134A3D3E906
:100550000023C4E9056626706660E660FFF7D0FDFB
:10056000206105F021FB8046B9F1000F07D13E78EC
:1005700006F00F06A6F10106B6FA86F6760994F89B
:100580002400236966F3000010F0010684F82400BB
:1005900040F07481264A2748049303F24713A9FBCD
:1005A0000001069402961360912303FB0911224B6C
:1005B0000793224B05934FF6FF7309924FF0020900
:1005C00003930EAF16A3D3E90023CDF83890089714
:1005D000FFF796FD4346CDE900604A4630460321C9
:1005E00005F062F9394608F07BF888B994F86A306A
:1005F00043F0010384F86A3009F0D2F918B90120F8
:100600000FF0A8FB73E70025284611B0BDE8F08F76
:10061000236A002B3FF46AAF08F01AFD0C2566E749
:100620008D49FD1A07000000284C002000CA9A3BA3
:10063000A04C0020002AE784817E0000399200004F
:1006400007F0C8FF8246002800F0508107F0CEFF77
:100650008346002800F047810AF008F80646002883
:1006600000F03E814FF6FF73406F338506F11C03A7
:100670000B93002800F03C8106F1680206F164014A
:1006800003F06AFEB6F86030DFF86CC223F4EF6363
:1006900023F0070343F4887343F00103A6F86030A6
:1006A00096F8393003F03F0363F07F0386F8393062
:1006B00096F87A3023F0070386F87A3096F83C30C3
:1006C00023F0070386F83C3096F8D6304FF0000848
:1006D0004FF01B10C6E9160C68F300037F2086F864
:1006E000D63086F8BD00FF2306220DF1310106F158
:1006F000D700A6F8C020C6E91288C6F87480A6F80C
:100700007880A6F82E80C6F8308086F83B80C6F840
:100710005080A6F8C480A6F8C880A6F8D080A6F8B5
:10072000CC808DF831308DF832308DF833308DF843
:1007300034308DF835308DF830808DF836301AF041
:10074000D3FB96F8D61068F3410186F8D610FF2344
:1007500006220DF1390106F1DD008DF839308DF8F2
:100760003A308DF83B308DF83C308DF83D308DF8C7
:100770003E308DF838801AF0B7FB96F8E430A6F8D2
:10078000F08023F0070386F8E43086F8F280C6F89C
:100790001481A6F81881A6F8308107F031FB96F88D
:1007A0004A31A6F8488123F0030386F84A3196F8C7
:1007B0007A30A6F8508123F0180386F87A3096F83C
:1007C000763186F8538123F0070386F8763196F860
:1007D0009631C6F854A168F3451386F8963196F819
:1007E000BE31A6F8748168F3C303002286F8BE31D7
:1007F0000023C6E94E01C6E9502386F8E580A6F835
:100800009481C6F8EC80A6F8BC81A6F8C8810AF0ED
:1008100041FBA6F8D2000AF043FBD6F8CC21374BB7
:10082000A6F8D4001340C6F8CC310AF03FFB96F886
:10083000D03160F3020386F8D0310AF03DFB06F1B7
:100840001C03236296F8D031C6F8D48160F3C50347
:10085000C4E918ABC6E97888C6E97688C6E9058890
:1008600086F80080F66186F8D03110F0F1FA0028A1
:100870003FF452AE08F0ECFB032538E60020204A96
:10088000DFF88090049302260EAF019305920321B6
:10089000CDE902000694434600900897CDF81C90DD
:1008A00032460E9605F056F8394607F019FF002833
:1008B0007FF4AEAE144A05924AF2D8320092CDE9E6
:1008C0000300CDE90100CDF81C900897069443463B
:1008D000012203210E9605F03DF883E6122506E677
:1008E000584607F089FE504607F07AFE0725FEE5D8
:1008F00006F16C007067BFE6480148010000FFF692
:1009000039920000817E00009D8F000000000000F1
:1009100070B590F824308AB0C3F342030D46044604
:1009200001210DF1230016468DF8233003F094FECB
:1009300071780246284608F047FC1D491AA3D3E9FE
:100940000023A0FB0101FFF7DBFB2369984205466A
:1009500020D21B1A00220192164A0293164BA21AA9
:10096000A3FB02320221920900230A4409AE099135
:1009700012490591CDE903330321D2B206960093C3
:10098000184605F059F8314607F0AAFE48B9256126
:100990000AB070BD02D9C21A0023DCE700200AB0F9
:1009A00070BD0C200AB070BD8D49FD1A0700000013
:1009B00000CA9A3B284C002089888888817E0000E4
:1009C00038B5194C9DF810E094F844C01CF00105AE
:1009D00022D163F3420C400194F83230A1874FEAF0
:1009E000CE0E0EF0180E00F0200040EA0E0023F0AC
:1009F000380303430D4884F83230A2FB00019123F1
:100A000003FB021106A3D3E9002384F844C0FFF7D7
:100A100077FB2064284638BD0C25284638BD00BF2A
:100A20008D49FD1A07000000C44C0020002AE7840D
:100A300010B59DF808C0044649014FEACC0000F00B
:100A4000180001F0200CA17D22844CEA000C0C4817
:100A500021F038014CEA010C9122A3FB000102FBBA
:100A6000031184F816C004A3D3E90023FFF748FB61
:100A7000606210BDAFF300808D49FD1A07000000D1
:100A8000002AE784000000002DE9F047044600F149
:100A9000350190F8440094F83230C0F3400060F320
:100AA00086138CB084F8323005F0B6F894F8322012
:100AB000A38F4D48E46102F079020025A3FB0001F9
:100AC00084F83220912202FB0311C4E9055544A3A6
:100AD000D3E900232570FFF713FB3123C4E9015349
:100AE000236CE5600933A0F13102934232BF2361E8
:100AF00022612564064605F057F8236A07460DF182
:100B00002C08002B4CD0394D394BCDF82080069461
:100B1000651BA3FB05353448A38F4FF0000AA3FBE8
:100B200000019122CDF80CA002FB0311236904936C
:100B3000304B0793304B05934FF0020928A3D3E9BC
:100B40000023CDF82C90FFF7DBFA104619464FF43E
:100B50007A720023FFF7D4FA2D090435EDB22A4644
:100B6000CDE901603B460321CDF800A0504604F0DA
:100B7000F1FE414607F0B4FD054668B994F84430EB
:100B800043F0010384F8443008F0F8FC0446F8B15F
:100B900028460CB0BDE8F0870C200CB0BDE8F0870B
:100BA000CDE90A33216943460AAA032001F0ACF9D2
:100BB0000028A8D10B99114809A3D3E90023A1FB70
:100BC0000001FFF79DFA0A9F20F07F4007449AE753
:100BD00048460FF0BFF820460CB0BDE8F08700BFD4
:100BE0008D49FD1A07000000002AE784C44C00204C
:100BF000398EE338817E0000A197000000CA9A3B3D
:100C00002DE9F04FC38D458E1D4490F81A31ADB2D9
:100C10002944164613F007028BB0044689B20AD065
:100C2000531E042B00F22E83DFE813F0A8011102FB
:100C3000890140011402B0F8F470C91B1FFA81F851
:100C4000090400F15E8190F93930002BC0F2448232
:100C500094F8F03084F8F13094F8942194F89531B8
:100C600094F8181184F8191193420AD094F8963127
:100C700003F00F03062B04D1002384F89521A4F878
:100C8000C830B34BD4F814911A68944204BF0022C0
:100C90001A60B9F1000F00F04A81D9F8000000286D
:100CA00000F04581B4F81C31B4F82AC04268C4F899
:100CB00014216345B4F81E21B4F8201100F0148209
:100CC000B4F828C0A9F81E30192389F8043000238D
:100CD000A9F806C0A9F82020A9F8221089F81C302C
:100CE000494607F08FFC07F097FCA368002B09DA50
:100CF000E168626823F0004391422CBF7618B61871
:100D0000A360F61A608DB4F81C9110FB08F080B255
:100D1000B0FBF9F119FB01F39BB298421FFA81FA7B
:100D200080F0F4801B1A40F2E2418A4803FB01F193
:100D3000A1FB000184A3D3E90023FFF7E1F920F030
:100D40007F400644E38D1F4494F939307D1B5544A0
:100D500040F2E24B002BE5850BFB09F7C0F2E68180
:100D6000D4F824117B4878A3D3E90023A1FB000128
:100D7000FFF7C6F920F07F483D4608F10108764AA2
:100D8000B4F82031B4F81E017449A4F82A903A440A
:100D9000B2FBF7F2A4F8C62042F2107202FB037312
:100DA0003944013BB1FBF7F1B3FBF7F78AB2831D7E
:100DB0009A42A085A4F8C270A4F8CE2004DDC0F544
:100DC0007F43FA331A4492B294F81A31A4F8CA2035
:100DD0001B0744BF0023A4F8C4300221012012F0F5
:100DE000C1FF002202218146012003F005FB5C497E
:100DF0004FF4F872204603F08FFA00F1050A5FFA0B
:100E00008AFA584B009452460121002004F02CFE2F
:100E100030F0020304D0544840F6DF4101F04AFDAF
:100E20004C4FA5FB077B48A3D3E90023384659461E
:100E3000FFF766F920F07F454C480723A5FB00012A
:100E4000381A03FB05116BEB01014FF47A72002392
:100E5000FFF756F9CDE9015008940694CDF80080CB
:100E6000216994F93950424804914249424C07940F
:100E700011EA250138BF014605914FF6FE71334650
:100E8000039152460121002004F064FD30F002037A
:100E900004D0354840F6F94101F00CFDB9F1000FDE
:100EA00040F03E8100200BB0BDE8F08F828D90F8BD
:100EB0001A51D0F8F83006321144D0F8D42189B252
:100EC0006FF30205A0F8F4101981A3F10900D4F81A
:100ED000D81184F81A5122B194F87651AE0740F136
:100EE0007381002900F08781D4F8DC21116843F870
:100EF000091C106053F8092CC4F8DC01002A00F02A
:100F000077816FF076000BB0BDE8F08F09FB11011F
:100F100040F2E2430F4889B203FB01F1A1FB00015B
:100F200009A3D3E90023FFF7EBF8361A0AE70E48C6
:100F300040F6344101F0BEFCD9F80000B2E66FF093
:100F40000F000BB0BDE8F08F8D49FD1A07000000BF
:100F5000204D002000CA9A3BFF5962027FC3C9019D
:100F6000E00C0020719C0000BCD401008D49FD1AEA
:100F7000ADEB000019EA0000419C0000DFF820837F
:100F8000012007F04FFB0746002800F04581C548C7
:100F900003F08CF90546002800F03E81C24B1A6828
:100FA000002A00F00F8107F05DFB3B68D4F81421A4
:100FB0005A602B79C4F8147143F003032B710C238E
:100FC0006B710023EB7194F828312B72B74AD4F877
:100FD0002431A2FB03239B0AA5F80930B4F81C3185
:100FE000A5F80B30B4F81E31A5F80D30B4F8203157
:100FF000A5F80F3094F81A31C4F8FC60032262F3AC
:10100000020384F81A31A368002B0ADAE1686268E7
:1010100023F0004391422CBF7618B618F31AC4F897
:10102000FC30A34B01220935C4F8F85002211046C8
:10103000C3E9024803F012FA00283FF462AF9D486A
:1010400040F6873101F036FC6FF076002BE7DFF8D1
:10105000688295E7D0F8F820D0F8D43190F8F00005
:1010600084F8F10094F818018F4984F8190194F874
:10107000940184F8950100200860D4F8D801A2F109
:101080000901B3B194F87651AD0712D494F8CF5159
:10109000EF070ED4D4F8E051AB4200F0D78058B936
:1010A000187900F00300032800F0DF80C4F8D8317D
:1010B00004E0002800F0A980D4F8DC31186842F878
:1010C000090C196052F8093CC4F8DC11002B00F03F
:1010D000A6806FF08B00E6E690F8E530002B3FF439
:1010E000B7AD80F8E520B7E5B4F82CC094457FF49F
:1010F000E7AD40F2E24C0CFB03FE42F2107C0CFB2D
:1011000001EC0CF1FF3CBCFBFEFCB4F8C2E01FFAA2
:101110008CFCE6457FF4D4AD012389F80430DFE58B
:1011200001220221104603F067F9BBE6226CA36C92
:1011300002FB1833A3640FF0F7FE054694F8E400B1
:10114000DFF87881C0F3C2000FF0F0FE054407FB22
:1011500005F55B4B94F8282105F5742505F23F252C
:10116000A3FB0535AD0CA36C25640BFB02F205FB5C
:101170000AF022657A080344963A934228BF134640
:10118000C4E911230023A0FB0801C4F8EC3042A3FA
:10119000D3E90023FEF7B4FF444B361AD4F82401F8
:1011A000A3FB0030800A0BFB00F0A0FB08013AA370
:1011B000D3E90023FEF7A4FF7D1BB4F81C9120F0B7
:1011C0007F48DCE51C60EEE694F8CF51ED073FF573
:1011D00088AED4F8E051AA4226D000297FF484AE2C
:1011E000117901F00301032946D0C4F8D8217DE626
:1011F000C4F8E40185E643F8092CC4E97500C4F895
:10120000DC01002A7FF47DAEF2E742F8093CC4E934
:101210007511C4F8DC1159E76FF0680043E6C4F8B3
:10122000E4116FF08B003EE61568C4F8E051002928
:101230007FF45AAE116843F8091C106053F8092C6A
:10124000C4E97600002A7FF45CAED1E71D68C4F8DB
:10125000E05100287FF430AF186842F8090C19609B
:1012600052F8093CC4E9761130E7D8790328F3D065
:101270000A287FF41BAFEFE7D1790329DAD00A29D6
:10128000B3D1D7E70B4840F6DB3101F013FB4FF049
:10129000000875E6AFF300808D49FD1A07000000D5
:1012A00021F20000484E0020204D00205917B7D1F0
:1012B000AC070020BCD40100611F000000CA9A3BAB
:1012C00083DE1B43000000002DE9F04F0B68D2F8CD
:1012D00000B01B6897B08A460A93037F00F11E0195
:1012E000C3F380130446154614A806228DF8473030
:1012F00019F0FAFD9AF811000C90FF280DF1480939
:1013000000F083804A460DF147010EF039FA9DF84E
:1013100047600236F6B28DF847600A9B277FD4F803
:1013200000C0CDF82CC003F17108FF094B4606F050
:1013300001024146384609F0C5FD00284BD19BF813
:10134000D6200D9066F341028BF8D620494606223E
:101350000BF1DD0019F0C8FD9BF8D62067F3000201
:1013600041468BF8D6200BF1D700062219F0BCFDC0
:101370002F1D032204F12E0105F1080019F0B4FD20
:1013800005F11806042204F12A01384619F0ACFDD3
:10139000052204F13A01304619F0A6FD3046052138
:1013A00003F05AF96A7F94F83F1000F03F0060F3B1
:1013B00005026A77C1F30402AA77A68EEE8101289E
:1013C000B6B201F01F0206D91B3202F01F020B2A2F
:1013D00001D80D9B0EBB0A9BE6680B9800225A6150
:1013E00095F82030012762F3000385F8203021466C
:1013F000277107F007F930683771314607F002F9B5
:1014000007F00AF917B0BDE8F08F062214A9484684
:1014100019F06AFD9DF847607FE7DAF80020536015
:1014200094F8372094F8363043EA02232B829BF855
:10143000E430628E0E92490961F3C5038BF8E43003
:101440000FF072FD0D909BF8E400C0F3C2000FF0A6
:101450006DFD0D9BB64A298A40F2E24808FB06F66C
:10146000034406FB03F303F5742303F23F23A2FBBB
:1014700003239B0C6B6294F83130AE4A08FB03F3F4
:10148000AB637308963BAB62B4F83880AA4B42F268
:1014900010703244B2FBF6F2ABF8C6201FFA88F2A5
:1014A00000FB02623344013A881DB2FBF6F2B3FB43
:1014B000F6F3ABF8C2209AB28242ABF8CE2004DD3C
:1014C000C1F57F41FA310A4492B2ABF8CA203946DD
:1014D00004220BF1E80019F007FD234613F81C2F36
:1014E000C2F34011DA070F910D9100F1F7804FF42C
:1014F0008073A3830A9B93F826000EF0E1FE014659
:10150000062204F12B00002900F0E08004F1240100
:1015100019F0EAFC0C9BFF2B04F1250000F0D980A8
:1015200014A9062219F0E0FC9DF84730A37749463C
:10153000062204F11F0019F0D7FC9BF8E430EA8979
:101540006286C3F3C2032A8AA28684F83830A4F8DC
:101550003680584609F096F82146A881E080DAF8EE
:1015600004400B9807F04EF8AB89E3801C232371ED
:101570000D9BD4F80080002B40F0BD809DF83C30DE
:1015800023772146404607F03DF807F045F895F8E7
:101590004500B5F84040B5F84270012100F0070061
:1015A0000FF0FCFA274407F5E177391881466348C4
:1015B00000273123CBF80830A1FB00015AA3D3E95F
:1015C0000023CBF80470CBF80C70FEF799FD6B6A22
:1015D0000E9ADAF80C4020F07F40F61A40F2E2430F
:1015E00003FB024402213A46CBF81000012002F02E
:1015F00003FF0A9D284607F0A7FF821C504B009569
:10160000D2B23846012104F02FFA04F2B244012884
:10161000A4EB09047AD00A9B93F82430DB0762D448
:10162000584609F02FF8DFF81491A6FB09863EA36F
:10163000D3E90023054631464046FEF761FDDAF85E
:101640000830CDF818B0A3F13A0A3E4B07933E4B51
:1016500005934FF4E4730893DBF81030049320F003
:101660007F473A480023A7FB000103930723B8EB09
:10167000000003FB071166EB01014FF47A720023AF
:10168000FEF73EFD28A3D3E90023CDE90170A4FBBA
:101690000901FEF735FD053520F07F40EDB20090E1
:1016A00053462A460121002004F054F930F0020389
:1016B00004D0274840F2C91101F0FCF801220221B0
:1016C000104602F099FE17B0BDE8F08F19F017FC34
:1016D00020E70622002119F012FC25E71C48F12121
:1016E00001F0E8F803E700230122009318461146B1
:1016F00004F0BAF994E76B7F43F040036B77384608
:101700000DF03CFE0123E88323773AE707F01AF84F
:101710000A9B83423FF47FAF0D4840F29F2101F0C6
:10172000C9F878E7AFF300808D49FD1A0700000083
:1017300083DE1B43FF5962027FC3C90100CA9A3B83
:10174000F1E90000DDE9000019EA00008D49FD1A09
:1017500008D50100000000002DE9F04F8BB0CDE965
:1017600004011F460020BDF860309DF85490BDF87C
:1017700058A0BDF85CB00393164608F01FF9002886
:1017800000F0BE8109F001080546404604F034FA35
:101790000290B8F1000F6AD1149B02993A46404674
:1017A00009F090FB002840F0BC812B6A05F11C0277
:1017B0000692002B62D02B6A1C6807F0010A93F88E
:1017C00044000293C0F3C00100F007000FF0E4F9F9
:1017D000029BB3F8401000F5E1700144B3F84200F9
:1017E0000144D948D6A3D3E90023A1FB0001FEF7A9
:1017F00087FC20F07F40206130460EF0EBFA95F830
:1018000033306FF3410385F83330FF2385F83430EC
:10181000002E00F07981A9F10203012B40F28581AD
:1018200095F84430149969F3420385F8443095F8EB
:1018300033306AF3000385F83330062205F12400C3
:1018400019F052FB039B2B8605F11C00DDE90423F4
:1018500000210096FFF7ECF80FF0FAFA002840F0AC
:101860007F812846FFF710F90BB0BDE8F08F062105
:1018700002F066FD00288FD11220F5E706F0AAFEDF
:101880000690002800F0988108F0F0FE0446002839
:1018900000F0A081203002F0F3FE04F11C030028C8
:1018A00040F07F81032104F1240007930FF05AF8E0
:1018B000606F079BA4F82CB04FF6FF72A4F82AA023
:1018C0002285002800F0748104F1640104F16802AB
:1018D000079302F041FDB4F860209C4B22F4EF62C4
:1018E00022F0070242F4887242F00102A4F860205C
:1018F00094F87A2022F0070284F87A204FF01B1225
:101900004FF0000BC4E916237F2284F8BD20C4F8F1
:1019100074B0A4F878B0A4F82EB0C4F830B004F1D4
:1019200034000DF0DFFC94F8392060F3050284F8F0
:10193000392001210DF127000FF014F89DF8271030
:10194000834AA08D84F83BB0A2FB0132D20802EB9F
:101950004202A1EB8202053284F83A2094F8392041
:10196000039BA4F8C4B002F03F0240F2E24184F8C5
:10197000392094F83C20A4F8C8B001FB0AFA754954
:10198000A4F8D0B022F00302514484F83C20B1FB0B
:10199000FAF1714AA4F8C61042F2107101FB03A1DA
:1019A00052440139B2FBFAF2B1FBFAFA0621A4F86B
:1019B000C01000F1060C91B26145079BA4F8CCB0B1
:1019C000A4F8C2A0A4F8CE1002DD0639091A89B223
:1019D00094F8E420A4F8CA104FF0000B22F007029C
:1019E00084F8E420A4F8F0B084F8F2B0C4F814B19C
:1019F000A4F818B1A4F830B1079306F001FA94F8EE
:101A00004A21069BC4F8543122F0030284F84A218B
:101A100094F87A20A4F848B122F0180284F87A20C9
:101A200094F87621A4F850B122F0070284F87621C8
:101A300094F8962184F853B16BF3451284F89621FB
:101A400094F8BE21A4F874B16BF3C302C4E94E014B
:101A500000210020C4E9500184F8BE21A4F894B10B
:101A6000A4F8BCB1A4F8C8B109F014FAA4F8D200E3
:101A700009F016FAD4F8CC11384AA4F8D4000A4078
:101A8000C4F8CC2109F012FA94F8D02160F30202D4
:101A900084F8D02109F010FA94F8D0211499C4F8F0
:101AA000D4B160F3C50284F8D02194F8D620C4F8EC
:101AB00004B007F0010A6AF3410284F8D62031220B
:101AC000A260C4E978BB0622C4E976BBC4F80CB0B6
:101AD00004F1DD0019F008FA94F8D620029969F3B0
:101AE000000284F8D62004F1D700062219F0FCF990
:101AF000079B2B62C4E905BB84F800B0E4615EE695
:101B00000C200BB0BDE8F08F0EF026FD00283FF44E
:101B100082AE1499384632460EF0B4FA85F8340095
:101B200079E60B200BB0BDE8F08F00200EF076F9BF
:101B300095F8333043F00203C14685F833306FE641
:101B40008D49FD1A0700000000CA9A3B4801480170
:101B5000ABAAAAAAFF5962027FC3C9010000FFF61F
:101B60002C6AA36D23B11E4840F2BC4100F0A2FED6
:101B700004F14C0104F1480002F0F2FB064618B3F0
:101B80002768A665D7F85441C4B1204606F028FD61
:101B9000384608F071FD002303202B620BB0BDE82E
:101BA000F08F0F480793BF2100F084FE079B79E672
:101BB00004F16C00606787E6072055E6084840F2AC
:101BC000C54100F077FEE0E7054840F2BE4100F075
:101BD00071FED5E7069806F003FD072044E600BF36
:101BE00050D50100000000002DE9F04F80468FB075
:101BF00004460F46154600F1240106220CA818F8E9
:101C00001C6F19F071F994F81C9018F0010FC9F3CA
:101C1000401BC6F3C016D94640F0F4800023A383CE
:101C2000B97C97F8118011F0010104F12B004FF0FD
:101C3000060200F0D18004F11E0119F055F9B8F147
:101C4000FF0F04F1250304F11F0A00F0CF80524674
:101C5000404604F11E010B930DF092FD0B9B1846BC
:101C6000A37F02330CA9A377062219F03DF93B6844
:101C7000D3F800A0EB8963862B8AA386BAF83030AC
:101C8000E3860FF04FF984F83800D5F8008040461D
:101C900008F0F8FC7E68A8812146E080206806F004
:101CA000B1FCAB89F3801C2334683371B9F1000FA8
:101CB00040F0AE8086F81CB03146204606F0A2FC0B
:101CC00006F0AAFCD8F80430D8F8086095F844006B
:101CD000B5F80E90FC689E4238BF1E46C0F3C001A6
:101CE00040F2E24300F0070003FB09F90EF054FF55
:101CF000203400220221241A012002F07DFB5046EC
:101D000007F034FE021D4A4BCDF800A0D2B20121EB
:101D1000002003F0A9FE30F0020304D0454840F251
:101D2000CD3100F0C7FD4FF0000A534603220121D8
:101D3000CDF800A0504603F097FE404608F0A2FC04
:101D4000BB68CDF81880093B9E1B3B4B07933B4B70
:101D5000059340F2FD333A4F0893D8F81030A9FBB1
:101D60000798CDE903A3451D2FA3D3E900234846D7
:101D70004146FEF7C5F9104619464FF47A72002322
:101D8000FEF7BEF928A3D3E9002302904146484656
:101D9000FEF7B6F924A3D3E900230190A4FB0701C1
:101DA000FEF7AEF9EDB220F07F40009033462A46B0
:101DB0000121504603F0CEFD30F0020304D01D484F
:101DC00040F2FE3100F076FD01220221104602F0C1
:101DD00013FB0FB0BDE8F08F19F091F8B8F1FF0FC9
:101DE00004F1250304F11F0A7FF431AF18460622DF
:101DF000002119F084F8A6770CA95046062219F0A4
:101E000073F834E70B484FF4537100F053FD05E7C6
:101E10006B7F43F040036B77281D0DF0AFFA012371
:101E2000E883337748E700BF8D49FD1A07000000BB
:101E300095EB000050D5010099EB0000ADEB0000E0
:101E400000CA9A3B000000002DE9F04186B005ACC5
:101E50000094039216461D46044604AB03AA0220D2
:101E60000DF064F9FF2830D0DDE90413244F0B4452
:101E7000A3FB07014FF0070808FB03111EA3D3E9DA
:101E80000023FEF73DF9803028600398831B1B0276
:101E90001ED4314603F08AFE0346A0FB070108FB6F
:101EA000031115A3D3E90023FEF72AF92A68024497
:101EB0002A60002A09DB40F2E24004FB00F0904275
:101EC00003D2121A8242FCD82A6006B0BDE8F08123
:101ED0000146304603F06AFE0346A0FB070108FBFB
:101EE000031105A3D3E90023FEF70AF92A68121AA1
:101EF0002A60DEE7AFF3008000CA9A3B00000000D2
:101F00008D49FD1A0000000010B584B003AC9C465A
:101F1000009402AB64460DF009F9FF2812D0DDE908
:101F200002210D480A44A2FB0001072303FB021112
:101F300007A3D3E90023FEF7E3F8803020600020F8
:101F400004B010BD6FF00900FAE700BFAFF30080E6
:101F500000CA9A3B000000008D49FD1A00000000F5
:101F60002DE9F041B0F8A41188B0044640F2E243F4
:101F70004748002603FB01F105AD0623C5E90166CC
:101F80008DF80F30A1FB00013FA3D3E90023059694
:101F9000FEF7B6F80DF10F0301950093B4F89A31EE
:101FA000049004AA204601210CF088FF9DF80F80C0
:101FB00008F1FF3C5FFA8CFC0DF11603304604F586
:101FC000D27703EB4C0C04F5D8764FF6FF7E3A88B7
:101FD000B8F1000F0AD02B46724504D019889142FF
:101FE0004FF001001DD002339C45F5D10237BE42AF
:101FF000EDD1D4F8F83048BBBDF8142040F2E241EE
:1020000002FB01F1100AC4F824111A70587094F8F8
:102010001A31042262F3020384F81A3108B0BDE8D1
:10202000F081D4F8F81040F2E24302FB03F3100A07
:10203000C4F824310A70487094F81A31042262F30B
:10204000020384F81A3108B0BDE8F081032203F8D6
:10205000042C13F8052C94F81A11052542F00302FC
:10206000112003F8020C03F8052C65F302010F2080
:10207000202203F8010C1A7084F81A1108B0BDE888
:10208000F08100BFAFF300808D49FD1A070000000A
:1020900000CA9A3B0000000038B504460FF006FD68
:1020A000A27DC2F34103013303F00303032B34D0B9
:1020B00063F34202A27503F125000EF037FD636859
:1020C0000BB32369FBB111F0A1FC054603F06CFDD5
:1020D000C11C002011F04AFC11F0E4FC11F096FC48
:1020E000294603F063FD124903460722A0FB0101C4
:1020F00002FB03110CA3D3E90023FEF701F82369C7
:102100001B1A236138BD03F04FFDC11C002011F0E4
:102110002DFCBDE8384011F0C5BC6FF34202A2753A
:102120002520CAE7AFF3008000CA9A3B00000000F8
:102130008D49FD1A000000002DE9F04F89B00446DA
:1021400011F02EF9C0B250B90EF03CFDB84821464E
:1021500010F06AFF09B0BDE8F04F11F0F5B811F0CA
:102160003FF9054611F06CFB834611F073FB814685
:1021700011F0B8FD064611F099FD824611F024FBDE
:10218000EDB2804611F0FEFA0EF01CFD002DDDD000
:10219000012006F085FB0546002800F085811BF034
:1021A000FF0BF6B240F07781002E40F0D380FF277E
:1021B0005A463B46314620460FF03CFE0028C5D02B
:1021C0002B7F626800218DF81B105FFA88F803F0FE
:1021D0000F01002A00F0DA80626892F82020900750
:1021E00000F1D4800729B1D0A27D120740F16281AD
:1021F000002940F0B5806B7F252B00F22A81042056
:1022000006F04EFB0028A1D011F054FC636A814611
:1022100043B9238C40F2712202FB03F3B0FBF3F2CB
:1022200003FB120923681A69824B0721A2FB0303EF
:1022300001FB02317CA3D3E90023FDF761FFA0F28B
:1022400042334B4582D311F08FFA636805933846C9
:102250000EF044F8E37D9B07814640F1CE810028D3
:1022600000F0CB8101464FF0010B049111F0C6F84C
:102270002B7F049907AA039205F11E02CDE901B153
:1022800082460146C3F380130092204600220FF0DD
:10229000EBFD504611F02AF811F078F8002840F0D4
:1022A000C1816548214610F0BFFEB8F1000F40F033
:1022B000BF816168A37D91F8202043F0800342F044
:1022C000010281F82020A37506F00AFB172380463F
:1022D00003714FF6FF732D7FC380514624221C30BB
:1022E00018F002FE98F81C30C8F80840C5F34015F5
:1022F00065F3451388F81C3011F088FB0021C8F8FD
:1023000010000120079D11F005F8002E08BFFF27DF
:1023100088F81970E37D2D1A13F00203C8F81450E1
:1023200003D0B9F1000318BF012398F81A2063F312
:10233000000288F81A2006F0D3FA03464146D8F87E
:102340000000C8F80C3006F0E1FA06F0EFFA09B028
:10235000BDE8F08F5FFA8AF00EF024F8074627E711
:10236000012915D16B7F0C2B7FF4F0AE2A7F0097EB
:1023700000230193D20905F1240320460FF0CCFC81
:1023800000287FF43CAF297F01F00F01002955D0D0
:10239000062953D0022900F0A080012959D16B7F72
:1023A0000C2B7FF4D3AE2A7F00970DF11B03019312
:1023B000D20905F12403002120460FF0ADFC0028CE
:1023C00047D06B7F002B3FF4C1AE63682BB12B7FEE
:1023D00003F00F03072B7FF4B9AE03209DF81B9089
:1023E00006F05EFA054600283FF4B0AE06F078FA33
:1023F0004FF6FF73EB8005232B71B8F1000F68D106
:102400007F20AB7E2876002E08BFFF2769F34103AB
:102410002868AB7629466F7606F078FA06F086FAD9
:1024200094E600BFAFF3008000CA9A3B00000000B2
:102430004D1B01008D49FD1AC91C01006B7F252B26
:1024400007D8A27D920602D56268002A47D0252BC4
:10245000B8D92B7F03F00F03042B7FF477AE6B7F8B
:10246000252B3FF673AEA37DD9077FF56FAE10F035
:10247000C5FF2B7F0278C3F38013B3EBD21F7FF429
:1024800065AE0830062205F11E0118F004FD002893
:102490007FF45CAE95E7A07D5FFA89F1C0F3C000E0
:1024A0000DF040FF074683E6674840F2C62100F082
:1024B00001FA74E6FF2F8DF81C70C3F3801978D0F1
:1024C000237EDB1BB3FA83F35B09002B7FF490AE12
:1024D0005CE711F06BF9C0B293E76B7FB7E796202A
:1024E00011F0CEF9002011F0FFF8032006F0D8F922
:1024F000814600283FF42AAE06F0F2F94FF6FF734A
:10250000A9F80630052389F80430B8F1000F70D11E
:102510007F23002E89F8183014BF3B46FF2389F82B
:10252000193099F81A30D9F800006FF3410389F88F
:102530001A30494606F0EAF906F0F8F910F05EFFA5
:102540002B7F0646C3F380133278DB0102F0700262
:1025500043F00303134333700C23384673700DF0BC
:10256000BDFEE37D9F074ED500284CD03378014651
:10257000304643F0400300F8023B062218F0B4FC5A
:10258000062205F11E0106F1080018F0ADFC3046E8
:1025900010F0ACFE10F0FAFE00284FD111F082FAD4
:1025A000A37D2A4843F00103A375214610F03CFDAA
:1025B000CDE605F11E0A07AA514648460DF070FF08
:1025C00000283FF4E0AEE37D03F001034B457FF4C8
:1025D000DAAE5146062204F1080018F05CFC297FAF
:1025E000B0FA80F35B0901F00F01002B7FF400AE1D
:1025F000CCE611F0DBF8C3B28BE7A27D04F1190140
:10260000C2F3801B31E6A37D3278C3F380133046DA
:1026100063F3861200F8022B04F11901062218F068
:1026200063FCADE7084840F29F4100F043F938E60B
:1026300011F0BCF8059B83F8A1003AE6024840F28D
:10264000245100F037F9A9E7C4D60100611B01004D
:1026500038B5094D4FF0FF324FF0FF33284618F0E0
:1026600018FD044601F0DAFD10B1204611F0C2FD5C
:1026700014F0F6FFEEE700BFA40A002010B50F4CDF
:10268000204619F067FEA0B1204618F057F8204602
:1026900018F05CF8A3682BB11B6E1BB1084900222F
:1026A00020469847A3681B6C33B104489847002024
:1026B00010BD6FF01500FBE71846F9E778CF010071
:1026C000C52600002DE9F047704CA568EB6C8CB076
:1026D0002BB12046984710B9204618F028F86B48CF
:1026E00018F025F860B16A4C2368A3B96948002244
:1026F000002318F0CEFC206068B9644818F026F872
:10270000EB6CFBB9644E654D3378032B1ED8DFE8C4
:1027100003F0203893AD236899689A89EB6A73B106
:102720005A48984701462068083018F005FD20688F
:102730008689002EE4D111F05DFD2660E0E76FF0A0
:102740005701F0E7514898470028DBD10CB0BDE8AD
:10275000F087534C4D480122214617F0E1FF002835
:10276000F4D02278531EDBB2012B01D9052ACBD13C
:10277000042B96BF4B4A0023D3562B6001233370A2
:10278000C2E7DFF81CA1DFF820919AF800303F483B
:10279000013BDBB2042B9CBF424AD1562A6888BF5A
:1027A0000021891A494417F0BBFF2F683F1A0446DD
:1027B0002F60002F56D10123CDE900A30022002372
:1027C000062001F0C7FCDFF8E480C8F8000008B973
:1027D0003070BBE79AF80030022B26D0052B1FD0B3
:1027E000012B25D199F802202A60013BDBB2042B92
:1027F00098BF2C4A2C4998BFD75608303A4618F053
:1028000089FCD8F80000083018F0A6FC2B68984224
:1028100010D2D8F8000011F0EDFC0323337021E052
:10282000B9F80220C2F30D02DEE7B9F80220DBE7B7
:102830003A46D9E70223F1E71C4F2A683B68134860
:1028400099899B68194417F06BFF39682F688B8949
:102850003F1A034404468B812F601FB9144818F0B7
:1028600036FC3770002C7FF44FAF6FE72A680748BB
:10287000212A28BF212203A917F052FF2B681B1A17
:1028800004462B60002BEDD1C8E700BF78CF0100D4
:102890009C2F0020BC0A0020D26D0020A02F002019
:1028A000D36D0020C8DE0100CE6D0020982F0020DF
:1028B000A40A002070B504460E464FF02002EFF344
:1028C000118382F31288BFF36F8F234817F036FF0E
:1028D000214817F03BFF002C37D125461E48042124
:1028E00017F031FF1C48FF2117F02DFFA91D1A48D2
:1028F000C9B217F028FF1848AA2117F024FF3DB1EC
:10290000154D013C14F8011F11BB134817F01BFFB4
:102910001148F1B217F017FF0F48C6F3072117F05F
:1029200012FF0D48C6F3074117F00DFF0A48310E9C
:1029300017F009FFFEE701332F2A08BF1D46E25CAE
:10294000002AF8D12C445D1BC8E700252B46F6E78A
:10295000284617F0F8FED5E778CF010070B5244877
:10296000244E8AB001F064FC04238DF820300E233D
:102970008DF8213003238DF82230002401238DF8B7
:102980002330ADF8244008AD15F8011B3046013462
:1029900017F0D9FE062CF7D100220023CDE906233B
:1029A00000236FF00802CDE90323CDE90133009342
:1029B0001149124B12484FF4806214F0D3F81149B8
:1029C0000F480B4D104E0B4C19F09DFD4FF0FF3290
:1029D0004FF0FF33284618F05CFB0146304618F0F4
:1029E00076FBA3685B6B002BF0D020469847EDE7A1
:1029F0008C0A002078CF0100206E002051260000B4
:102A0000580B0020BCDE0100BC0A00200B6801331B
:102A10000B60014B1B681847E8000020014B186051
:102A2000704700BFE800002007B50B4600210246B2
:102A30000191034801A900F0E5F803B05DF804FB3B
:102A40000D2A00002DE9F84FB0F8189019F0080889
:102A5000044693460DD001290CBF49F0100949F0F6
:102A60002009A0F818908BF31188BFF36F8FBDE891
:102A7000F88F09F00709022907D1204617F0C1FE97
:102A80000028F0D00128238B4ED16769218B002FBD
:102A900015DA256821F00701C4E9008841F0010139
:102AA00021830026218B01F0070ACA4502D0A368C2
:102AB000002B5AD10DB9002E71D0002356E001F041
:102AC00007035A1F012A1ED821F00701062B25688B
:102AD00089B2C4E900880AD13DB1638B2A461268E5
:102AE00001339BB2002AFAD1638341F002012183B2
:102AF000204617F086FE06460028D3D0238B43F0ED
:102B000020032383CDE7042B0CD121F0070189B2E8
:102B10002183204617F075FE05460028C1D041F0FC
:102B2000200121830025BCE7032809D1226923F075
:102B30000703166843F00603238300252F46B1E7F9
:102B4000042806D1226923F00703566843F00403E2
:102B5000F2E7052806D1226923F00703966843F0BF
:102B60000503E9E700252E46E8E7012341F00801C7
:102B700021838BF31188BFF36F8FFBB985BB16B12F
:102B80001F492046B0474FF02003EFF3118B83F32A
:102B90001288BFF36F8F238B23F008032383238BCB
:102BA000DA0625D523F0100323830121B4F8189009
:102BB00009F0070900297FF45EAF54E7A1680029F6
:102BC000DCD0D1F80090D1F804B03B465246204604
:102BD000D847B9F1000FD1D04946D9F80090F2E7B3
:102BE00029463B46524620462D6817F026FEC5E78B
:102BF00013F020011EBF23F0200323830221D5E719
:102C000067A801002DE9F04F91B08B4602909246E3
:102C10001C4600259AF8000008B928465FE32528DD
:102C20000AF1010707D0029B594698470028C0F2D5
:102C30005683013512E2182200210AA818F05FF924
:102C40009AF80130252B78D00022104696469446FB
:102C50001646394617F8013B2B2B00F09D8000F2F9
:102C60009480202B00F09B80232B00F09B802EB1C2
:102C70009DF8306046F004068DF83060BCF1000F1E
:102C800005D09DF8306046F008068DF83060BEF142
:102C9000000F05D09DF8306046F010068DF83060CA
:102CA00028B19DF8300040F020008DF830002AB1A6
:102CB0009DF8302042F040028DF830209DF8302001
:102CC00002F04400442803D16FF386128DF83020BF
:102CD0009DF830202A2B42F080028DF830207BD1E5
:102CE0009DF8312042F001024B1C8DF831201A78FA
:102CF0002E2A9DF831200CBF0121002161F34102F1
:102D00008DF8312074D15A782A2A6AD001330021F3
:102D10000A26184610F8012BA2F13007092F40F2BD
:102D20008E809DF830200E91C2F3400040EAD171B0
:102D300061F341028DF830205AE00AF102078DF864
:102D400033309DF83130D90740F1498154F8049B64
:102D5000B9F1000F07DA9DF8302042F004028DF837
:102D60003020C9F100095A0740F1428154F8048B20
:102D7000B8F1000F80F241819DF831306FF34103CB
:102D80008DF831304FF0FF3837E12D2B0CD0302B40
:102D90007FF46DAF01225CE74FF0010C59E74FF073
:102DA000010E56E7012054E7012652E70CFB020210
:102DB000303A33461E4616F8010BA0F13007092FB2
:102DC000F4D9994293D09DF830100D92D20F62F34E
:102DD00041018DF830108AE70B4600224FF00A0CB3
:102DE000E8E79DF8312042F004028DF831200233EB
:102DF0001F4617F8012B6C2A41D025D8682A2BD002
:102E00006A2A46D04C2A4CD01F4617F8012B9DF851
:102E100031308DF83320782A00F2D980572A4DD8E6
:102E2000412A03D0453A022A00F2D1809DF832307F
:102E3000042262F302038DF8323001239EE006FB88
:102E400001213039034664E7742A26D07A2ADBD17F
:102E50009DF8313006220DE05A78682A9DF831201D
:102E600006D1012161F3C6028DF831209F1CCCE709
:102E70001346022262F3C6038DF83130C5E75A7853
:102E80006C2A9DF8312001D10421EBE7134603227F
:102E9000F0E79DF831300522ECE79DF8313007224C
:102EA000E8E7BDF8303023F4F04323F0020343F4A5
:102EB000804343F00203ADF83030A6E7A2F1580199
:102EC000202900F2848001A050F821F0912F000009
:102ED000CF2F0000CF2F0000CF2F0000CF2F0000FA
:102EE000CF2F0000CF2F0000CF2F0000CF2F0000EA
:102EF0002D2E0000CF2F0000912F0000512F000039
:102F00002D2E00002D2E00002D2E0000CF2F0000B2
:102F1000512F0000CF2F0000CF2F0000CF2F000037
:102F2000CF2F0000992F0000912F0000B52F000037
:102F3000CF2F0000CF2F0000B52F0000CF2F0000B3
:102F4000912F0000CF2F0000CF2F0000912F000005
:102F50009DF83210012003F0780360F30201402B4A
:102F60008DF8321002BF9DF8301041F001018DF84C
:102F70003010632A31D1003B18BF01239DF8302067
:102F8000C2F340010B4363F341028DF83020D8E6D1
:102F90009DF832100220DEE79DF8322003F078031E
:102FA000A3F14000032161F3020243428DF8322075
:102FB0004341E3E79DF83220032113F0780F61F3DA
:102FC00002028DF8322014BF01230023D6E79DF8BA
:102FD000303043F001038DF830300023CEE79DF907
:102FE0003020002AB4BFDDF834904FF0FF39BAE644
:102FF0009B077FF5C7AEDDF838809DF831100023C0
:10300000CDE90D339DF8323003F00703012BC1F3F6
:10301000C30138D1CB1E042B22D8DFE803F003090B
:103020000921210054F8043BDA17CDE90A3206E001
:10303000073424F00704F4E80223CDE90A239DF8BD
:10304000303013F0030656D002983B46524659469C
:1030500017F0D9FE0028C0F242810544BA46D9E5EE
:1030600054F8043B01294FEAE372CDE90A3205D155
:103070009DF828300A9300230B93E0E70229DED164
:10308000BDF92830D0E7022B23D1CB1E042B13D857
:10309000DFE803F0030A0A12120022680A920023F2
:1030A000201D0B930446CAE7E01D20F00700F0E85E
:1030B0000223CDE90A23F5E754F8043B0A930129DA
:1030C0004FF000030B93D3D00229B8D1BDF82830BC
:1030D000D0E7042B09D1E31D23F0070303F1080413
:1030E000D3E90023CDE90A23A9E7032B04BF54F851
:1030F000043B0A93A3E79DF833007828AED86228F2
:1031000022D825283FF48FAD5828A7D10DF12603EA
:103110000093DDE90A0104AB0CAA17F02EFE8246EB
:10312000B8F1000F0DF126000CDB9DF83020A0EB6C
:103130000A036FF3861298458DF8302002D9A8EB68
:1031400003030D9380463DE06338152886D801A21D
:1031500052F820F0D5310000393200005D30000017
:103160005D3000005D3000005D300000393200004D
:103170005D3000005D3000005D3000005D3000001B
:103180009332000061320000653200005D300000C3
:103190005D300000AD3100005D30000061320000A4
:1031A0005D3000005D30000061320000B8F1000FBA
:1031B000DDF828A00ADB4146504617F057FE0AEB1F
:1031C00000080026BAF1000F0CD147E7504617F06F
:1031D00046FEF4E70A9B8DF8103000260DF1100A28
:1031E0000DF11108A8EB0A0306B101339DF8322056
:1031F000D00668D5023352060D9948BF0E9A0B448B
:1032000048BF9B18B9F1000F76DD9DF83020A9EB7F
:103210000309C2F38003039353076DD4500661D5AD
:1032200046B1029B594630469847002857DB039B1E
:1032300001351E46302356E01E070FD413F010064A
:1032400018BF2026DDE90A23002BBFF65FAF5242EC
:1032500063EB4303CDE90A232D2657E72B26F1E73D
:10326000002653E70A9840B30DF1260300930CAAF9
:1032700004AB002117F081FDBDF8323003F0EF03FD
:1032800043F4F04343F010038246ADF83230002699
:1032900046E70A9B07293FF6E1AEDFE801F00C04A0
:1032A000060C08080C0C1D70D8E61D80D6E6EA173F
:1032B000C3E90052D2E61D60D0E6DFF8C8A006469A
:1032C0000AF105088EE7110748BF013393E7184656
:1032D00003935946029B98470028039B04DA11B0D8
:1032E000BDE8F08F20234D444A46002AA5EB090192
:1032F00009F1FF39EBDC0D4636B1029B59463046E9
:1033000098470028EBDB01359DF83230D90601D40F
:103310001A0706D5029B5946302098470028DEDB65
:1033200001359DF83230DB0607D59DF83300029B4E
:10333000594698470028D2DB01350D9E2E44731B59
:10334000002B16DC029843465246594617F05BFDA7
:103350000028C4DB0544A944A9EB0503002B7FF733
:103360007DAE029B5946202098470028B7DB0135E7
:10337000F2E7029B5946302098470028AFDB013521
:10338000DDE700BFCDDE010008B54FF02002EFF30E
:10339000118382F31288BFF36F8F00F005FE03489C
:1033A00017F008FA00F032FAFCE700BFD3DE0100A4
:1033B0002DE9F84305464FF02003EFF3118683F320
:1033C0001288BFF36F8F0E4B1C689CB10D4FDFF856
:1033D00038804FF00C09D4E90132002D08BF1346A4
:1033E0002BB198F8142009FB02F2B85C98472468C6
:1033F000002CF0D186F31188BFF36F8FBDE8F883FE
:10340000A42F0020AC2F0020C0620020420901231D
:1034100000F01F0003FA00F0074BBFF35B8FC043BF
:1034200003EB820353E8002F024043E80021002908
:10343000F8D1BFF35B8F7047B82F002038B51A4B17
:103440001C7DBFF35B8F04F01F0301229A40174BD2
:103450006109D04303EB810353E8001F01EA000533
:1034600043E8005CBCF1000FF6D1BFF35B8F114263
:1034700013D00F4B0F4D8BB10C236343EA18E85C5C
:10348000517817F054FD0020FFF792FF0C235C43A6
:103490002A1900232B51C2E9013338BD83F3118867
:1034A000BFF36F8FEFE700BFC0620020BC2F00208A
:1034B0002FAF0100AC2F00202DE9F843324B334AE7
:1034C0001C7DBFF35B8F63094FEA830952F82330F9
:1034D0002F4EBFF35B8F04F01F0843FA08F313F07D
:1034E000010F07460AD10146204600F069F828B1CD
:1034F00007C80C2303FB046383E807000C23634322
:10350000F218F55C2DB92046FFF780FF2846BDE88C
:10351000F8837B1C0FD0D2F808C01E481E4A4FF417
:10352000004500210023ECFB0501FCF7E9FD01212A
:10353000381A19F0BDFA13F09BFE0120FFF738FF8F
:10354000BFF35B8F012303FA08F8144B994459E841
:10355000003F43EA080349E80032002AF7D1BFF3ED
:103560005B8F0F4B33B10C236343F218F05C51783F
:1035700017F0D1FCFFF762FF2046FFF747FF14F07A
:1035800047F80120C3E700BFC0620020B82F002029
:10359000AC2F00203F420F0040420F00BC2F002004
:1035A00017AF0100054BBFF35B8F53F82000BFF34B
:1035B0005B8F003818BF0120704700BFC02F00206C
:1035C0002DE9F04F85B00F4603A900F047F8DFF86A
:1035D0008080DFF880A0441E24B24FF0000B631CF3
:1035E00004D10026304605B0BDE8F08F039A04EB05
:1035F000440302EB830612F82300FFF7D3FF0546CE
:1036000010BB70684FF40049C4462946E0FB09C16D
:1036100052465B466046FCF773FD0190B068C446B5
:103620002946E0FB09C15B4652466046FCF768FD4F
:10363000094B1B68591C01D0834205D97A1CD1D093
:10364000019B1844B842CDD9013C24B2C7E700BF62
:103650003F420F0040420F00EC00002008B9024B2F
:103660000B600020704700BF68D10100014814F0D2
:1036700005BC00BF68D1010010B5044618B90D4B58
:103680000D485B689847616808290DD031F0040344
:103690000AD011F0020108D00848214618F004FFB2
:1036A000002323600023636010BD2068142217F0FC
:1036B00026FCF7E778090020FCDE0100DC2F002063
:1036C00008B508B34368042B10D101220368BFF387
:1036D0005B8F53E8001F002903D143E80020002836
:1036E000F7D1BFF35B8F0BD1002008BD53B1006849
:1036F0004FF0FF324FF0FF3313F0D8FA0028F3D029
:103700000348F2E70348F0E76FF4E040EDE700BF5D
:10371000E98FFFFFEA8FFFFF08B5D0B14368042BA4
:1037200011D100220368BFF35B8F53E8001F01290A
:1037300003D143E800200028F7D1BFF35B8F07488F
:1037400008BF104608BD3BB1006813F027FB0020FE
:10375000F8E76FF4E040F5E70148F3E7E98FFFFF92
:10376000EA8FFFFF10B5044618B9164B16485B6880
:1037700098476368042B23D0082B21D0CBB923684A
:10378000BBB912484FF0FF324FF0FF33214613F020
:1037900089F908B923681BB90A4B0D485B6898473B
:1037A00020681422002117F0AAFB636843F002038B
:1037B0006360206818F0BBFE636843F00103636038
:1037C00010BD00BF78090020FCDE0100DC2F0020C6
:1037D00022DF010008B5064906484023142218F0EC
:1037E00048FEBDE808400449044814F0FBBB00BF94
:1037F000F82F0020DC2F002080D1010070D10100C3
:10380000014910220A60704710ED00E072B6404096
:1038100080F31188BFF36F8FBFF34F8F30BF62B655
:10382000BFF36F8F704700BF72B6494081F31188B4
:1038300020BF80F3118862B6704700BF43B2002BEF
:1038400008DB012200F01F0002FA00F05B09024AC7
:1038500042F82300704700BF00E100E043B2002BB4
:103860000DDB01225B0900F01F0002FA00F020339B
:10387000034A42F82300BFF34F8FBFF36F8F7047A7
:1038800000E100E0054B420900F01F0053F8222040
:10389000012303FA00F01040704700BF00E100E090
:1038A00043B2002BA8BF03F1604301F10101B8BF8F
:1038B000064B4FEA4111ACBF03F5614300F00F0026
:1038C000C9B2B4BF195483F80013704714ED00E077
:1038D00008B572B6044B9A691AB100229A6118F0C1
:1038E00017FE62B608BD00BFC062002030BFFFF700
:1038F000FDBF00BF0B4A08B50B4B22F07F029A6058
:10390000BFF34F8FBFF36F8FD3F8882022F470027C
:10391000C3F8882012F0E4FF13F0AEFF00F0D0F9F6
:1039200013F022F80000000000ED00E0094A0A4907
:1039300093680968D967094998674B6843F08053D1
:103940004B60002383F31188BFF36F8F9368D86FA8
:10395000704700BFC062002030DD010000ED00E0D4
:1039600012498A684FF030001044EFF3098C80E868
:10397000F01F202080F31288BFF36F8F0C4F4FF0A1
:103980000066CA698A603E60906F0023936780F387
:10399000118804B5104600F02FFABDE8044002F18A
:1039A000300090E8F01F8CF309887047C062002057
:1039B00004ED00E01EF0040F0CBFEFF30880EFF3FE
:1039C0000980816911F8021C0229FFD001B517F0A6
:1039D00037FA01BD42F8203C009B42F81C3C0A49E2
:1039E000019B42F8183C029B42F8143C21F0010173
:1039F0004FF0807342F8043C42F8081C0023203A40
:103A000002658367704700BFDBA90100094A0346CE
:103A1000906870B113F1160F806E05D0A0F12002EE
:103A20009A4205D8834203D2814228BF00207047C2
:103A300000207047C062002008B5094B98600D4611
:103A4000144600F0D9F9204685F30988002163B6B1
:103A500081F31188BFF36F8F0022002316F0BDFFA2
:103A6000C062002001B572B60B4A906900281EBFE3
:103A70000021916118F04CFD62B6EFF30580A0F1D2
:103A800010004FEAC0000549014409C99847BDE844
:103A90000140034908470000C062002090CF0100A8
:103AA000A53A0000044B9968D869884203D00349BD
:103AB0004FF080520A607047C062002004ED00E0C1
:103AC00038B51C4B14469A6A9A6A9A6A054690075A
:103AD00020D5586B9A6A12061CD519B19A6A22F041
:103AE00080029A629A6A9A6A9A6AD20615D49B6A86
:103AF0009B0712D400200F4B9A6A920642BF5A6A63
:103B000022F400525A629A6A42F0FF029A6200233B
:103B1000237038BD6FF01500E4E7064B5B681905AC
:103B2000E8D52946FFF772FF0028E3D080F3098823
:103B30000220E0E700ED00E00D4B9A6A9A6A9A6A6B
:103B4000920508D59A6B9A6A120404D518B19A6A3C
:103B500022F400429A62064B9A6A9A6AD20558BFCA
:103B60009A6A9A6A002042F47F429A62087070470B
:103B700000ED00E070B5484B5B688AB00D46C3F3BA
:103B80000803002686F31188BFF36F8F02F07F4190
:103B9000B1F17F4F11D102F00C0108290DD01107AE
:103BA00001D4054601260022033B8DF80720032B94
:103BB0006BD8DFE803F00455595D3546F3E7364B23
:103BC000DC6A14F0020460D1DA6A002A15DBDA6AD2
:103BD000520012D5AA6932F8021C4DF602729142C7
:103BE0000AD093F828200AB30DF1070201212846D4
:103BF000FFF766FF044600E02C689DF807309BB98C
:103C00002022294602A817F06FF9099B002E3ED00A
:103C1000C3F3080222B96FEA53236FEA43230993DF
:103C200002A9204617F00AF90AB070BD93F82920BE
:103C30002AB10DF107010120FFF77EFFDAE75A8D67
:103C400092B2002AD9D09A6A9A6A9A6A9A6A9A6A49
:103C50009A6A9A6A6FEA02426FEA12429A62CCE763
:103C60000DF107020021C2E70DF107010020E3E793
:103C7000094B9A6A9A6A9A6A9A6A9A6A9A6A9A6AD4
:103C80006FEA02426FEA12429A620024B5E723F417
:103C9000FF7323F00103C2E700ED00E0024A53691D
:103CA00043F010035361704700ED00E0EFF308802C
:103CB000EFF3098101B57246FFF75CFF01BD00BF5C
:103CC000044800232021C2180133302B82F800134E
:103CD000F9D1704700E100E0002080F31488BFF3C1
:103CE0006F8F19F0A3F800200D490860BFF34F8FC4
:103CF0000C4880F3088800F02BF8202080F311880E
:103D000009484FF40261401880F30988EFF31480EA
:103D10000221084380F31488BFF36F8FFFF7EAFD99
:103D200094ED00E0407B0020C07C00200749D1F8E2
:103D300090200023C2F307221846934200D1704717
:103D4000C1F89830C1F8A0000133F6E700ED00E0BB
:103D500008B572B6002383F31388FFF7E7FF144B0F
:103D60004FF0FF32C3F88020C3F88420C3F88820C6
:103D7000C3F88C20C3F89020C3F89420C3F898208F
:103D8000C3F89C20C3F88021C3F88421C3F888219C
:103D9000C3F88C21C3F89021C3F89421C3F898216B
:103DA000C3F89C2162B6BFF34F8FBFF36F8F08BD7E
:103DB00000E100E0084B9B6883420BD1EFF30583E1
:103DC00043B1064B5A6842F080525A605A6A22F454
:103DD00000425A6213F0ECBCC062002000ED00E02B
:103DE000024B034A0348012100F06EB80000042092
:103DF0000000002094D10100826E054B203A1A6029
:103E0000044A2021C3E901121846012100F066B8D6
:103E1000F834002000000B15F0B51F4F00268E422D
:103E200001DB1046F0BD44689CB353B104F1FF3C84
:103E300014EA0C0F18D11F2C16D905681CEA050FBF
:103E400012D1202C0568D0F808C0D2B20FD9B4F135
:103E5000004F0ED8013CB4FA84F4C4F11F0464008E
:103E6000072A4CEA040406D96FF01502D9E70824A2
:103E7000F6E73E24F4E725F01F05154345F010054D
:103E800044F00104C7F89820C7F89C500132C7F8E5
:103E9000A04001360C30C2E700ED00E0044B0522E3
:103EA000C3F89420BFF34F8FBFF36F8F704700BFED
:103EB00000ED00E0BFF35F8F024B0022C3F89420B7
:103EC000704700BF00ED00E010B5034C01232278DD
:103ED000FFF7A2FF207010BDD46D002008B5094A7D
:103EE00000231278FFF798FF10F1160F02D0064A50
:103EF000072800DD08BDC2F89800C2F8A0300130E4
:103F0000F6E700BFD46D002000ED00E0144908681A
:103F1000082810B521D8FFF7CDFF124C49680022C0
:103F2000904201F10C0105D10F4B1870FFF7B6FF5D
:103F3000002010BDC4F8982051F80C3C23F01F035A
:103F4000134343F01003C4F89C3051F8043C43F091
:103F50000103C4F8A0300132E2E74FF0FF30E8E798
:103F6000A0D1010000ED00E0D46D0020014B1860ED
:103F7000704700BF100100204FF02003EFF31182C3
:103F800083F31288BFF36F8F06490123C1F84035D0
:103F90004FF08041C1F8783582F31188BFF36F8FFD
:103FA0000020704700E001404FF08043C0B2C3F8EA
:103FB0001C05BFF34F8F0549054BCA6802F4E06248
:103FC0001343CB60BFF34F8F00BFFDE700ED00E070
:103FD0000400FA0520B1034B800143F001031847A8
:103FE000704700BF60D1010010B518F08DF804468D
:103FF000094816F0DFFB0948214616F0DBFBBFF34A
:104000004F8F0749074BCA6802F4E0621343CB6045
:10401000BFF34F8F00BFFDE75EDF010087DF0100C8
:1040200000ED00E00400FA05F7B52F4D0026EF88FB
:104030002C68204618F08EF9002851D02B7A297967
:10404000002B14BF4FF4D0124FF4B01220463A4365
:1040500016F073FF044658B901360E2E05F10C0513
:10406000E5D1224D284618F075F920B96FF0040407
:10407000204603B0F0BD1E4A0221284616F05DFF1F
:104080000028F3D11B491C4BAC684B6004238B60A8
:10409000E369002BEAD00122284698470028E5D1A1
:1040A0002E69A469336813F0040F0CBF4FF08063CE
:1040B0004FF000734FF0A07202212846A04704463B
:1040C0000028D3D1AB6801A95B682846984720B97E
:1040D000336801985840C0F380000028F2DCC7E73D
:1040E0006FF01204C4E700BFC0D1010000CF01008F
:1040F0002000010004350020E93F0000074A034684
:10410000106828B9D96831B1596921B11360704775
:104110006FF0770070476FF0150070471035002082
:10412000052870B5054611D8012606FA00F414F0EA
:104130002A0409D0064816F0A7FF044620B13146EC
:10414000083016F0C0FF2575204670BD0024FBE73F
:104150002C0B00202DE9F0410228DDE90667054619
:104160002AD0062802D048B300242EE01849097846
:104170000129F9D13578012D1BD0022DF4D1154834
:104180000136013F16F080FF04460028ECD000F114
:1041900008080121404616F096FF2575AEB1A7B17B
:1041A000404616F0D9FFB8420AD2204610F022F855
:1041B000DAE709480025E3E70648E3E70648E1E7D0
:1041C0003A463146404616F0A5FF2046BDE8F0814C
:1041D000E8090020D40A0020000B002010B50D4B88
:1041E0001B78012B04460CD1037D012B04D0032B3B
:1041F0000ED06FF0150010BD042104F1080016F078
:1042000092FF054B2146186816F061FF0020F2E787
:104210000221F2E7E80900201435002083891BB150
:10422000024B1B685B69184712207047103500204D
:10423000044B054A1B6810600BB1DB6818476FF030
:104240001200704710350020143500202DE9F04190
:104250001646C21D22F00302751E0F46ADB218604D
:1042600082B0044616800021042207FB050016F0E8
:1042700046FEBDB1023EB6B206FB077306FB07F869
:104280001C44A8EB03080025042204EB08000DEBF6
:104290000201019416F028FEB542A4EB070405F1D3
:1042A0000105F1D102B0BDE8F08100BF70B505682D
:1042B00082B095B1EB1D23F0030304220446294686
:1042C0000DEB02001E8816F00FFE019B23B1DA1DD4
:1042D00022F00302013E16802360284602B070BD22
:1042E0000B6870B50C46054683B1073323F0030312
:1042F0001E880136B6B204222146284616F0F4FD87
:10430000EB1D23F003031E80256070BD0126F2E73C
:1043100002FB0100704700BF401A90FBF2F080B230
:10432000704700BF531E11449BB242B1DB430138BA
:10433000CA1811F8013D00F8013F9142F9D17047C8
:10434000014402E010F8013B1BB98842FAD1002079
:1043500070470120704700BF10600860704700BFC1
:104360000A6803460068904205BF00220A600020E8
:104370001A607047D2F800C0CCF80000D2F800C034
:10438000CCF8041010607047884203D01AB143681B
:1043900013607047002070470B68834209D02AB130
:1043A000586810601A680A6018467047002BF9D1E7
:1043B000FAE70023F8E700BF2DE9F041DFF830808D
:1043C0000C4E0C2706F130044546221D2146284696
:1043D0000C3CFFF7C1FFB442A5F10805F5D1043F3D
:1043E0003B1DA8F12008A4F13006EBD1BDE8F08117
:1043F000903500202036002010B40346154C8C4622
:1044000092B100EB40010CEB4C00000100EB81018C
:104410002144487A0C7AA04204BF0130087210BCD3
:10442000614618460FF08ABC01EB4102120100EB15
:10443000400302EB830323449C7ADA7AA24201D040
:1044400010BC704701329A72034B01225A5410BCBF
:104450000FF0B2BC9C3500209835002070B582B0BA
:10446000064601911C460D462AB322786378D21A7B
:1044700012F0030205D0012A42D00133DBB22370CF
:104480000FE00133DBB230212370042311FB05312F
:104490001C4A60680C2313FB06131A442146FFF7DD
:1044A00069FF194B012230465A5529460FF084FC0A
:1044B000002002B070BD0FF069FC0028D5D029465D
:1044C00030460FF04FFC0028CFD005EB450212011B
:1044D0000C4906EB460302EB83030B449A7ADB7A22
:1044E0009A42C2D122786378D21A920702D002335C
:1044F000DBB22370D4E902039847002002B070BDFC
:104500001046D6E79C35002098350020504A135CB1
:10451000002B00F09B802DE9F04F00234D4F1354EA
:1045200087B01A464FF03C0BCDE901200BFB007B16
:10453000039300EB40030BF1040807EB03174FF064
:1045400003090023D7E9090105AA0593FFF71CFF1A
:1045500007F124068346002834D0059C637825782B
:10456000ED1A05F00305012D06D1013B6370D4E976
:1045700002029047059C63782078C31A03F0030376
:10458000012B4FF0000231465FFA80FA0FD0B86A73
:10459000FFF702FF94F801C02378C4F804B0A3EB3E
:1045A0000C0303F00303012B84F801A046D0D7E9E4
:1045B000090105AAFFF7E8FE012D009083462BD0E4
:1045C0000028CAD197F82E3097F82F209A4203D0AE
:1045D00087F82F300123019397F82C3097F82D207E
:1045E0009A4203D087F82D300123039309F1FF3954
:1045F0005FFA89F9B9F1FF0FA7F10C07A1D1DDE945
:10460000013AC3B1039BB3B91A465146504607B0AD
:10461000BDE8F04F0FF092BBB9F1000F01D10028B7
:10462000D0D0DDF808A00A4A012302F80A3051462A
:1046300050460FF0C1FB07B0BDE8F08F424621465F
:10464000584684F801C0FFF795FEB0E7704700BFF9
:10465000983500209C3500204B1EDBB271B1411E05
:1046600000EB030C002011F8013F23B15A1E01306A
:104670001340C0B2FAD16145F5D170470846704782
:104680002DE9F04FA24D83B00746032601240421F3
:1046900038460CF067F938684FF000084FEAD07ED2
:1046A0001E234FF0010AC346C1461AE008F101017A
:1046B0000E2BC9B25FFA83FE40F29980D2B39646C0
:1046C000CC461C2B40F2A2801B2B40F20F811929F3
:1046D0003BD088469246BCF10C0FE14635D0013BF9
:1046E0003BD320FA03F202F001027245DED10AF157
:1046F0000102072BD2B240F2DD80062A40F2D480BC
:10470000BEF1000F51D004FA03F220EA0200CC46B9
:104710004FF0000E08F101010E2BC9B288BF012233
:10472000D5D8E14500F0BD8019290ED088464FF05C
:10473000010AD4E7CC460122052B40F28680062AE6
:104740004FF0000EBDD11929C3D1013304FA03F390
:10475000BEF1000F3DD05B42184080EA0503019393
:104760000DF1040C0DF1080E00221CF8013B23B1E1
:10477000591E01320B40D2B2FAD1E645F5D1012AD9
:1047800009D983B2B3EB104F4FEA104224D1C3B220
:10479000B3EB106F20D1013E16F0FF067FF477AF28
:1047A0006FF00D0003B0BDE8F08F04FA03F2104380
:1047B0004146CC464FF0010E8845ABD00E2B8AD82F
:1047C000E1458CD141460CF1010C5FFA8CFC52465C
:1047D0007DE7013B1843C0E7C0F30721130A387097
:1047E00000207970BA70FB7003B0BDE8F08F09F15A
:1047F000010CBEF1070F5FFA8CFC1DD912B9964669
:1048000001225EE7012907D0964660E700297FF480
:104810005BAFBEF1000F37D004FA03F2072B20EA9A
:10482000020088BF4FF0000EC6D80BF1FF3B5FFAC5
:104830008BFB4FF0000EBFE7002A3FF47CAF0BF17B
:10484000010B5FFA8BFB96463EE7BBF1000F0BD0E6
:10485000042B3FF674AFBBF1010F05D9032B3FF6D4
:104860006EAFBBF1020F09D804FA03F210430BF14B
:10487000010B5FFA8BFB4FF0010E9DE7062A0DD06E
:1048800011B14FF0000E1FE704FA03F2072B40EAC4
:10489000020088BF4FF0010E8ED8E8E74FF0000EFF
:1048A00015E74FF0010A8EE7BEF1000F12D1414625
:1048B000CC4641E7BEF1000F1FD00BF1010B062AD9
:1048C0005FFA8BFB0BD904FA03F220EA020041469F
:1048D000CC46AAE7062A18D14146CC46F9E6FBD0D9
:1048E0004146CC46B8F1000F96D0EDE601293FF6DF
:1048F000EEAEBEF1000FC7D08EE7062AD7D904FA74
:1049000003F210434146CC46B1E74146CC46D8E6D7
:10491000D6BE898E30B5437F0568FF2B14D003EBDC
:1049200043028B4205EB021228D04FF0000C01E04D
:1049300099420BD09E4613789468FF2B03EB4302F9
:10494000A44405EB0212F3D1002030BD714518D00C
:10495000137890680FFA8EFE0EEB4E0E4FEA0E1E85
:1049600005F80E301378FF2B06D003EB430305EB5D
:104970000315AB680344AB60604430BD9E464FF006
:10498000000C13784377E4E7A2EB010C1CF4000F52
:1049900010B4836844690AD12CF07F410B44A342D0
:1049A00014D91B1B002110BC836041617047891A18
:1049B00021F07F418B4206D82144C91A002310BC44
:1049C0008360416170475B1AA342EAD8E11AF5E7B8
:1049D0002DE9F04F87B00346427A019000680290BB
:1049E00058680590002A00F0F480531EDBB200EBFB
:1049F000C3030F460393039B5A685E780492FF2F0C
:104A00005ED007EB4704029B4FEA041AB84613F83E
:104A10000A7003EB04140025019B4FF0FF0984F892
:104A20000090D3F800E05A7F0EEB0A0B4A45DBF802
:104A300008100FD1C8E0091A06D1BBF81EA0BCF8B7
:104A40001EC0E24500F286801EF80330FF2B91461F
:104A500072D01A4602EB42030EEB031C1B01DCF87A
:104A600008008842E7D9B9F1FF0FCBF808108BF89E
:104A7000002066D1019B83F81D80FF2A08D002EB3D
:104A800042020EEB021EDEF808305B1ACEF8083048
:104A9000A37801336370002DB1D04FF00002EB6AB0
:104AA0002A700022AA6213B1296B104698476368E6
:104AB000002BA4D1D5E90B23FF2FC4E90823A0D1F3
:104AC000039B9878B0422FD0DDE903B906EB46028C
:104AD00006EB82029BF8001019F822300136F6B27C
:104AE000B14208BF0026042B09EB82051AD195F8C4
:104AF0000180029908EB480301EB03144FEA031A03
:104B0000A17863785B1A13F0FF0325D04FF0000300
:104B100009F82230EB6A0120A8620BB1296B984793
:104B20009BF80200B042D1D1039A05999142A2F1BB
:104B300008034ED003935EE7CBF808108BF80030E3
:104B40001A460FFA89F909EB49094FEA09190EF8D3
:104B5000098092E7014686E7AA8A0199D5F8249050
:104B60004969D5E903EC4FF6FE708242C4F82890FB
:104B7000C4F804E0C4F820C024D04FF6FF73D31A61
:104B8000B3FA83F35B0984F82C304FF6FD739A4235
:104B900088BF0022AB69A361EB69E3602B6A2361E4
:104BA000AB68A3600023A28363616A6820469946CC
:104BB000FFF7EAFE4FF00103C4F82490A4F81E901A
:104BC000E37029E71A46E5E70EF80A2083F81D800E
:104BD0005EE707B0BDE8F08F2DE9F04F827F8FB020
:104BE00001230692C377002A5BD1437FFF2B8146C6
:104BF00056D00EF0B1F9D9F8142099F81C3099F874
:104C00001D80801AFF2B20F07F4700F03C81D9F8EF
:104C10001830BB4294BF002301230393B8F1FF0F68
:104C2000D9F800B000F045814FF0000ACDF810909F
:104C300008EB48080BEB08144FEA0818A368BB42BE
:104C400037D8A1781BF80880FF1A9A4463785B1A5A
:104C5000DBB2012B2AD1A669002E54D0039B002B76
:104C60004CD0E38B0593A36A3BB11A681AB11A7A48
:104C7000002A00F0EF8000221A72059A94F82C00A6
:104C8000013292B2E28378B1A08B90420CD2002B19
:104C900000F0FC801A7A012A06D04FF0010C36E0B1
:104CA000C2770FB0BDE8F08F0139A170B8F1FF0FE6
:104CB000BED1DDF81090514699F80B3099F80A20D2
:104CC0009A420AD10132D2B2022A1CBF134606937D
:104CD000069A89F80B2008BF002309EB8303D9F853
:104CE0002440D960002289F81F204B46012204216C
:104CF0000320A4460FB0BDE8F04F604794F92D3073
:104D00000793803341D1A36AF3B14FF0000C002226
:104D10001A72E568481E59685A60A070002DC5D007
:104D2000049B60695B69626A2669AAEB000018440B
:104D300020F07F40E378BCF1000F16D0CDE90036BB
:104D40004FF6FF73A847B1E7E5680139A170002D60
:104D5000ACD019466369626A2669AAEB0300049B1A
:104D60005B691844E37820F07F40B4F81EC0CDE9B9
:104D700000366346A847A369002B039B18BF012395
:104D800003930023E383E37090E7B8F1FF0FBAD0F9
:104D9000E28BA38B656805929A4228BFD21A02FB68
:104DA000055008900798CDE90A17121ACDE90CA80A
:104DB00043460992A0464FF0000C2C461BB203EB71
:104DC00043030BEB03121B01D2F808E0F4446645E1
:104DD00039D3916999B3D18B908BD2F8049092F921
:104DE0002D7081420D4628BF0D1AB9F1000F3ED03B
:104DF000A9EB0E0EBCB309FB05EEDDF82090F145E2
:104E00008CBF4FF0010E4FF0000E34BF4FF0010980
:104E10004FF00009814292F803A098F803200ED3C6
:104E2000924529D817F1800F26D0099AED1B95429B
:104E300002DDBEF1000F1FD0079ABA4219D01BF84D
:104E40000330FF2BBAD14446DDE90B7A0A99DDF82D
:104E5000348058E7A28B059882423FF60CAF4FF0A2
:104E600001021A7209E74FF0010EA146D2E7CE46C1
:104E7000C0E7B9F1000FE2D04446DDE90B7A0A99A8
:104E8000DDF83480EFE6069B0393C7E6E568013959
:104E9000A170002D3FF40AAF19466369626A266962
:104EA000AAEB0300049B5B69184420F07F40E37881
:104EB00044E700231946FFE6C37F002B40F0298416
:104EC0002DE9F04F827F8DB08346002A7DD1837A11
:104ED000C17A01208BF81E009942DBF8140007907C
:104EE00000F03D840133DBB2022B08BF13460BEB0D
:104EF00083028BF80A309BF81D30D2680993079B18
:104F00000392134423F07F439BF80920CBF814301D
:104F1000DBF800300093DBF804300593531E069253
:104F2000DBB2002A00F0CE8101220B92059A02EB3F
:104F3000C30900230893FF230193CA46DAF80480CB
:104F40009AF803C09AF80270674537D09AF80020A3
:104F50007B1C3EB2DBB29A4208BF002306EB46023E
:104F600006EB82068AF8023018F82600042808EBBF
:104F7000860434D908285CD86178009A01EB410591
:104F800002EB05156A7895F802E0A2EB0E0212F02A
:104F9000FF0226D106284CD19BF81C308B422AD028
:104FA000002008F82600E36AA0620BB1216B984745
:104FB0009AF803C09AF802706745C7D1059A52451E
:104FC000AAF108036CD09A46B8E7446A0421034664
:104FD00001220420A4460DB0BDE8F04F60471F46F3
:104FE000B2E705283ED0012A32D0062848D19BF8E6
:104FF0001C308B42D4D1FF238BF81C3018F826309C
:10500000062B00F04181082B00F03E810DF0A4FF3B
:10501000DBF81420831A1D0200F13D81039A23F06E
:105020007F431344DBF818209A4288BFCBF818302E
:10503000B6E7002208F82620E26A0120A062002AD2
:10504000CDD0216B90479AF803C09AF802707BE7A5
:105050000628A1D05846FFF75DFCAB78A8606B70BE
:10506000617899E7606848B9A06838B9E06828B9FC
:10507000206918B9606930F07F40DAD0012A6AD01F
:1050800004215B460122DBF824400846A047059A2C
:105090008AF80270012352450893AAF1080392D1BD
:1050A0009BF81D30099A9B1A18BF012306930B9B8E
:1050B000002B40F00B8101995846FFF789FC9BF8C3
:1050C0001D300093009B099A934200F00C83089BCB
:1050D000002B00F086829BF81D300093009BFF2B75
:1050E00000F06883099BFF2B00F06F83009ADBF8C8
:1050F0000030714E02EB420203EB02130A279D6857
:105100000DF02AFFDBF81440031B23F07F43033329
:10511000AB422CBFE418641924F07F44DBF828303C
:105120008046204698470DF017FFA0EB080323F0B8
:105130007F43A4EB0804033324F07F44A34207F128
:10514000FF3740F2D782002FDAD14FF41461304696
:10515000FDF7B0FBD4E75846FFF7DCFBDBF8143073
:10516000A860074602930DF0F7FE029BC21A039B4C
:1051700022F07F42D1188F42814640F295806B69C0
:1051800004937A1AD5F804C0BCF1000F51D0A38A59
:10519000002B4ED0013B9FB29445EB8BA78223D2CC
:1051A0000CF1010ECDF818800A9418E0696ADFF856
:1051B0000C81434C8844A04584BF01F1E87101F59E
:1051C000D43170462C6A94BF604601F5A571013B4D
:1051D000121A091B9BB294456962EB8301D29F426C
:1051E000E4D3DDF818800A9C9F4221D90CF101001C
:1051F000D5E908E106900A9405E001339BB26046C8
:105200009F42024411D02D482D4C71440818A042F1
:10521000F3D801330698A1F1E8719BB2A1F5D4311E
:105220009F42A1F5A5710244EDD10A9C6962EF830A
:10523000AF836168A068049B0A44AA60AA6A034419
:105240006B611AB113680BB1091A51604A46029991
:105250002846FFF799FBE268AB6913442269934241
:105260008CBF9B1A0023AB61A37D03B1EB70E37D80
:1052700013B1013B85F82C30019B2B706B78627861
:10528000019201336B708BE66068DBF81420831A9F
:105290001D027FF5C3AE131A039A23F07F43934296
:1052A00034BFD31A0023BDE66B69DA1B531804938D
:1052B0006B61002266E700BF98D201005A2B17FFEE
:1052C000592B177F069B0893FF2301930DF044FE93
:1052D000079B9BF81D60C31A23F07F430493FF2EA6
:1052E000DBF8003000934FD0DFF89082DFF8909227
:1052F000039F4FF0000A009A06EB460302EB0314EB
:105300001B010293A3689F42C0F04682049AB4F83E
:105310001EE0DDF808C0D21A0492DBF81820934290
:10532000A7EB03079A4425BF4FF0FF338BF81C30DF
:10533000D31A0023CBF81830A2786378A069A16A49
:1053400065689B1ADBB20593009B13F80CC018B17B
:10535000059B022B00F035810023A3608BF81DC054
:10536000002D40F0DA8019B1097A012900F011818D
:10537000059B23B1012B45D0BEF1000F42D16270D5
:105380009BF81D60FF2EB6D1069B099A01999642A3
:1053900018BF012358460693FFF71AFB9BF81D30F0
:1053A000DBF800A0CDE9003B0022009BFF2B0FD0D3
:1053B000009E33B203EB43030AEB03151B01AF6AF4
:1053C00017B1397A012925D01AF80360FF2EF0D1E0
:1053D000DDF804B0002A3FF475AE009B09998B42BA
:1053E0007FF475AE089B002B7FF478AEDBF80430B9
:1053F00001939BF809305F1EFFB2002B3FF46EAEA5
:105400000692FAE0236A002BB9D0616A012098471E
:10541000A278B4E7019B1B7FFF2B4BD0019B039A23
:105420009B69934246D9A3EB020C7A68AB6895F866
:1054300000B0D31A02933B689A4280F0BD80BBF162
:10544000FF0FA3EB020800F0B780D5F818E0F04595
:105450004FF0000331D3F1465A461C461CE08168E8
:105460000B1F0429234409D9434528BF43469945C6
:1054700004D2B3EB0E0301D09C451ED983691AF800
:10548000022001EB030C0C44A8EB0E03FF2A04EBF3
:105490000E0912D0C84510D302EB42020AEB0210EB
:1054A0001201816A0029DAD0097A0129D7D11AF8C4
:1054B0000220EBE74FF0000CB7E7029A1A447A603B
:1054C0005C46AB604FF0FF0E00E0144621B201EBEA
:1054D00041020AEB021C1201DCF80800834240F290
:1054E00051811B1AAB601AF80220FF2AA646ECD1A4
:1054F000019BCDF800B001EB4101090183F81DB01B
:105500001AF801302B700AF80160EB8B013BEB833A
:105510004FF002033B72012247E711B10B7A012BD6
:1055200037D0BEF1000F59D1B4F81CE07246681CA8
:10553000D4E908C30021059004E02846013A01445B
:10554000501C0FD0634403EB08004845F5D805987C
:10555000A3F1E873013AA3F5D4330144501CA3F539
:10556000A573EFD194F82C206362002A00F0D2805A
:1055700000227244A160E2830DE000BF5A2B17FFA6
:10558000592B177FC4F808E08BF81DC0002D3FF49D
:10559000EBAE6270A760079BDBF8141003EB0A0206
:1055A0002046FFF7F1F9DDE90131009A01965354E5
:1055B000637801336370E3E6029B7B600023AB609A
:1055C000A3E7BEF1000F7FF4C7AE11B10B7A012B38
:1055D000D8D0CBF818008BF81C60BDE662700022B2
:1055E000A5E79BF80930DBF8042001925F1EFFB2AB
:1055F000002B3FF470AD01230693019B002503EBC4
:10560000C7074FF0010A7B78FA787E689A420CD17E
:105610005BE0012B53D07B7839780133DBB29942C0
:1056200008BF00239A427B704FD01BB203EB4301AB
:1056300003EB810306EB830016F82330022B17D00F
:10564000032BE6D143789BF808209A423AD9DBF83D
:10565000002003EB430302EB0313027983F82D20B0
:105660008562C36A13B1016B806A9847FA78D2E702
:10567000D0E901C19CF80020D0F80CE0DBF8004034
:10568000DBF81430FF2A03D0D1F80080984523D0EE
:105690009BF81D200B604FF000080AE002EB42036C
:1056A00004EB03111B01D1F808908969C84411B9B2
:1056B000E25CFF2AF2D18CF80020CEF80080C36AA9
:1056C0008562CFE7C0F828A0CBE7019ABA42A7F1DC
:1056D00008030BD01F4696E702EB42021301DEF8E7
:1056E0000080E25CE5E7089B002B58D0069B002B6E
:1056F0007FF4F1AC9BF81F3000228BF81E202BB1F9
:10570000DBF824405B460122032162E40DB0BDE8D2
:10571000F08F7047049888427FF62BAF681C05977E
:105720000A94049F044605E02846014401328F4252
:1057300092B210D9634403EB08004845F4D82046E0
:10574000A3F1E8730144A3F5D43301328F42A3F5EA
:10575000A57392B2EED80A9C059F636209E79BF895
:105760001D309BF809100993DBF800300093DBF83B
:10577000043005934B1E0891DBB2A1B30B92039248
:10578000FFF7D4BBC31ABEF1FF0FCCF808303FF4CB
:10579000BCAE0FFA8EF1ABE6DB1BA360F4E59BF821
:1057A0000930DBF8042001925F1EFFB2002B7FF46A
:1057B00024AF9BE70DF0B6FB00289BD1CBF8180077
:1057C0000DF0CAFBCBF8140094E70DF0C5FB0446BE
:1057D0000DF098FB9BF81D30009300287FF486ACF9
:1057E000CBF8144082E4FF230691019363E400BFE9
:1057F000F0B4049D9DF81470069C002837D11D4E0E
:1058000001F1FF3C317232605FFA8CFC49B10CEB64
:105810004C0C02EB0C11914281F82D00A1F13001EA
:10582000F9D15A1E73727560D2B283B105EBC20210
:105830005460104612F8083903EB430103EB810171
:105840008542A7EB030304EB8104DFB2F0D177B903
:10585000079A3262089A72624FF6FF73099AB2622F
:105860003846C6E90577B3837781F0BC70470120DD
:10587000F0BC70475C3600200A4B2C2202FB003241
:1058800010B4546A5CB100EB800200EB420003EB01
:105890008003A446012210BC03210220604710BCF3
:1058A000704700BF5C3600202DE9F843284EBDF854
:1058B0002C8004462C2505FB0465084604EB840176
:1058C00004EB4104696801EBC00706EB840697F816
:1058D00003E011F8304079780EF1010C5FFA8CFC8E
:1058E000644598BF4FF0000C61452ED079680EEBEF
:1058F0004E040EEB840E01EB8E044FF0040901F808
:105900002E906360089BA360099BE3600A9B236160
:105910000C9BA361119B63620D9BE3610E9B236251
:105920000F9BE362109B236302236270A362A4F8BF
:10593000148087F803C0D5E90835984733464946AF
:105940000022A847A06ABDE8F8830120BDE8F883DB
:105950005C36002010B58AB00C9C00940D9C01941C
:105960000E9C0294BDF83C400394109C0494119C3E
:105970000594129C0694139C0794149C089400248C
:105980000994FFF791FF0AB010BD00BF2DE9F84F51
:10599000284DBDF834709DF83880044608462C2107
:1059A00001FB045104EB840604EB460405EB84057B
:1059B0004C6804EBC00614F8309096F803E0747855
:1059C0000EF1010C5FFA8CFCE14598BF4FF0000C22
:1059D00064459DF844902AD0D6F804A00EEB4E04FE
:1059E0000EEB840E0AEB8E044FF0050B0AF82EB076
:1059F00063600A9BA3600B9BE3600C9B23610F9B7E
:105A0000E362109B236302236270A362A78284F87F
:105A1000168084F8179086F803C0D1E908369847B5
:105A20002B4600220421B047A06ABDE8F88F012070
:105A3000BDE8F88F5C36002010B588B00A9C009451
:105A40000B9C01940C9C0294BDF8344003949DF887
:105A5000384004940F9C0594109C069400240794ED
:105A6000FFF794FF08B010BD2DE9F0411E4C8446AD
:105A700008462C2101FB0C410CEB8C050CEB450C72
:105A80004D6805EBC00615F8307096F803E07578A0
:105A900004EB8C040EF1010C5FFA8CFC674598BF97
:105AA0004FF0000C65451CD077680EEB4E050EEBF1
:105AB000850E07EB8E054FF0070807F82E80EB6286
:105AC000069B2B6302236A70AB6286F803C0D1E9A0
:105AD00008369847234600220421B047A86ABDE84B
:105AE000F0810120BDE8F0815C3600202DE9F04115
:105AF000204D844608462C2101FB0C510CEB8C04F4
:105B00000CEB440C4C6804EBC00614F8307096F8AB
:105B100003E0747805EB8C050EF1010C5FFA8CFC48
:105B2000674598BF4FF0000C644520D077680EEBB6
:105B30004E040EEB840E07EB8E044FF6027827F826
:105B40002E80C4E90123069BE360079BE362089B68
:105B500023630223A36286F803C0D1E9083698477D
:105B60002B4600220421B047A06ABDE8F081012045
:105B7000BDE8F0815C36002070B50A4D2C2202FB96
:105B80000052D2E9083604460846984704EB8403DD
:105B900004EB430305EB8303B4460022BDE87040E9
:105BA000042160475C3600200DF0D6B9401A20F081
:105BB0007F40704770B5044600200D4603F0ECFCB2
:105BC00098B903F007FF10F006060ED134B1062293
:105BD0002946074815F088F9304670BD0622294647
:105BE000044815F081F9204670BD0C2070BD00BF3F
:105BF00090360020883600200128034605D8044A44
:105C00000448002B18BF104670470020704700BFA3
:105C10009036002088360020012810B503460BD8A6
:105C20000846074C0749002B18BF0C4606222146A0
:105C300015F05AF9204610BD0024204610BD00BFC3
:105C40008836002090360020022801D001207047BD
:105C500038B5044608461D4604F024FD10B1002066
:105C6000287038BD204638BD002303700B70704784
:105C700008B50248FEF742FA002008BD38D30100FB
:105C800030B5838983B023B1037D0446C3B1022BB1
:105C900004D06FF01505284603B030BD01A901F00E
:105CA0005FFB019B054613B1184615F0AAF9002DBC
:105CB000F1D120460EF09EFA0025284603B030BDF3
:105CC00001A9019300F0CAFB0028F2D015F099F960
:105CD000019D002DEDD0284602F03AF86871019937
:105CE000014816F09BFCE4E7740A00202DE9F0411E
:105CF0002E4F2F4E82B00CE015F080F92246BDF8F1
:105D00000210044602F00CF8204615F07AF911F062
:105D1000A7FC0DF1020101A802F0CCFA04464FF0F5
:105D2000FF324FF0FF3300211320002CE4D1019B00
:105D3000B3B102F029FBDDF80480404602F008F818
:105D4000019D88F805006B79032B02D12B79182B64
:105D50000ED02946304616F061FC019B002BD8D1AD
:105D60004FF0FF324FF0FF33384611F0B3F8D0E771
:105D70004FF0FF3321464FF0FF320520B5F8068083
:105D800015F03CF941460246044605F11C0001F0BD
:105D90004BFB404601F068FB204624B115F031F979
:105DA00020460EF027FA019DD3E700BF5C0A0020D1
:105DB000740A0020D0B51B4888B002F05FFF04468B
:105DC00060BB194801F0DAFF002600276FF00902D6
:105DD000CDE90324CDE90667CDE90144134B14490D
:105DE00000944FF4E072134810F0BCFE12491148C1
:105DF00016F089FB6FF00702CDE90324CDE90667B1
:105E0000CDE901440D4B0E4900944FF440720D480A
:105E100010F0A8FE0C490B4816F075FB204608B0A0
:105E2000D0BD00BF5C0A00203C010020ED5C0000FA
:105E300040720020D80B0020D8D201004D5E000037
:105E400020740020580C0020E4D201002DE9F04F0E
:105E5000AC4DAD4FDFF8B482DFF8B4A2DFF8B492F6
:105E6000DFF8B4B285B04FF0FF324FF0FF330221BC
:105E7000284611F0EBFE002840F0AD80EB6803F4FB
:105E8000FC23B3F5005F00F0A2802B6A03F4FC232F
:105E9000B3F5004F00F006810024EA682B6A6FF327
:105EA00052326FF35233EA602B629C4A9C4B1E685D
:105EB000BFF35B8F52E8003F23F0010142E800107E
:105EC0000028F7D1BFF35B8FDB0744BF0023C7E98E
:105ED0000033002E40F3ED80DAF80010D9F80030DE
:105EE000711A19443B68C8F80010002B00F00681B5
:105EF0005A79002C75D1042A47D8022A00F2BA80B8
:105F000040F212215846CDE90032FCF7D3FC019A49
:105F1000009B0393002A40F0B38040F2A31158463F
:105F2000FCF7C8FC039B00221A6003A802F0BEFA2B
:105F3000DAF80030F61AD9F800301E443B68C8F889
:105F400000602BB15B79DA1E012A16D9052B12D01D
:105F5000002C88D0204615F0C7F8214606460020C0
:105F600015F0C6F8B389044630465BB1FEF736F942
:105F700011F076FBECE7002EEAD00021694811F021
:105F8000C1FEE5E70EF036F9F2E7052A16D1002941
:105F90003FF469AF79681A683A608B4200F0EE808E
:105FA00003934FF0FF324FF0FF330320FEF7B8F8B2
:105FB00004460146039801F079FAB3E740F2122152
:105FC00058460093FCF776FC009B0393A5E72B69EA
:105FD00000249C6061E740F24A215846FCF76AFCC5
:105FE0004CE7D01E012840F28280052A00F09C80F8
:105FF0000131627965D0511E3B68052900F2D180DC
:10600000DFE801F003031B1B3003042A03945DD96E
:10601000052A1BD14FF0FF324FF0FF330320FEF76C
:106020007FF804462146039801F040FA039B0022C2
:106030001A6003A802F03AFA8AE70121C8F80010B2
:10604000002B40F08A800394002A3FD1584640F24A
:10605000A311FCF72FFC039B00221A6003A802F097
:1060600025FA00E7002B78D1D8F80030002B74D047
:106070000394CFE778681968396083427CD0039332
:10608000022A71D04FF0FF324FF0FF330120FEF7AC
:1060900047F80446002C3FF445AF0398214601F031
:1060A0005BFA3FE7686A0022002310F0B9FE04465D
:1060B000F3E64FF0FF33C8F80030002C3FF4D3AEC6
:1060C00062790394042AA3D8002ABFD0022A5DD0A3
:1060D00001204FF0FF324FF0FF33FEF721F8044666
:1060E000002C4DD00398214601F036FA9EE700219E
:1060F0000C4811F007FED8F8001079E7002C7FF467
:1061000077AFB0E6140100209C36002098360020BE
:106110005837002034370020ECD2010060370020CF
:106120005C3700203C0100200029E0D16279511E3B
:10613000052936D801A050F821F000BF0B600000FF
:106140000B600000556100005561000065600000B3
:106150000B6000000123C8F800307B680022226039
:10616000E3B11C607C607EE6002200230121002058
:1061700014F044FF04468DE7796080E77A600FE70A
:10618000039B03A81C6002F091F96CE6012100203A
:106190000022002314F032FF0446A1E7C7E90044BF
:1061A00061E640F2C9115846FCF784FB03944DE7C1
:1061B0002DE9F047DFF8A890D9F80030002B804691
:1061C0000F46164612DD274C002521460622304692
:1061D00014F061FE18B914F8013CBB4229D0D9F87B
:1061E000003001359D4204F10804EEDB1E4D1F4CCA
:1061F000D5F800A031464FEACA06701C204406229A
:1062000014F072FE012303FA08F8D9F8003004F8FC
:106210003A7034440F2B84F807801CDC01331A4693
:10622000C9F800302B600020102A08BF2860BDE8A4
:10623000F0870E4B03EBC5050120EA7922FA08F33B
:1062400013F00103F3D100FA08F842EA0802EA71F8
:106250001846BDE8F0872A6801322A60E3E700BFEC
:10626000A8360020B1360020AC360020B036002021
:10627000F8B5194C6468A40004D51546174A12688D
:10628000120700D4F8BD03F1080407460E46204665
:10629000022114F039FF3E2303700C2343700121C7
:1062A000204614F031FF034604221A7020460B21C9
:1062B00014F02AFF08220770A0F801502FB9311DF1
:1062C0000330BDE8F84014F00FBEBDE8F8400021EF
:1062D000033014F014BE00BF0000002008000020AE
:1062E000F0B5013887B01546092806D8DFE800F078
:1062F000092744050558056C899E6FF0150007B005
:10630000F0BD544B0D21188814F099FE0D21286022
:10631000083014F0F9FE0346022200200324632112
:1063200018705A709870DA70187158719C71D87121
:10633000187259729872D872187307B0F0BD454B35
:106340004121188814F07BFE41212860083014F0A8
:10635000DBFE00240546402200F8014B214614F0E4
:10636000CEFD6A78AB7862F0580243F00303204612
:106370006A70AB7007B0F0BD364B0921188814F075
:106380005EFE09212860083014F0BEFE002400F8EB
:10639000014B0822214614F0B2FD204607B0F0BDA3
:1063A00089680020FFF706FC2A4B0121188814F0A9
:1063B00046FE01210446083014F0A6FE03460020E4
:1063C00018702C6007B0F0BD234E224F0FCE0DF198
:1063D000040CACE80F0033683888ACF800301321A7
:1063E00014F02DFE13212860083014F08DFE0024D7
:1063F00000F8014B122201A914F076FD204607B0E7
:10640000F0BD144B1821188814F019FE18212860CB
:10641000083014F079FE00240546012100F8024BF3
:106420000DF070FD6870204607B0F0BD094B2121CA
:10643000188814F004FE21212860083014F064FE4E
:106440000146002401F8114B01300DF0CFFD20462C
:1064500007B0F0BDC46D002050D30100F0B58389B2
:106460008FB00022022B099233D904460E46083021
:10647000032114F069FEA28983789A4229D3028805
:10648000D04FC2F38523082B90B23A80C2F309059E
:106490000DD8BBB1013B072B14D8DFE813F01E0069
:1064A00013002D007901AB01130013007C003F2B7A
:1064B00008D109AA21462846FFF712FF163040F0FE
:1064C000FA863888012114F0CCFD044620460FB02E
:1064D000F0BD002420460FB0F0BD062D00F0D4869C
:1064E0001D2DEFD1A368188804F00CFB01463888F5
:1064F00014F0B7FD0446E9E7352D00F2B1812C2DEB
:1065000000F29481012D00F0D381032DDAD1AE4841
:10651000AE49AF4AAF4B4FF0FF34046041F6FF7510
:106520004FF0FF34C1E9004500200021C2E900011D
:106530001F200021C3E9000102F00CFC0121388872
:1065400014F07DFD01210546083014F0DDFDA24B5D
:10655000A249A34A00241C60A24B04700C60146082
:10656000A1481C6020222146099514F0C8FCBFF305
:106570005B8F9E4B53E8002F42F0010243E800215D
:106580000029F7D1BFF35B8F994B1868214611F0B2
:10659000B9FB099C9AE76A1E7A2A93D801A353F89B
:1065A00022F000BF797200005172000003720000F7
:1065B000C5640000F9710000C1710000A371000002
:1065C000977100008B7100008171000069710000FB
:1065D00039710000B3700000AB70000087700000DC
:1065E0008170000079700000717000004970000037
:1065F0004170000015700000FF6F0000C96F0000BF
:10660000A56F0000856F0000756F0000656F0000CA
:10661000316F0000196F0000FF6E0000D36E0000A4
:10662000B56E00009D6E0000C36D00008B6D000014
:106630007F6D0000C5640000C5640000716D00003E
:10664000696D0000636D00003F6D00000F6D00007C
:106650006D6E0000636E0000416E0000F36D00007F
:10666000B36C0000956C0000376C00001F6C0000DC
:10667000056C0000C5640000C5640000C56400002E
:10668000C5640000C5640000C5640000C564000066
:10669000C5640000C5640000C5640000C564000056
:1066A000C5640000C5640000C5640000C564000046
:1066B000C5640000C5640000C5640000C564000036
:1066C000C5640000C5640000C5640000E16B000003
:1066D000C5640000C5640000D76B0000B56B000006
:1066E000816B0000C5640000C5640000C564000043
:1066F000C5640000C5640000C5640000C5640000F6
:10670000C5640000C5640000C5640000C5640000E5
:10671000C5640000C5640000C5640000C5640000D5
:10672000C5640000C5640000C5640000C5640000C5
:10673000C5640000C5640000C5640000C5640000B5
:10674000C5640000C5640000C5640000C5640000A5
:10675000C5640000C5640000C5640000C564000095
:10676000C5640000C5640000C5640000C564000085
:10677000C5640000C5640000C5640000C564000075
:10678000C5640000C5640000C5640000436B0000E0
:106790006A1E082A3FF696AE01A353F822F000BF06
:1067A000E76900001D690000F5680000C56400008D
:1067B000C5640000C5640000C5640000C564000035
:1067C000D3680000C46D0020A8360020000000201F
:1067D000D80C002008000020A43600205C370020E0
:1067E0005837002034370020383700206037002029
:1067F00030370020052D7FF465AEA36804211D8885
:1068000014F01DFC042103460830099314F07CFCAD
:106810000446E11CA8B204F09DFAA4F801502070CF
:10682000002841D07F23E370099C4FE6A5F12D029B
:10683000082A3FF647AE01A353F822F0756A00001C
:10684000C5640000C5640000C56400001D6A000046
:10685000C5640000136B0000C5640000A56A000059
:106860007B2D00F02B857C2D15D1A3681D885988C0
:10687000A8B204F0AFFA03210446388814F0DFFB15
:10688000032103460830099314F03EFC0470099C70
:10689000A0F801501AE6632D7FF414AEA268BE4B37
:1068A00011681960526808E0E3785B425BB2BAE7AE
:1068B000A268BA4B1168526819605A60012114F03D
:1068C000BEFB01210446083014F01EFC00230370B7
:1068D000FCE5072114F0B3FB0721034608300993B8
:1068E00014F012FC0146002001F8010BFFF794F9A7
:1068F000099CEBE5092114F0A2FB092103460830AD
:10690000099314F001FC00210546082200F8011B40
:1069100014F0F5FA6023099C6B71D7E5412114F05E
:106920008EFB412103460830099314F0EDFB002152
:106930000546402200F8011B14F0E1FAAB79E97832
:10694000EA7BE87A6C7863F03F03AB712B7C61F0F3
:106950007F0142F0280243F02203E970EA73E97DE7
:10696000AA7E2B746B7F41F0040162F0080243F0B1
:106970007F036B77E97595F8253095F82210AA7694
:1069800095F8212061F00F0142F0300243F001033D
:1069900085F8212085F8221095F8232095F82E10EF
:1069A00085F8253095F8283060F01B00E87244F037
:1069B0002004FF2043F01C0362F0060241F00101B5
:1069C0006C70E876287785F8240085F82E1085F815
:1069D000232085F8283095F82730099C63F07F0341
:1069E00085F8273072E5092114F029FB09210346B7
:1069F0000830099314F088FB00230C214FF0FF327C
:106A000003706FF00E0441708370C37005234471EE
:106A10000171099C8371C271027257E5A368604DD0
:106A20001C78012114F00BFB012103460830099367
:106A300014F06AFB2B68002B00F03B84594A126863
:106A4000002A40F036840270002C00F05E84012C95
:106A50005BD1002B00F32F845348544B002101607D
:106A600020225348196014F04AFA2B68099C5B42B3
:106A70002B602BE5A36804211E889F7814F0DFFAB1
:106A800004210990083014F03FFBB4B20546C31C42
:106A900021463A460220FFF7D7F82870099CA5F84E
:106AA000016013E53E4B1B68002B40F3F9833D4B1F
:106AB0001B680BB3A76897F800C06546BCF1000FD0
:106AC00000F0178400223A4E15460BE036F81430D9
:106AD0009942A3EB01030FD826F81430D3B29C459A
:106AE00040F2078407EB82030132B3F80140B3F8A8
:106AF00003100F2C0D44E9D9012114F0A0FA012153
:106B000003460830099314F0FFFA12230370099C1E
:106B1000DCE4A3680121B3F803401D8814F08FFA68
:106B2000012103460830099314F0EEFA1C4B1A6851
:106B3000002A40F0BE831A2DE7D962421A60099CF0
:106B4000C4E4A468A579E378A27820786119E61DE9
:106B500091F907C06178CDE9036C029565790195DB
:106B6000247900940CF0C2F805463888012114F00D
:106B700066FA01210446083014F0C6FA0570A5E44F
:106B8000A46825467F2615F8070BE378A27861787C
:106B9000CDE90356A579E0E7D80C002000000020DD
:106BA0005C370020A43600205837002034370020FE
:106BB00038370020A4682546E37815F8070BA2783B
:106BC00061780395A57902956579019524790094FA
:106BD0000CF010F9C8E7A068C17908F0F3FFC3E72B
:106BE000032114F02CFA032103460830099314F012
:106BF0008BFA0146002301F8023B0130FFF734F81D
:106C0000099C63E4A0680024C37882784178007806
:106C1000CDE90244CDE900447F240494A2E7A368AF
:106C20009A78597818780023CDE90233CDE90033FA
:106C30000CF0E0F898E7A36899781D88B3F8054050
:106C4000CE0703D5DA7842F00702DA708A0703D557
:106C50001A7942F007021A71D9781B7941EA0302C6
:106C600012F0F80F40F06C834E0700F057835A077C
:106C700000F0548314F003021CBF04F1FF3404F04D
:106C80000102284604F010F80146388814F0E9F9AA
:106C900004461BE4A3681A78D10744BF0721597042
:106CA000920744BF07229A709978587803F0F2FF50
:106CB0005AE7A36805211E8814F0C1F9052103468F
:106CC0000830099314F020FA05462A1DB0B2E91CD9
:106CD00003F0BEFFEB782870002B93FAA3F22B7918
:106CE000B2FA82F208BF4FF0FF32002B93FAA3F3FF
:106CF000B3FA83F302F1010208BF4FF0FF33EA70E9
:106D00000133099C2B71A5F80160FFF7DFBB072257
:106D1000A1680AA814F0E8F80721388814F08FF960
:106D2000072103460830099314F0EEF90446411C8C
:106D30000AA808F0B5FE2070099CFFF7C7BB022126
:106D400014F07DF9022103460830099314F0DCF9B0
:106D5000044608F045FD002360702370099CFFF78E
:106D6000B5BB08F03FFDFFE6A06808F07DFDFBE63F
:106D7000A06800F11702C11D09F0C4F9F4E6A36888
:106D80005988188803F04EFFEEE6052114F057F9F4
:106D9000052103460830099314F0B6F90AA90546FF
:106DA0000DF1220003F032FFBDF82230A5F80130CA
:106DB0000022BDF828302A70099CA5F80330FFF79F
:106DC00085BBA3681D889A885988A8B203F0C2FEC3
:106DD00004460321388814F032F9032103460830B1
:106DE000099314F091F90470099CA0F80150FFF781
:106DF0006DBB092114F023F90921034608300993DA
:106E000014F082F90AAB05460DF1220208A90DF132
:106E10001E0003F011FFBDF82030BDF81E20A5F8BC
:106E20000120A5F80330BDF82230A5F80530002276
:106E3000BDF828302A70099CA5F80730FFF746BB3B
:106E4000A368188808F0B4FE3888012114F0F7F818
:106E500001210446083014F057F900220270FFF7B0
:106E600035BBA368187808F087FE7DE60722A16885
:106E70000AA814F039F80721388814F0E0F807213F
:106E800003460830099314F03FF90446411C0AA850
:106E900008F040FE2070099CFFF718BBA268158817
:106EA00092780023CDE9013300930221A8B203F0C8
:106EB000FBFC8DE7A2681189158853880291D1885F
:106EC00001919188009100220221A8B203F0ECFC0C
:106ED0007EE70AA80BF0CAFF03210446388814F0A5
:106EE000AEF8032103460830099314F00DF904703D
:106EF000BDF82820099CA0F80120FFF7E7BAA36895
:106F00007F249A785978187804940023CDE90233C5
:106F1000CDE90033012325E6A26800231078012182
:106F2000CDE90233CDE900331A460BF063FF1BE6CF
:106F3000092114F084F8092103460830099314F05C
:106F4000E3F80346FF2200213F20D87019705A70E1
:106F50009A700320099C1A715A719871D97119722B
:106F6000FFF7B4BAA3681D8800220621A8B207F073
:106F7000C7FD2DE7A26832F8025B0021A8B207F036
:106F8000BFFD25E7A268114602F10C0331F8020BA0
:106F90000A3207F09DFE0146388814F062F8044674
:106FA000FFF794BA092114F04AF809210346083082
:106FB000099314F0A9F8002300F8013B082109F017
:106FC000D1FC099CFFF782BAA0680AAA002300F14D
:106FD00010010BF0F7FF1121388814F030F811215F
:106FE00003460830099314F08FF8002300F8013BA2
:106FF00010220AA913F078FF099CFFF767BAA3686B
:10700000188803F057FD0146388814F02AF8044622
:10701000FFF75CBAA36808211E8814F010F8082155
:1070200003460844099314F06FF80546E91CB0B212
:1070300003F0D0FC2870099CA5F80160FFF746BA60
:10704000A06808F039F98FE5A1680A894B8808889B
:107050000292CA880192898800910022114603F0A9
:1070600023FC0146388813F0FCFF0446FFF72EBAD4
:10707000A06808F037FB77E5A06808F099FA73E597
:1070800008F06CFA70E5022113F0D9FF02210346E3
:107090000830099314F038F800230370044608F010
:1070A0005BFA6070099CFFF711BA304607F0CCFD1F
:1070B0005AE5A4682288131F9BB243F6FC75AB42C5
:1070C00000F22C8161880B1F9BB2AB4200F226813B
:1070D000B4F80F50AB1F40F67A469BB2B34200F2B1
:1070E0001D81B4F81160B6F5FA7F80F01781B4F80D
:1070F00013C0ACF10A0340F6764E9BB2734500F222
:107100000D81731C9BB205FB03F3B3EB8C0F80F274
:1071100005816379104622790295CDE9036C063426
:10712000A57901950094FAF717FB0146388813F00A
:1071300098FF0446FFF7CAB9A3681878002800F042
:10714000E8805B78002B00F0E4808049804A0023CF
:107150000B60136002F08AFB0C2805464FF001011A
:10716000388808BF002502E5A4686379B4F80320D5
:10717000B4F801102078A4790094F9F721FCF3E425
:10718000A3681878F9F774F9EEE4A16811F8010B17
:1071900002F0FAFAE8E4A16811F8010B02F0AAFA89
:1071A000E2E4022113F04BFF022103460830099369
:1071B00013F0AAFF002202704270099CFFF786B903
:1071C000A4682179228801290AD063889A4200F2B2
:1071D000AB801F2A40F2A880B3F5804F00F2A48054
:1071E000A57BA379104662790295657B01950734EA
:1071F000009402F09BF8B7E4A1680120FEF7DAFCE6
:10720000B2E4092113F01BFF09210346083009935A
:1072100013F07AFF00210546082200F8011B13F045
:107220006EFE00F0EDFD0B460246010C6A70C2F3E3
:1072300007201A0CA870E970C3F30720090A6B71C4
:10724000130A099C2971A871EA712B72FFF73EB9E4
:10725000042113F0F4FE042103460830099313F0CF
:1072600053FF0346002207201A701B21D870099C87
:1072700059709A70FFF72AB9A268364B11685268A4
:1072800019605A600121E1E5A3689978188803F034
:10729000C5FB0146388813F0E4FE0446FFF716B933
:1072A000012113F0CCFE012103460830099313F0AD
:1072B0002BFF0C230370099CFFF708B9A3681D88F6
:1072C0000AA9A8B203F060FD05210446388813F02E
:1072D000B6FE052103460830099313F015FF04702C
:1072E000A0F80150BDF82830099CA0F80330FFF742
:1072F000EDB8194A1949136808682B441360002136
:1073000010F000FD099CFFF7E1B8002BBFF6A4AB1D
:10731000D1E70E4B4FF0FF321A601BE7122113F03A
:10732000A0FE0446FFF7D2B8012113F088FE012128
:107330000446083013F0E8FE12230370FFF7C6B8C6
:10734000112113F08EFE0446FFF7C0B8A8360020C6
:10735000AC360020080000203437002030370020F1
:107360002DE9F84383890022032B0A6018D90546CA
:1073700088460830042113F0E7FEAB894688B0F850
:107380000090B3420CD31B2E0AD803F09FF94FEAAA
:107390001937044618B3BB0802D1D7B1012F03D067
:1073A0006FF01500BDE8F883037967F301030371FB
:1073B0006671A9683246E01D13F096FD2146C9F3B7
:1073C0000B0003F08FF90028ECD0204603F084F97D
:1073D000E6E70379022262F301030371E8E7114B48
:1073E0001B689B0102D46FF06800DBE74FF0FF33AE
:1073F0004FF0FF320120FCF793FE0221C8F8000095
:10740000083013F081FE01241A2202704470D8F86B
:1074100000002146083013F077FE03466FF0680045
:107420001C70BFE700000020F8B50E4B1B68DB06A0
:1074300000D4F8BD02F1080405460E46204602219C
:1074400013F062FE03460421052259701A7020468B
:1074500013F05AFE00270770A0F801602B78C37064
:10746000F8BD00BF000000200F2810B504460FD85B
:107470000A480B49D0F800C031F81430094A634477
:10748000036013680020013B21F81400136010BD55
:10749000054841F6C641FBF70DFAE9E7343700200D
:1074A00038370020A436002064D30100037F03F0A6
:1074B0000303013B012B04D9224841F62671FBF757
:1074C000F9B970B5044601F1080528460421E6889B
:1074D00013F01AFE237F03F00303022B0CBF46F4C4
:1074E000005346F480530380617F4180284613F0A7
:1074F0000BFE627F04F11F0113F0F6FC124B1A68B9
:10750000002A10DD114C124923680968591A91426A
:1075100010D201330F2E236006D80E4A32F81630EF
:10752000013322F8163070BD064841F61F71FBF793
:10753000C1F9F2E7034841F61971FBF7BBF923687B
:10754000E7E700BF64D301005C3700205837002014
:1075500034370020383700202DE9F04F90F804C070
:10756000C688BCF1030F89B004460D4600F11C0724
:107570001FD0ACF1050CBCF1180F3ED8DFE81CF0B1
:1075800045003D003D003D003D003D003D003D000B
:107590003D003D003D003D003D003D003D003D0003
:1075A0003D003D00C20020012801330058016B015D
:1075B0008C01C37F033B122B00F2B481DFE813F090
:1075C0005702B201B20134024D02B2010402B2010B
:1075D000B2018602A702B2010D02B2011A00B20185
:1075E000B201B601B601C84B5B681F044FF000043E
:1075F00000F1C38109B0BDE8F08FC44841F61A61BB
:1076000009B0BDE8F04FFBF755B9C14A037EA67E2D
:1076100094F8198092E803005B425FB20B0C8DF87E
:107620001E30237FADF81C1059060690C6F34006A5
:1076300000F1B381B44B5B6803F00053002E40F0BF
:10764000A882002BD6D0B34B1B689B07D2D5B24B78
:107650001B68002B04F11E0A09DB207F5246C0F391
:10766000801100F00F00FEF7A3FD0028C2D1237F98
:1076700003F00F03012B00F03F83637F03F1060B40
:10768000A3F106095FFA8BF25FFA89F905330592D7
:107690005FFA83FB4E4608350221284613F034FD7D
:1076A000059B43703E2202700121284613F02CFDF9
:1076B0000246022313705946284613F025FD012384
:1076C0000370237F08AA03F00F031344054613F841
:1076D000083C437008F084F8804580F0E68240461C
:1076E000EA1CA91C08F04CF8AB780233AB7085F8A3
:1076F00009900A3504F124013246284613F0F4FBC0
:10770000AF5577E7FF0700F15981277F002F00F081
:107710004C817D4B5B6898007FF56CAF7D4B1B689F
:1077200040F20122134203F400783FF463AF0835BE
:10773000002F40F01182794A1368013304F11F09C8
:107740001360B8F1000F00F081820221284613F087
:10775000DBFC3E2303701F2343700121284613F0F6
:10776000D3FC03460A221A7028461E2113F0CCFCD3
:107770000770A0F80160637FC370A37F03710546A3
:1077800049460622053013F0AFFB062204F12B0117
:1077900005F10B0013F0A8FB062204F1250105F109
:1077A000110013F0A1FBE38E618EA28EA5F81920C3
:1077B000A5F81710A5F81B3094F838306B7719E747
:1077C0000A463846314609B0BDE8F04FFFF72CBEF7
:1077D0004D4B5B6899007FF50DAF4E4B1B685A0708
:1077E0007FF508AF08350221284613F08DFC3E23B3
:1077F00003700A2343700121284613F085FC0346D9
:10780000032228461A70092113F07EFCFB07054667
:1078100000F16C82237F2B70E18B228C638CA5F8A6
:107820000730A5F80160A5F80310A5F80520E1E6EA
:107830003B4B1B6818027FF5DDAE08350221284658
:1078400013F062FC0221572303704170284613F0A5
:107850005BFC0680CEE62C4B5B6899007FF5CAAED8
:107860002C4B1B681A037FF5C5AE0835022128464C
:1078700013F04AFC3E230370042343700121284681
:1078800013F042FC142303700321284613F03CFC40
:107890000680237F8370ADE61B4B5B689B007FF502
:1078A000A9AE1C4B1B681F057FF5A4AE083502214D
:1078B000284613F029FC3E23037006234370012160
:1078C000284613F021FC0C2303700521284613F0F1
:1078D0001BFC237F0370A0F80160627F002A92FAEC
:1078E000A2F3B3FA83F308BF4FF0FF330133C37041
:1078F000A27F92FAA2F3002AB3FA83F308BF4FF0F3
:10790000FF330133037175E60000002064D30100EA
:1079100050D1010008000020A8360020A436002025
:10792000D80C0020C54841F6FA6169E6C44B5B6893
:107930009A007FF55FAEC34B1B685B067FF55AAEBE
:1079400008350221284613F0DFFB3E2303700B238A
:1079500043700121284613F0D7FB072303700A2147
:10796000284613F0D1FB0680A38C4380E38C8380F0
:10797000238CC380638C03813CE6083502212846B2
:1079800013F0C2FB3023032103704170284613F02B
:10799000BBFB0470A0F801602CE6002104F11E037B
:1079A0004246084608F01AF844E6A07F04F1250391
:1079B000FF2204F11F0108F011F8AAE69F4841F6E2
:1079C0005A41FAF777FFA0E60B46324639460020C7
:1079D00009B0BDE8F04FFEF74BBC994B5B689800CF
:1079E00040F1B080974B1B68990640F1AB80083599
:1079F0000221284613F088FB3E2303700B234370BB
:107A00000121284613F080FB062303700A21284633
:107A100013F07AFB0680238C4380638C8380A38CD5
:107A2000C380E38C0381E5E5854B1B681A064FF0A4
:107A300000047FF5DFAD08350221284613F064FB12
:107A40000823042103704170284613F05DFB0123D5
:107A50000470A0F80160C370CCE590F820300E2BC4
:107A60007FF4C8AD0B46324600211A20B0E7744BB4
:107A70005B6898007FF5BEAD724B1B68D9067FF539
:107A8000B9AD08350221284613F03EFB3E230370B2
:107A90000D2343700121284613F036FB05230370A4
:107AA0000C21284613F030FB04F120010546082282
:107AB00020F8026B13F018FA022204F1280105F1F4
:107AC0000A0009B0BDE8F04F13F00EBA5C4B1B681A
:107AD0001B054FF000077FF58DAD083502212846C4
:107AE00013F012FB034608210C2259701A70284625
:107AF00013F00AFB0770A0F8016094F82030C370FF
:107B0000B4F821308380B4F82330C38072E54C4B45
:107B10001B681F067FF56EAD08350221284694F8D4
:107B2000204013F0F1FA0823042103704170284625
:107B300013F0EAFAB4FA84F35B090470A0F8016068
:107B4000C37057E50023CDE9013300931A220221C7
:107B5000304602F0A9FE4DE502212846B8F1000F9B
:107B600040F0AD8013F0D0FA3E230370132343702E
:107B70000121284613F0C8FA012303701221284678
:107B800013F0C2FA04461222414613F0B8F92770E6
:107B900030E5002B3FF42EAD2A4B1B685A057FF5CC
:107BA00029AD237F03F00F03012B04D0234841F2BA
:107BB0007451FAF77FFE244B1B68002B04F11E065C
:107BC0000ADB207F3246C0F3801100F00F00FEF781
:107BD000EFFA00287FF40EAD08350221284613F095
:107BE00093FA3E230370122343700121284613F0B9
:107BF0008BFA03460B221A702846112113F084FADF
:107C0000012303704370054607F0EAFD80457AD2F0
:107C1000EA1C4046A91C07F0B3FDAB780233AB70F9
:107C2000237FC3F3C01306226B7204F1240105F114
:107C30000A0013F059F92F74DCE400BF64D301008B
:107C40000000002008000020A8360020022128465D
:107C500013F05AFA3E230370132343700121284680
:107C600013F052FA034601221A702846122113F02B
:107C70004BFA0770A0F80160637FC370A37F03F025
:107C800001030546037149460622053013F02CF91D
:107C9000E38E618EA28EA5F80D20A5F80B10A5F835
:107CA0000F3094F838306B74A4E4237FC3F380134F
:107CB0005146AB700622E81C13F016F917E513F0D5
:107CC00023FA3E221F23027043700121284613F03D
:107CD0001BFA0A2303701E21284613F015FA0446E6
:107CE0001E22002113F00BF9277083E40B4841F6A4
:107CF000DF41FAF7DFFD8DE500260C234FF00B0B7B
:107D00000593B146C7E4237FC3F380133146AB70BC
:107D10000622E81C13F0E8F882E700BF64D30100F4
:107D200070B500F108040E4620460221154613F0F6
:107D3000EBF91323052103704170204613F0E4F999
:107D400001230370A0F80160A0F8035070BD00BFCC
:107D50000379032B08D0053BDBB2182B01D9002097
:107D60007047054AD05C7047037F03F00303032B81
:107D70000CBF042005207047A0D30100124B4FF028
:107D8000FF32D0B41A60114B114C124A20604FF0F0
:107D9000FF3641F6FF77C3E900670F4B0F48104CE1
:107DA00000260027C2E900670E4A1F26002700218F
:107DB000C3E900670C4B0160116021600B4819603A
:107DC000D0BC202213F09BB8A83600200000002071
:107DD00030370020D80C002008000020A4360020F6
:107DE000583700205C370020343700203837002017
:107DF00008F0B8BD08B500230BF0E4F8002008BD7A
:107E000001480021704700BFFF49010010B504463A
:107E100008F0DEFD68B909F05DF998B909F0E0FFF6
:107E2000C8B90AF007F9F8B92046BDE810400FF0CC
:107E30002BB8124840F64F01FAF73CFD09F04AF919
:107E40000028EBD00D4840F65401FAF733FD09F055
:107E5000C7FF0028E5D0094840F65A01FAF72AFD85
:107E60000AF0E8F80028DFD004484FF40661FAF77A
:107E700021FD2046BDE810400FF006B8BCD301003C
:107E8000086001480FF000B8784500200EF0FCBFF4
:107E90002DE9F84F2C4D0C469146A97822782B7885
:107EA00091429CBF2A7922704A45824642D012FBF9
:107EB00003F30132D2B2254F914208BF0022227053
:107EC000FA5A028000263B444FF0010B4FF00208A3
:107ED00021E062B3027902F00302013A012A2DD9AE
:107EE000C3F8048002F0F8FB2378A9782878994237
:107EF0009CBF2B79237099451DD05A1CD2B2914258
:107F000008BF002213FB00F32270F95ABAF80020D0
:107F100091423B440FD15868012820F00302D8D881
:107F20000136F6B2C3F804B0002ADDD0DAE7C3F8B0
:107F30000480D9E700263046BDE8F88F0136C3F843
:107F400004B0F6B2CEE700BF040400200C04002009
:107F50002DE9F047344F3B8898425CD9DEB24BB3F1
:107F6000324DDFF8CC806C79DFF8C890AA782B7995
:107F70000134E4B2A24208BF0024A34240461BD011
:107F8000FCF794F982464846BAF1000F12D0FCF78C
:107F90008DF9002841D0C0F800A06A792B7802FB47
:107FA000035398603B886C71013E013B16F0FF065D
:107FB0003B80DBD1BDE8F0873B88002BFAD01E4D1B
:107FC0001B4E6C79DFF86C804FF00009AA782B7992
:107FD0000134E4B2A24208BF0024A3423046E9D0F3
:107FE000FCF764F982464046BAF1000FE2D0FCF794
:107FF0005DF990B1CAF80490C0F800A06A792B78B6
:1080000002FB035398603B886C71013B9BB23B8041
:10801000002BDBD1CEE70646A2E750460449BDE877
:10802000F047FCF75DB900BFC0370020CC0200204C
:10803000C4370020A8390020400200202DE9F04379
:10804000314FDFF8C880324D83B0D7E9000101AA73
:10805000FCF79AF90446002840D078680022394697
:10806000FCF79AF9DDF80490D9F81C6036B1337842
:10807000002B42D03378013BDBB2337099F82030CB
:1080800023B1012B33D1484605F050FF6B79A87816
:10809000297901330022DBB2984208BF1346994286
:1080A00089F820202A781CD0C9F80040697901FBA2
:1080B0000252C2F808906B71002EC6D03378002BA4
:1080C000C3D17369002BC0D0B0699847D7E90001CC
:1080D00001AAFCF759F904460028BED103B0BDE857
:1080E000F0834FF42C614046FAF7E4FBE4E740F6F6
:1080F000B9214046FAF7DEFBC8E740F66221404668
:10810000FAF7D8FBB6E700BF64450020BCD30100F6
:10811000240200202DE9F047614FDFF88881DFF865
:10812000889186B0D7E9000103AAFCF72DF905462E
:10813000002836D0039B002B00F09D80187804AAFD
:1081400002A906F0CFF90446002856D0DDE9031352
:10815000BDF8082091F800A0ADF80A2005AE0593FF
:108160000DF10A0506F0D8F92146059ABDF80A0076
:1081700006F010FA204606F08DF9324629465046A0
:1081800006F0B0F904460028ECD1D8F800000EF053
:108190007BFED7E9000103AAFCF7F6F805460028A4
:1081A000C8D104AA02A90DF1070006F07FF9044620
:1081B00000285DD0049B05939DF807A0BDF808300A
:1081C000ADF80A3005AE0DF10A0506F0A5F9214615
:1081D000059ABDF80A0006F0DDF9204606F05AF9C6
:1081E00032462946504606F07DF904460028ECD177
:1081F000D8F800000EF048FECBE7039B05931B79EF
:10820000013B172B0DD8DFE803F0120C2E0C120CDB
:108210000C0C0C0C0C0C0C0C0C0C0C0C0C0C0C0C9E
:10822000241240F64F214846FAF744FB7AE73946D4
:1082300078680022FCF7B0F81C4B05995B7928465A
:108240001B4A0B70FCF796F8D8F800000EF01CFEE5
:108250009FE7394678680022FCF79EF80599284682
:1082600002F06AFE5EE705A9284602F081FE48B1E9
:1082700006B0BDE8F08740F6FD014846FAF71AFB64
:10828000039B5BE7024639467868FCF785F8059959
:1082900000293FF447AF054B28465B79D0E700BF84
:1082A0006C45002074450020BCD30100040400206C
:1082B000604500202DE9F04F2D4C2E4F2E4E85B0FD
:1082C0008946019004F1040A07F1040B019A002386
:1082D0001360D6E9000103AAFCF756F8054600280A
:1082E00037D0039B51461A784846FFF7D1FD002846
:1082F00034D123798DF80930627980460DF1090176
:108300000DF10A00FFF7C4FD48EA000212F0FF0277
:10831000F2D1039B1979012923D117497068FCF721
:108320003BF859462846FBF7DBFF3B88282B09D84A
:108330000398124901333B80FBF7D2FF0120FFF77E
:1083400007FEC3E70E4840F22761FAF7B3FA3B880D
:10835000EEE762790B494846FFF79AFD05B0BDE8A4
:10836000F08F019910460B6005B0BDE8F08F00BF9B
:1083700004040020C03700205C450020A8390020FC
:10838000BCD301000804002070B5444982B000232A
:108390004868019301AAFBF7FFFF0446002852D06A
:1083A0003F492046FBF79CFF019A13791D2B10D8FB
:1083B000DFE803F0160F0F160F160F0F0F0F0F0F3A
:1083C0000F0F0F0F0F0F0F0F0F0F0F1F1616161691
:1083D0001616344840F2E641FAF76CFA02B070BD66
:1083E000002BFBD12F4840F2E241FAF763FA02B0CA
:1083F00070BD137F95683C2B2C682AD0537FD3B176
:10840000606E20B1002328496366FBF769FF94F88A
:108410006A306FF3000384F86A30002001F0DAFA62
:108420000446002001F0B8F850EA4400D6D107F025
:1084300091FC02B070BD94F84420236263F3000203
:1084400084F84420E9E717484FF46F71FAF732FADD
:10845000A6E76E68AEB1B36D00226A6023B1114821
:1084600040F23541FAF726FA06F14C0106F14800D0
:10847000FBF776FF054650B13068B56502F0FCF8B1
:10848000C5E7084840F23241FAF714FAE3E7054835
:108490004FF48761FAF70EFAEEE700BF5C45002063
:1084A000C4370020BCD30100A83900202DE9F043D7
:1084B000046883B0804604B3434F444EDFF8109104
:1084C000254624682B791D2B10D8DFE803F02B0FED
:1084D0000F2B0F2B0F0F0F0F0F0F0F0F0F0F0F0F74
:1084E0000F0F0F0F0F1F3D2B2B2B2B2B40F21B6160
:1084F0003846FAF7DFF9002CE2D10023FF20C8F854
:10850000003003B0BDE8F043FFF722BD2B7F3C2BCA
:108510003DD0022B42D05BB140F24A513846FAF7C7
:10852000C9F92B7923B940F29C513846FAF7C2F9C0
:108530003388282B24D80133494628463380FBF75B
:10854000CFFE002CBCD1D8E7E8880F28D3D802F0A2
:10855000A1F8436F054623B140F20D613846FAF7A2
:10856000A9F905F1680105F16400FBF7F9FE03467E
:1085700008B36B67284602F07FF8002CA0D1BCE757
:1085800040F227613846FAF795F93388D3E7284651
:108590004946FBF7A5FE002C92D1AEE7284606F02F
:1085A00031FC002000F0EAFF0028A4D107F0D2FB44
:1085B000002C85D1A1E701904FF4C2613846FAF74B
:1085C00079F9019BD5E700BFBCD30100C03700207B
:1085D000A83900200148FBF769BE00BFC43700205E
:1085E0000149FBF77DBE00BFC43700200148FBF7FF
:1085F0005DBE00BFA83900200149FBF771BE00BF76
:10860000A8390020024B034A5B790B70FBF7B2BE1E
:108610000404002060450020014B18680EF034BCB3
:10862000744500200E4B19795A7991420AD8A2EB71
:10863000010C5FFA8CFC604502D8914218780AD18F
:1086400000207047B3F802C0ACEB010C6244D2B218
:108650009042F5D8187801FB00339868704700BF46
:1086600040020020094B19795A79187893F802C012
:108670008A4209D04A1CD2B201FB0031944508BF9E
:10868000002288681A71704700207047400200205D
:1086900038B5114A92F805C0947892F804E015783C
:1086A0000CF10103DBB29C4208BF00239E450AD0B7
:1086B0001CFB05FC02F1080E2EF80C00F444CCF86B
:1086C0000410537138BD054840F27961FAF7F2F8A9
:1086D00000231B80FFDE00BF04040020BCD3010088
:1086E00030F0020310B50C4602D00B68022B08D004
:1086F0004FF0FF324FF0FF3305480EF0EBFB2068E0
:1087000010BD044840F2AD61FAF7D4F8F0E700BFBD
:1087100078450020BCD30100034A0346106800B12D
:1087200070471360184670478C370020044A13685E
:1087300023B1984206BF00211160002318467047FC
:108740008C370020014B1868704700BF8C37002021
:10875000034A0346106800B170471360184670471B
:1087600090370020044A136823B1984206BF0021C5
:10877000116000231846704790370020014B18689D
:10878000704700BF9037002030B505682B7887B060
:1087900013B3044601220021684613F090FF2B78A2
:1087A0000F4AC5F818D06A61B3B10E4B00221146CA
:1087B00003209C60FBF752FE40B94FF0FF324FF0B0
:1087C000FF3368460EF086FB07B030BD064840F226
:1087D0002A71FAF76FF8F0E76FF07700F4E700BF5F
:1087E0008D7E00008C040020BCD30100F0B5284D24
:1087F0002B6885B00C461646002B3AD099421AD108
:108800000223039303AB024600930321214B002074
:10881000FDF72AF930F0020311D11F484FF0FF3263
:108820004FF0FF330EF056FB039F8FB12B680BB157
:108830009C4220D04CB36FF02D0005B0F0BD039BDF
:10884000022BEAD1154840F2AD61FAF733F8E4E7BC
:108850003046FFF799FF2B680BB19C4211D0002CDA
:10886000E9D10028E9D010F1780F08BF002005B049
:10887000F0BD2960C4E700236FF077002B6005B0DE
:10888000F0BD2F600028D8D0EDE76FF07700D4E777
:108890008C370020817E000078450020BCD3010089
:1088A0000E4B19795A7991420AD8A2EB010C5FFA62
:1088B0008CFC604502D8914218780AD1002070479C
:1088C000B3F802C0ACEB010C6244D2B29042F5D8CE
:1088D000187801FB00339868704700BFCC02002075
:1088E000094B19795A79187893F802C08A4209D04D
:1088F0004A1CD2B201FB0031944508BF00228868AF
:108900001A71704700207047CC02002038B50C4621
:10891000054605F0C5FD21462070034A2846BDE8FE
:108920003840FBF727BD00BF704500200122024BF5
:1089300011460020FBF792BD7C0400202DE9F04792
:10894000164E9DF820A0994673790F465D1C11467E
:10895000B278EDB2AA4208BF00253279AA42804619
:10896000307816D006F1080403FB0044102220469C
:1089700012F0BAFA237FA7610AF0010A23F0030379
:1089800043EA0A03C4E90498237775712046BDE8D9
:10899000F08700242046BDE8F08700BFFC020020DD
:1089A000054B18795A79197882421ABF083300FBAF
:1089B00001300020704700BFFC02002000B50D4BC5
:1089C0000278997893F805C093F800E091429CBF33
:1089D0001A79027094450AD0531CDBB2994208BF41
:1089E00000230549037002FB0E105DF804FB002014
:1089F000FBE700BFFC020020040300202DE9F04744
:108A00001F4C227961792378914227D004F108061E
:108A1000DFF87080DFF87090074602FB0360037F89
:108A20009A07C3F3400A03F0010519D52279617949
:108A3000207894F802C0531C9142DBB20ED09C45C2
:108A400008BF00239942237108D003FB0060BAF1EC
:108A5000000FE4D115B1037FDB07E0D5BDE8F08757
:108A6000C8F80800074B524651463846FBF7F6FC5B
:108A70000028DBD040F2A1714846F9F71BFFD5E78B
:108A8000FC0200204C040020BCD30100064B1A79E4
:108A900059791878914205D002FB0033986810B1DB
:108AA00020307047002070472402002070B5134A20
:108AB0001379547911789C42064690781BD003FBB9
:108AC000012101338C68DBB2984208BF0023137187
:108AD0007CB1022300252068094A237121462560C4
:108AE000E661FBF747FC0122064B11462846FBF7DF
:108AF000B5FC204670BD0024FBE700BF2402002027
:108B0000684500206C0400202DE9F04F83B01D461D
:108B10000C9C9DF83C30CDE90004DDE90DA93BB388
:108B20005C1E95F800B088461746E4B20BF10103CD
:108B30005FFA83FBD84508BF4FF0000B5F454846FE
:108B400016D0FBF7B3FB064650468EB1FBF7AEFBE3
:108B500088B10023736006602A78009B12FB03F241
:108B6000019B9850013CE4B2FF2C85F800B0DDD1A8
:108B700003B0BDE8F08F4946304603B0BDE8F04F82
:108B8000FBF7AEBB70B5334C334DA279A188334EA1
:108B9000002084B02346A88004F10800FBF756FBB0
:108BA000E379A279301D1A4408213346FBF74EFBC6
:108BB00002962E46A37916F8080B2A79A978039312
:108BC000CDE900646B1DFFF79FFF254B2C22181D7C
:108BD0004421FBF73BFB234B3C22181D0821FBF7EC
:108BE00035FB2048FBF762FB044608B31E4A2046CB
:108BF000111FFBF7B1FB1948FBF758FB0446E8B11E
:108C00001A4A2046111FFBF7A7FB1648FBF74EFB3D
:108C10000446C8B1164A2046111FFBF79DFB154BB1
:108C20002922FF201A80FFF793F9002004B070BDBD
:108C3000114840F62D01F9F73DFED7E70E4840F602
:108C40003501F9F737FEDBE70B4840F63D01F9F750
:108C500031FEDFE74C010020240200209437002081
:108C6000A8390020C4370020704500206845002046
:108C700060450020C0370020BCD3010030B52C4B2C
:108C80002C4D186087B00AF02FF9FBF795FB2A4AA4
:108C90002A4C2B49CDE904252A4A0220CDE9022499
:108CA00004230C24CDE90014274A087408760B70BD
:108CB0000B7200201521FCF79BFD002832D1012208
:108CC0000021224813F0FBFC07F018FE044610B107
:108CD000204607B030BDFFF755FF04460028F7D106
:108CE00008F0E0F904460028F2D100F0FFFB04464A
:108CF0000028EDD109F072F804460028E8D100F010
:108D000083FD04460028E3D109F088F904460028D1
:108D1000DED102F085F804460028D9D1012006F002
:108D200099FFD5E70A4840F21F21F9F7C3FDC6E7CE
:108D300074450020FD3E0100253E0100ED3D01008F
:108D4000F04B00208049002090450020784500200D
:108D5000BCD3010010B586B000F0D8FB002834D198
:108D600000F054FD002839D102F05CF800283ED113
:108D70002C4B00249C80204606F06CFF2A492B4A8D
:108D80002B4B8C8094809C8001222146684613F0F6
:108D900096FC284B224621460320C3F808D0FBF757
:108DA0005DFB002837D14FF0FF324FF0FF336846AC
:108DB0000EF090F800F0B0FB38BB68460AF056F8A9
:108DC000FFF7E0FEC8B906B010BD1B4840F2BF2156
:108DD000F9F770FD00F01AFD0028C5D0164840F2E2
:108DE000D121F9F767FD02F01DF80028C0D0124824
:108DF00040F2F121F9F75EFDBAE70F4840F23A314F
:108E000006B0BDE81040F9F755BD0B4840F22D31D2
:108E1000F9F750FDD1E708484FF44871F9F74AFDDA
:108E2000C1E700BF04040020FC020020CC020020A7
:108E3000400200205C040020BCD3010010B582B0C9
:108E40000024CDE90044049B07F030FF02B010BDC0
:108E500010B50346007F1A699969012482B0204049
:108E6000CDE90004586907F021FF08B1773001D13E
:108E700002B010BD03484F2102B0BDE81040F9F721
:108E800019BD00BFF8D30100F8B505682F6E06467E
:108E9000D7B16C6E00232B660CB3002117236966D3
:108EA00023714FF6FF73E3801E2204F11C0012F0C1
:108EB00026F83C232377A66021463846FFF7A2FB1D
:108EC000BDE8F840FFF7A8BB084840F63811F9F7AD
:108ED000F1FC6C6E2F6E00232B66002CDDD1034855
:108EE00040F63C11F9F7E6FC6C6ED6E73CD4010085
:108EF00000B17047084B10B502460C460220012114
:108F00009C60FBF7ABFA00B910BDBDE81040034808
:108F100040F60C11F9F7CEBCBC0400203CD4010093
:108F200038B5044610F81C3BDBB1104D6369A860EE
:108F30002BB10F4840F62111F9F7BCFCA8680D4988
:108F40000A4B0022C4E9051011460120FBF786FAFE
:108F500000B938BDBDE83840054840F62811F9F79A
:108F6000A9BCBDE83840FFF78FBF00BFAC040020AC
:108F70003CD40100898E000000B9704710B50C4642
:108F8000FFF7E0FB844206D0BDE81040024840F6FF
:108F9000DD01F9F78FBC10BD3CD4010030B583B0C2
:108FA000124B079D124AEB1AA2FB032313F47F5FB7
:108FB000C3F3871414D1A21C0E4B0095D2B2012129
:108FC0000020FCF751FD30F0020307D00A484FF4AF
:108FD0000F6103B0BDE83040F9F76CBC03B030BDA1
:108FE000054840F6EB01F9F765FCE4E7284C002062
:108FF00089888888F18E00003CD4010000B5134BAD
:109000009A8C93F8291093F86AC003EB810122F43B
:10901000437222F00202C96A42F00E029A840620CC
:1090200000224FF4006E6FF3420CA3F868E083F85F
:109030006AC048700A7093F8351003EB810304226C
:109040009B6B58701A705DF804FB00BF284C002021
:1090500070B5134C256AAB6D23B1124840F666110A
:10906000F9F728FC05F14C0105F14800FBF778F908
:10907000064670B12868AE6501F0FEFA0025606E04
:109080002562FFF7B9FA206E6566FFF7A9FA256633
:1090900070BD044840F66811F9F70CFCEAE700BF20
:1090A000284C00203CD4010030B5434C94F86A3081
:1090B000D90785B047D5236A53B193F8202042F0F1
:1090C000020283F82020236A93F82030DA0755D46F
:1090D0003948FFF721FB844204D0384840F61D216F
:1090E000F9F7E8FB94F82430DB0703AD2ED4022215
:1090F0000321334B009500200392FCF7B5FC294671
:10910000FFF7EEFA00284BD12E48FFF73DFB08B1E0
:10911000783036D12848FFF709FB844204D027482D
:1091200040F63F21F9F7C6FB236A0BB1FFF790FF2A
:1091300094F86A306FF3000384F86A30002000F07E
:109140002FFC044640B3002005B030BD022103913E
:109150001B4B0095032101220020FCF785FC2946CA
:10916000FFF7BEFA0028C2D01348FFF7DFFA8442A7
:1091700004D0124840F62821F9F79CFB0C2005B0DA
:1091800030BD0E4840F63C21F9F794FB0A48FFF742
:10919000CDFA8442C3D1C7E706F0DCFD2046D3E711
:1091A0000548FFF7C3FA8442E8D0044840F6362168
:1091B000F9F780FB0C20C7E7284C00203CD40100C5
:1091C000817E0000444C002010B4047804F00F04A9
:1091D000531E022C1FFA83FC1FD0012C09D0103122
:1091E000C9008CB1062C0FD04FF42A734FF4F372E0
:1091F00003E04FF4876340F216220CFB02334FF674
:10920000FE70184010BC704743781033DB0001F546
:109210005C7103F5B3720B44EFE7407810BC0CEBC4
:109220008C03C3EB031310305B00C10003F5C8705F
:1092300001FB020080B270472DE9F0411D468AB063
:109240004FF6FF739D429DF84060119C17D0237824
:109250000133DBB2074690462370002B52D02C49D5
:109260002C4B0D8104F11C000022C860C1E900787C
:109270008E72996001201146FBF7F0F838B994F826
:10928000240010F001050CD00AB0BDE8F08122489E
:1092900040F6AF01F9F70EFB94F8240010F0010539
:1092A000F2D1042109A807F07FFB099B1B4A069411
:1092B000A2FB0312991A02EB5102120A40F2471163
:1092C00001FB1233164A1749A21AA1FB0212920996
:1092D000154902320133CDE90451CDE90255CDE9FA
:1092E0000055D2B2012128460993FCF7A5FB30F0C6
:1092F0000203C9D0084840F24471F9F7DBFA0AB01A
:10930000BDE8F081044840F6A201F9F7D3FAA6E7D8
:10931000AC4C00209C0400203CD4010021F1D490EE
:10932000284C002089888888798F00002DE9F04733
:10933000694C1F46694B94F86A6080468E4693E8F4
:10934000030082B016F0010615469DF82CC09DF86A
:10935000302000908DF8041040F089800CF0070C4C
:1093600002F003024FEA4C0C4CEA022C94F829203C
:10937000BEF1010F04EB820208BF4FF0000802AB00
:10938000A4F868809E44D2F82C80A28C98F800A0A3
:109390001EF8083C22F4437213F00E0F22F0020272
:1093A0002AF01F0103F00F034CEA020C43EA010309
:1093B0000CBF0122002262F34513A4F824C088F8F0
:1093C000003003F00F03012B0AF00F0A46D094F887
:1093D0006A3065F3420384F86A30DAB25B0708D575
:1093E00067F3C30284F86A203D480A99062211F007
:1093F0007BFD98F8003003F00F02012A05F0010907
:109400003AD098F80120FAB1BAF1010F4FD098F88C
:10941000003069F386136FF3C71388F8003094F8AF
:109420003530E46104EB8304AD01A36B05F0400526
:109430005A7845F004051D7012B906215970164678
:10944000304602B0BDE8F08769F3861362F3C713B4
:1094500088F80030062388F80130E0E7BAF1010F00
:10946000B5D098F80120B2B984F84060AFE70C2677
:10947000304602B0BDE8F087404669F3861367F3D3
:10948000C71300F8083B0A99062211F02DFD0C23A2
:1094900088F80130C3E7052A16D9063AD2B284F813
:1094A000402008F108010F4811F01EFD8FE794F8E5
:1094B00040200C4908F1080011F016FD94F84030E6
:1094C000063388F80130A2E707484FF4CE71F9F768
:1094D000F1F998F80120E0E7284C002058D101006C
:1094E000934C0020694C00203CD4010010B5064C80
:1094F00004F1280007F006FE04F1340007F002FE34
:10950000FFF77CFD002010BD284C002008B5FFF7B8
:10951000CBFD002008BD00BF38B50A4C04F128057A
:109520002846343407F0FEFD204607F0FBFD2846B0
:1095300007F0E8FD204607F0E5FDFFF75FFD00209E
:1095400038BD00BF284C0020034A044B801AA3FBFF
:109550000030C0F38F107047284C0020898888881D
:10956000044A0068044B801AA3FB0030C0F38F103C
:10957000704700BF284C00208988888838B9054882
:1095800090F86A3013F0010F08BF002070470020E8
:10959000704700BF284C002028B9044B93F86A009C
:1095A00000F0010070470020704700BF284C0020E9
:1095B00050B9064B93F86A0010F0010005D093F8FB
:1095C000250000F00300704700207047284C002061
:1095D000F8B50C46064690F8260006F01FFD2378E5
:1095E0000546C3F38010FCF707FB06220746014639
:1095F00006F1710011F078FC85B1237843F0400347
:109600002370A71C06222946384611F06DFC2378EA
:1096100003F00F03012B03D03846F8BD3D46F0E7B9
:1096200096F8260006F01CFD01460028F4D02378A9
:10963000204643F0800300F8083B062211F054FC5A
:109640003846F8BD1F2949D8F0B590F8293000EB0D
:10965000830383B0DE6A337803F00F03012B0D46DA
:10966000044617463CD00DF10701283007F0BAFD3B
:109670003146064611F8022BC2F34010C2F3030331
:1096800043EA4013C2F3801043EA801302F08002E1
:109690003046134300F8023B062211F025FC2A460F
:1096A000394606F10800063511F01EFC757094F875
:1096B0006A30DB0706D49DF8073084F82930002093
:1096C00003B0F0BD94F8353004EB830331469A6B58
:1096D0002046F7F71DF90028EDD0F1E7122070477A
:1096E00080F840100A464130394611F0FDFB002059
:1096F00003B0F0BD03460A4601481946FFF7A2BF72
:10970000284C0020F0B590F8353000EB830383B08F
:109710009D6B0E4604460DF107013430174607F0E5
:1097200061FD2946062211F8023BC3F380139B0119
:1097300043F004030370B31D43700546023011F07B
:10974000D3FB3246394605F1080011F0CDFB94F801
:109750006A30DB070AD594F8293004EB8303D96A11
:109760000B7813F00F0308D0062B06D09DF80730B6
:1097700084F83530002003B0F0BD2A462046F7F7C4
:10978000C7F80028F2D0F6E71F2803460A4603D898
:1097900002481946FFF7B6BF12207047284C002038
:1097A0002DE9F843099C9DF820802546814615F84F
:1097B0001C1B0131C9B217461E46217081B10F4CE6
:1097C0000F4B2681002211460120C4E90097E56075
:1097D00084F80A809C60FAF741FE38B9BDE8F88346
:1097E00008484FF43E71F9F765F8E8E7BDE8F8433B
:1097F000044840F20531F9F75DB800BF0C4D002078
:10980000CC0400207CD401000020704770B5154DB9
:10981000002405F11C0644B995F8444014F00104F5
:1098200003D02B6A0F4932460BB1002070BD0420D3
:10983000FEF7DCFF034638B17833F6D00A4840F231
:10984000FB11F9F737F8F0E795F8442060F30002D0
:1098500085F84420FFF792FE0028DCD106F07AFA62
:10986000D9E700BFC44C00207CD4010038B5324C8D
:1098700094F8443003F0010258B35ABB9A07C3F37B
:1098800041050BD50120FCF7B7F90621FAF758FD81
:1098900000284AD094F84450C5F3410594F83200AA
:1098A000C0F3C10006F096FA94F8333094F83220F1
:1098B0006FF34103FF2184F83330930684F83410AA
:1098C00002D5023D012D1AD9BDE838401A48F7F7F4
:1098D000DBB80AB90C2038BD236A002BFAD104F199
:1098E0001C0221460420FEF781FF054688B1783529
:1098F000F0D0124840F2FB11F8F7DCFFEAE7002055
:1099000006F08CFA94F8333043F0020384F83330D5
:10991000DAE794F8443060F3000384F84430FFF74A
:109920002DFE044618B1284638BD122038BD06F079
:1099300011FA204638BD00BFC44C00207CD4010081
:10994000043008B501F11C02C0B2FEF74FFF10B1A0
:10995000783001D10C2008BD034840F2FB11F8F724
:10996000A9FF0C2008BD00BF7CD40100034A044BB2
:10997000801AA3FB0030C0F307107047C44C0020CE
:10998000398EE338044A0068044B801AA3FB003088
:10999000C0F30710704700BFC44C0020398EE33875
:1099A00038B9054890F8443013F0010F08BF002083
:1099B00070470020704700BFC44C0020044A92F852
:1099C000443003F0010303430CBF104600207047EE
:1099D000C44C002090B90A4A92F8443013F00100B8
:1099E0000DD092F83200126A03F00103C0F3401068
:1099F00003FA00F01AB140F00400704700207047ED
:109A0000C44C002050B9064B93F8440010F00100FC
:109A100005D093F83200C0F3C100704700207047B2
:109A2000C44C00204B070CD5800100F574739342A1
:109A30004FF4296028BF1346984238BF184680B2B9
:109A4000704701F0030C604400F10D03C1F34001C5
:109A5000DB00CB40B3F5A47F38BF4FF4A4739BB2B7
:109A60000CF1280093424FEAC00020FA01F028BF11
:109A70001346984238BF184680B2704710B5154B50
:109A80001548164C10224FF4F871FAF7DFFB144B0F
:109A90000722181D2421FAF7D9FB124B4022181D6A
:109AA0002C21FAF7D3FB104B4722181D0821FAF797
:109AB000CDFB0E490E4A0F4807234FF01B0CA4F8AC
:109AC00000C00B704FF4A47C1370A0F800C00020FD
:109AD00010BD00BF1C4D0020E00C0020C66D002012
:109AE000484D0020484E00204C590020D66D0020E3
:109AF000D56D0020C86D00202DE9F043D0F800801E
:109B00002C4983B005464FF4F8724046FAF704FC3E
:109B100005F14806294608F093FAE86C01AA314697
:109B2000FAF73AFC28B3244C4FF6FF7704F1080902
:109B3000627994F802C02179531CDBB29C4508BFBE
:109B40000023994294F800C02BD0019912FB0CF22B
:109B500009EB020C29F802700A68CCF804100260C4
:109B60000860E86C637101AA3146FAF715FC002819
:109B7000DED1D8F8540108F5AA7450B1002321466B
:109B8000C8F85431FEF7C2FEFEF7D0FE03B0BDE8C0
:109B9000F0830A4840F6EE11F8F78CFED8F854012D
:109BA000ECE7064840F6DA11F8F784FE00231B8044
:109BB000FFDE00BFE00C0020DC040020BCD401006C
:109BC00010B50C4640B90B4B0022012102209C60CD
:109BD000FAF744FC30B910BD074840F68E11F8F78B
:109BE00069FEF0E7BDE81040034840F69411F8F72D
:109BF00061BE00BF9C070020BCD4010008B5084B23
:109C00000022986011460120FAF728FC00B908BD2F
:109C1000BDE8084003484FF41C61F8F74BBE00BF95
:109C20006C070020BCD4010083685A68537FDB09AD
:109C300000F1080101D0F7F747BBF7F7D5BF00BF28
:109C400010B50C4660B92046FEF78CFD844206D064
:109C5000BDE81040054840F6C201F8F72BBE10BD24
:109C6000024840F6BF01F8F725FEECE7BCD401003E
:109C700010B50C4660B92046FEF76AFD844206D056
:109C8000BDE81040054840F6B801F8F713BE10BD16
:109C9000024840F6B501F8F70DFEECE7BCD4010030
:109CA00000B9704710B50C46FEF768FD84420AD033
:109CB000FEF748FD844206D0BDE81040024840F659
:109CC000AC01F8F7F7BD10BDBCD4010010B4D0E969
:109CD00075240346084664B1944221D0D3F8E011BC
:109CE0008A420BD01168C3F8D411002210BC026064
:109CF0007047D3F8E011914204D18AB10968C3F8E2
:109D0000E011EFE7117901F00301032913D0126884
:109D1000C3F8D4210022C3E9762210BC006070474A
:109D2000D3F8DC111268C3F8D421A14218BFC3F8DC
:109D3000D821F2D1EEE7D1790329D3D00A29E6D18F
:109D4000D0E700BF38B5044610F81C3BDBB1164D18
:109D50006369A8602BB1154840F6A911F8F7AAFD70
:109D6000A8681349104B0022C4E9051011460120D0
:109D7000FAF774FB00B938BDBDE838400B484FF422
:109D80001B61F8F797BD03F0FF020A4B114698607C
:109D90000120FAF763FB0028EDD0BDE83840034806
:109DA0004FF41C61F8F786BD8C070020BCD401007D
:109DB000FD9B00006C070020F8B5044690F8E40015
:109DC00087070D4633D42E4817461E46FAF76EFA1B
:109DD000002838D094F8E43043F0020384F8E430EB
:109DE000032343711122D4F8D431C2710279D4F81B
:109DF000D811077242F0030246720271DBB194F887
:109E00007621960717D494F8CF21D20713D4D4F82B
:109E1000E021934222D0C9B1D4F8DC311A68026043
:109E200018600368C4F8DC010BB9C4F8E40101232D
:109E30002B710020F8BD0029EED10360C4E9750044
:109E4000C4F8DC01F0E76FF06800F8BD1A7902F0A1
:109E50000302032A0ED0C4F8D831DFE71A68C4F829
:109E6000E0210029D8D11A68026018600368C4E9AB
:109E70007600D9E7DA79032AF5D00A2AEBD1F2E79E
:109E8000484E002038B590F87631D0F8D8210D46EC
:109E90009907044612D5002A3CD0D0F8DC311A6864
:109EA0002A601D602B6833B138BD42BB2A60C0E90F
:109EB0007555C0F8DC51C4F8E45138BDD0F8D41160
:109EC0000029F2D090F8F0C090F8CF3190F8F1006E
:109ED000844503D094F8F200032823D013F0010343
:109EE0000BD1D4F8E00181423DD072B33BB12D4893
:109EF00040F68221F8F7DEFC01E0002A43D0D4F8D6
:109F0000DC311A682A601D602B68C4F8DC51002B14
:109F1000CAD1D0E7D0F8D4312B60C0F8D451002B8F
:109F2000C2D1C8E7087900F003000328D6D1C87968
:109F3000032801D00A28D1D1DB072AD57AB11948E4
:109F400040F69421F8F7B6FCD9E70A7902F003024B
:109F5000032A20D0C4E97611002BD0D0C7E72960AE
:109F6000C4F8D45138BD0868C4F8E001002ABDD156
:109F70000A682A600D60002B94D12B68C4E97655DD
:109F8000002B91D197E72960C4E97555C4F8DC51DD
:109F900038BD0123A5E7CA79032AE9D00A2AD9D115
:109FA000E6E700BFBCD401002DE9F84390F8E46077
:109FB00016F002060F466DD105463A489146FAF76B
:109FC00075F9044600286AD095F8E430364943F024
:109FD000020385F8E430D9F80420D9F80830114399
:109FE000D5F838210A40C5F8382103F0FF03D5F829
:109FF0003C2143F010031340C5F83C31D9F80480EC
:10A00000D9F80890FDF7FCFE274B48EA030303400C
:10A0100003F0FF0028F0FF03034343F0076343F41A
:10A020000323C5F8403195F8E43043F0010385F887
:10A03000E430237909F0FF0949F0100243F00303EB
:10A04000C5F844210822237109236371E371A01824
:10A05000314610F054FFFDF7D3FED5F838312173A7
:10A06000034003F0FF0320F0FF0003431A0C2372A8
:10A07000A272C3F30723120A284663726673A6739B
:10A08000E673E2722146FFF7FDFE01233B71304685
:10A09000BDE8F88301230B710020BDE8F8836FF061
:10A0A0006800F5E7484E0020D0307808F8B590F801
:10A0B000BE3103F007020446062A00F2EA80DFE818
:10A0C00002F004515151525251007548FAF7EEF81E
:10A0D000002847D094F8BE11B4F8C221B4F8C631B4
:10A0E000A4F8D2200125A4F8D43065F3020184F845
:10A0F000BE1182810279092142F00302417102718D
:10A100001B22027294F8E4201421C171D7074FF08A
:10A1100000014172D4F8381101D50E0570D44FF406
:10A12000A4731946D4F8D421C3814181D4F8D8311D
:10A130003AB194F876118D0703D494F8CF11C9077A
:10A1400079D5002B00F08580D4F8DC311A680260E4
:10A1500018600268C4F8DC01002A4ED0B4F8C6309A
:10A16000A4F8C830F8BD03F00702B0F8C0C1B0F8D9
:10A17000C411B0F8C271B0F8C661A0F85AC0042A80
:10A18000A0F85E1024D0062262F3020380F8BE31EC
:10A19000D4F8145135B3286820B32B7F4268C4F833
:10A1A000142143F00303228D2B770923EA806B7778
:10A1B000032215236984A5F820C0AF84EE842946C4
:10A1C0002A71EB77FEF71EFABDE8F840FEF724BAD5
:10A1D000B0F8C8210ABB90F8BC31A0F8C82080F8BC
:10A1E000BD31D5E72F4841F2D401F8F763FB286869
:10A1F000B4F85AC0B4F85E10CFE7C4F8E401ADE794
:10A20000B3F5296F28BF4FF42963B3F5A47F38BF96
:10A210004FF4A4734FF4296184E7A0F8C22100220F
:10A2200062F3020380F8BE31B0F8CA31A0F8C82149
:10A23000A0F8C631ACE7D4F8E0118A420FD0D3B110
:10A24000D4F8DC211368036010600268C4F8DC01F4
:10A2500082E70260C4E97500C4F8DC017CE711689C
:10A26000C4F8E011002BEBD11368036010600268A2
:10A27000C4E9760070E7137903F00303032B02D0DF
:10A28000C4F8D821DEE7D379032BEDD00A2BF7D120
:10A29000EAE7BDE8F840034841F2FE01F8F70ABBDF
:10A2A000484E0020BCD401002DE9F04F90F8F45046
:10A2B00015F0010783B004460E4640F09D80B0F8CB
:10A2C000F610711A090400F19E8090F93920002AD5
:10A2D000C0F22481D0F81461AB4694F8F02084F8E1
:10A2E000F12094F8612094F86090B4F85E8002F058
:10A2F000070394F8E4200193D20709F0070900F15D
:10A3000094804FF4A47ACDF800A015F01C0F7DD1F5
:10A31000B4F85C7015F0E00F0CD094F8612094F85C
:10A320005A00690961F3020284F86120009AFFF77C
:10A3300079FB8046002E00F0E1803068002800F0B4
:10A34000DD8094F8602094F861C04168C4F814116D
:10A350001BF0020FC2F30205CCF3020102F0070268
:10A360000CF0070C02D1914500F0F480238DF380AE
:10A370001D23337100237577B17733773146FEF7AC
:10A3800041F9D4F81451002D00F0C180286800284C
:10A3900000F0BD80B4F85C204368C4F81431BA42C0
:10A3A00009D3524507D8B4F85E30434503D3009A29
:10A3B000934240F20481A4F85C70A4F85E802B7F85
:10A3C000228DEA8043F003030921032669772E7169
:10A3D0002B77B4F85A302B84B4F85830AB8415235B
:10A3E000A5F82280EF842946EB77FEF70BF903B03E
:10A3F000BDE8F04FFEF710B9D0E919010022F9F7D6
:10A40000C3FF054630B303B0BDE8F08F94F8602079
:10A4100094F85800C5F3820161F3020284F86020C9
:10A420005246FFF7FFFA074674E7D4F838211305C0
:10A430007FF567AFB4F8D4A0BAF5296F28BF4FF401
:10A44000296ABAF5A47F4FF4296338BF4FF4A47A80
:10A4500000935AE70220FEF7E5F880460028D2D0A4
:10A460008048F9F723FF07460028CCD094F8F43051
:10A4700065F30003C3F3421545EA930515F007059C
:10A4800084F8F430DBB27CD194F8F020A4F8F650D4
:10A490009E0784F8F12000F19E802B462A467B72AD
:10A4A00005233D727B717A811822D4F8D431D4F817
:10A4B000D811FA713A7942F003023A71002B00F098
:10A4C000828094F8762195077DD494F8CF21D00727
:10A4D00079D4D4F8E021934200F0A980002900F05B
:10A4E000B380D4F8DC311A683A601F603B68C4F866
:10A4F000DC71002B87D1C4F8E47184E75A4841F23B
:10A500002E21F8F7D7F9306894F8F4B019E75648D7
:10A5100041F25D21F8F7CEF928683BE7FEF7A2F893
:10A52000064600283FF46FAF0368D4F814215A6040
:10A5300094F9393094F8F450C4F81401002BAB4668
:10A54000BFF6CBAE94F8E520002A3FF4C6AE84F8FF
:10A55000E570C6E6019B63457FF408AF01233371C4
:10A560003146FEF74FF8D4F81451002D58D0286822
:10A57000002855D04268C4F81421012329462B71C4
:10A5800033E7A38DB11D1944A4F8F610FEF76AF85D
:10A59000D8F80030D4F814215A60C4F81481FEF7BA
:10A5A00061F80368D4F814215A6094F8F430B4F8D0
:10A5B000F620C4F81401C3F382055B096FE7012399
:10A5C0002B71294611E700298BD13B60C4E97577CF
:10A5D000C4F8DC718DE7FEF745F8238DA8F8063046
:10A5E0001D2388F81C5088F8043094F86030D8F89F
:10A5F0000000C3F3020388F81D3094F86130C3F300
:10A60000020388F81E304146FDF7FCFFFEF704F810
:10A6100094F8F430B4F8F620C3F382055B093EE702
:10A6200011484FF49251F8F745F92868A2E71A68E3
:10A63000C4F8E02100297FF454AF1A683A601F6023
:10A640003B68C4E9767754E71A7902F00302032ADB
:10A6500002D0C4E9763344E7DA79032AEDD00A2A36
:10A66000F7D1EAE7484E0020BCD401000148F9F7D1
:10A670001DBE00BF1C4D00200149F9F731BE00BFCF
:10A680001C4D002002494FF4F872F9F745BE00BF97
:10A69000E00C002002464FF4F8710148F9F738BE8B
:10A6A000E00C00200F280CD810B5044622464FF4C9
:10A6B000F8710548F9F72CFE038DA34218BF00205E
:10A6C00010BD0020704700BFE00C00200148F9F7E2
:10A6D000EDBD00BF484D00200149F9F701BE00BFA4
:10A6E000484D00200F2800F2C2802DE9F0410746B6
:10A6F0000C4663483A464FF4F871F9F709FE038DAA
:10A70000BB42804640F08C805E4D6A79A9782878FB
:10A71000531CDBB2994208BF00232979994200F00B
:10A72000958012FB00F205F108018F520A44546033
:10A730006B7198F8003003F0FF00002B79D0524D78
:10A740002B68062B3AD8514E514B00220121032091
:10A75000C3F80880F9F782FE98F93930002B70DBD6
:10A760004C4F11F0D1FC3A684B49A0EB020CCCF3F2
:10A770000E03A3FB01234FEADC3CD20B42EA434227
:10A78000ACFB01C312EB0C0243F100034FF0000CD1
:10A7900091427CEB030147D340482F6801680137A1
:10A7A00064790C4404603E48A4FB00012144F5F7A1
:10A7B000A7FC2F6030600020BDE8F08198F87A3067
:10A7C00098F86000314E37493268B1FBF2F2C3F3BA
:10A7D00000139B0000F0070CC0F3C00110F0040050
:10A7E000DBB237D163440CF1090124334FEA6C0C1E
:10A7F000C900DB0021FA0CF123FA0CF301F5967C79
:10A8000063449A4209D9C3EB420001F196035B000D
:10A8100018440138B0FBF3F0C0B207F09FFF93E794
:10A820006FF01500BDE8F081386061461B480127D4
:10A83000B6E707F093FF98F93930134D134E002B0C
:10A840008EDA3946404604F02DF989E76FF068004A
:10A85000BDE8F0811D33DBB2DB0049001B33013161
:10A860008B4003F274539A4204D80020D5E76FF06E
:10A8700015007047C3EB420040F2CC63C8E700BF4D
:10A88000E00C002024070020985B0020A05B002043
:10A890007C070020244D002000CA9A3B9C5B0020CE
:10A8A0000050D6DC00E6DF0C2DE9F0470F28BDF89C
:10A8B0002090BDF82480BDF8287036D882460C461A
:10A8C000434815464FF4F87152461E46F9F720FDED
:10A8D000038D5345844628D154BB90F89631990690
:10A8E0004BD490F8E430DA0743D49CF894219CF8D8
:10A8F000953193423AD1BCF89621ACF8986102F0B8
:10A90000E00242F01002ACF896219CF93920ACF834
:10A910009A910133002AACF89C81ACF89E718CF8B6
:10A9200094314FDB0020BDE8F0870220BDE8F087BE
:10A93000013C14F0FF04D8D090F8952190F89431A0
:10A940009A4213D090F8963103F00F02032A0DD1EA
:10A9500004F00F0423F01F0344F010041C4380F89C
:10A96000975180F896410020BDE8F0870C20BDE8A3
:10A97000F087D0F838319B07B7D49CF93930002BD9
:10A980001EDB9CF818219CF819319342EED19CF8FB
:10A990001A21ACF81C9101338CF8183122F00F0207
:10A9A000012342F0090200208CF82831ACF81E8106
:10A9B000ACF820718CF81A21CCF82401BDE8F0879E
:10A9C0001A20B3E76046514604F06CF80020ADE76A
:10A9D000E00C00200F281DD8F8B506460D460E489D
:10A9E00032464FF4F871F9F793FC038DB3420446F5
:10A9F0000ED100F13407002684F8E86105223946BB
:10AA0000284610F071FA94F8E8010028F4D1F8BD56
:10AA10000220F8BD02207047E00C00200F2840D82B
:10AA200038B505460C4622482A464FF4F871F9F726
:10AA30006FFC038DAB4225D190F8503190F8512135
:10AA40009A422CD1292C19D8042C19D9621F242AF6
:10AA500016D8DFE802F01915151515151515151579
:10AA60001515151519191915151515191515151586
:10AA70001515151515151515151519003B2C03D0B1
:10AA8000122038BD022038BD90F9392080F852419B
:10AA90000133002A80F8503105DB002038BD0C203E
:10AAA00038BD02207047294603F0FCFF002038BD66
:10AAB000E00C00200F2821D810B504464FF4F8719F
:10AAC0000F482246F9F724FC018DA1420ED190F8DF
:10AAD000304190F83121A2420AD190F93940013237
:10AAE000002C80F8302105DB002010BD022010BDB5
:10AAF0000C2010BD03F0D6FF002010BD02207047CF
:10AB0000E00C00200F2821D810B504464FF4F8714E
:10AB10000F482246F9F7FCFB018DA1420ED190F8B7
:10AB2000484190F84921A2420AD190F939400132B6
:10AB3000002C80F8482105DB002010BD022010BD4C
:10AB40000C2010BD03F0AEFF002010BD02207047A6
:10AB5000E00C00201B2935D8B2F5296F70B51646D8
:10AB60002ED80F28044629D802460D4626484FF411
:10AB7000F871F9F7CDFB038DA3421FD190F8BE31D8
:10AB80001A0725D490F8E420D1071DD490F8BC1101
:10AB900090F8BD218A421FD003F00703032B04D095
:10ABA000033303F00703012B14D8B0F8C8318BB975
:10ABB000A0F8C851A0F8CA61184670BD022070BD47
:10ABC000122070BD12207047D0F838219206DDD4D3
:10ABD0001A2070BD0C2070BD90F8BE3190F939106C
:10ABE000A0F8C25101326FF302030029A0F8C66138
:10ABF00080F8BC2180F8BE3101DB002070BD214609
:10AC000003F050FF002070BDE00C0020034A044B0D
:10AC100012881B8802800B80704700BFC66D002021
:10AC2000C86D0020024A034B108019800020704735
:10AC3000C66D0020C86D00204FF01B0CA0F800C0AE
:10AC40004FF42960A2F800C008801880704700BF48
:10AC50000F281BD870B504460E4615464FF4F87100
:10AC600002460B48F9F754FB028DA24203460BD172
:10AC700090F86040C4F30204347093F86130C3F379
:10AC800002032B70002070BD022070BD02207047AF
:10AC9000E00C0020024A034B10701970002070472E
:10ACA000D66D0020D56D00200F282DE9F04143D846
:10ACB00006460C4617464FF4F8710246244898465B
:10ACC000F9F726FB038DB34236D190F8CF5115F03A
:10ACD000080539D190F8E430DB0704D5D0F83831D5
:10ACE00013F4106F30D090F8CC3190F8CD11994218
:10ACF00026D104F00704B0F8CE21A400013144F4B9
:10AD0000806408F0070344EA431307F0010780F862
:10AD1000CC1122F4DF6290F9391043EA472322F084
:10AD2000070213430029A0F8CE3106DA314603F0BA
:10AD3000B9FE2846BDE8F08102252846BDE8F0812D
:10AD40000C252846BDE8F0811A252846BDE8F0818B
:10AD5000E00C00200F2812D838B504460D460948EB
:10AD600022464FF4F871F9F7D3FA038DA34204D1C8
:10AD700090F8BD302B70002038BD022038BD022075
:10AD8000704700BFE00C00200F281DD838B50446DE
:10AD90000D460E4822464FF4F871F9F7B9FA038DC3
:10ADA000A3420FD1418DB0F8CE30094A01FB03F325
:10ADB000C3EB431103EB8103A2FB03239B092B800D
:10ADC000002038BD022038BD02207047E00C002072
:10ADD000D34D62100F281ED838B505462A460F48B5
:10ADE0000C464FF4F871F9F793FA028DAA42034624
:10ADF0000FD1418D40F2E24201FB02F242F21071AA
:10AE000001FB042101390020B1FBF2F1A3F8CE10BF
:10AE100038BD022038BD0220704700BFE00C002082
:10AE2000FEF72CBEF8B503F0CBFF154E154F0025ED
:10AE3000AAB24FF4F8713046F9F76AFA0446681D71
:10AE400004F11C022146C0B20135FDF7CFFC30B140
:10AE5000783040F6F701384601D0F7F72BFD4FF672
:10AE6000FF720023102D22856367E1D10648074950
:10AE7000074A83808B801360BDE8F840FEF7FEBD73
:10AE8000E00C0020BCD4010024070020DC040020DA
:10AE9000204D0020014B1888704700BFC66D002070
:10AEA000014B1888704700BFC86D0020014B18780F
:10AEB000704700BFD66D0020014B1878704700BF67
:10AEC000D56D00202DE9F84F1A4F82468B469046EB
:10AED0009946002501E0102D29D0AEB232464FF43C
:10AEE000F8713846F9F714FA038DB342044605F1B8
:10AEF0000105F0D190F8D630C3F340034345EAD1C1
:10AF000006224946DD300FF0C6FF0028E3D194F851
:10AF1000D63003F001035345DDD104F1D7000622FA
:10AF200059460FF0B8FF0028D5D1012000E00020DD
:10AF3000BDE8F88FE00C002038B58B6808601D680C
:10AF40002B780C4653B16B6923B107484FF47871E5
:10AF5000F7F7B0FC054BC5E9053438BDBDE838400E
:10AF60000846FEF761BE00BFBCD40100299C00006A
:10AF70002DE9F04F0B68DD880F2D87B06DD80E4698
:10AF800007462A467E484FF4F871F9F7C1F9038D58
:10AF9000AB42044660D1356890F876C12B7F03F050
:10AFA0000303032B0CF0010140D195F81F8005F13C
:10AFB0001C02002957D090F93930002B0CF0040105
:10AFC000C0F2E280002940F06C81B8F1020F00F07D
:10AFD0009881B8F1050F00F0A585B8F1060F00F0D3
:10AFE0006885B8F10D0F00F00884B8F1110F2AD16F
:10AFF0006B7F032B76D195F82030033B132B1AD8A7
:10B00000DFE813F02A0619001900190019001900C9
:10B01000190019001900190019001900E805190094
:10B02000190019001900C90519004A064BB911B1D8
:10B030003D2380F8533101232B71002007B0BDE878
:10B04000F08F0029F9D03D220123002084F85321FC
:10B050002B7107B0BDE8F08F3368012200201A7110
:10B0600007B0BDE8F08FB8F1190F3BD801A353F832
:10B0700028F000BFBBB5000053B5000003B30000CB
:10B08000DDB000000DBB00001BBB0000B3BA000028
:10B0900067BA000059BA00007DB90000E9B80000A5
:10B0A00059BB000083B80000FBB70000DBB700000D
:10B0B000BDB7000099B60000F1AF0000F9B900007B
:10B0C00043BA00001BB300001BB30000F1B4000042
:10B0D000F9B3000073B400008FB3000090F9393069
:10B0E000002B60DB94F8E4309807A4D42548F9F7E6
:10B0F000DDF8002800F0E78594F8E43043F002031F
:10B1000084F8E430037980F8088043F00303037186
:10B1100002234371D4F8D4210723C371FAB194F800
:10B12000763199071BD494F8CF31DB0717D4D4F8C4
:10B13000E0319A4200F0CB85D4F8D831002B00F0F2
:10B140001E86D4F8DC211368036010600268C4F81E
:10B15000DC01002A7FF46FAFC4F8E4016BE7D4F898
:10B16000D831002B00F0A585D4F8DC311A680260D4
:10B1700018600268C4F8DC01002A7FF45CAFEBE7DA
:10B18000E00C0020484E0020002900F0B280B8F109
:10B19000020F00F0B680B8F10B0F00F0AB85B8F1EC
:10B1A000030F7FF41AAF6B7F172B9BD194F8F1201C
:10B1B00094F8F0309B1A03F00303022B01F03C8259
:10B1C000CA48F9F773F80646002800F07C85037931
:10B1D0000D2243F003034FF0040800F10807037148
:10B1E000427180F807800C21384605F0C9FB3946CA
:10B1F000082204F585700FF077FE424606F1100133
:10B2000004F198000FF070FED4F8D431002B00F058
:10B21000C08594F87621920700F1BB8594F8CF2180
:10B22000D70700F1B685D4F8E011D4F8D8218B42C5
:10B2300001F01183002A01F0FB82D4F8DC311A6896
:10B2400032601E60C4F8DC613368002B01F04C8072
:10B2500094F8002194F8F1300221023B61F30102DD
:10B26000032184F8F13084F8002184F8F2100822D8
:10B2700005F12A0104F581700FF036FE042205F174
:10B28000320104F194000FF02FFE94F87631B4F8F7
:10B29000C620A4F8C82043F0010384F876310020CA
:10B2A000CCE6B8F1020F2CD0B8F10B0F00F02E85D0
:10B2B000B8F1040F7FF48DAE6B7F0D2B7FF412AFCE
:10B2C000082205F1200104F585700FF00DFE04221F
:10B2D00005F1280104F198000FF006FE94F876318C
:10B2E000326843F00103012184F8763100201171A6
:10B2F000A4E6B8F1070F00F0B683B8F1020F7FF4AF
:10B300006CAE6B7F022B7FF4EDAE95F8202084F8B5
:10B310005321012300202B7190E66B7F092B7FF4D2
:10B32000E1AEB8F1140F00F0408590F8BC1190F830
:10B33000BD318B4201F09A81B0F85A30B0F8588094
:10B34000B0F85E90B0F85CA090F8BE2102930023A4
:10B3500002F00702022A00F0498595F81F80B8F133
:10B36000150F3FF46AAE18466049F8F7B9FF94F834
:10B37000BE3194F8E42003F007036FF34102042B7D
:10B3800084F8E4207FF459AE6FF00F0056E690F990
:10B390003930002BFFF6A6AE6B7F032B7FF4A2AEF5
:10B3A00090F8601090F8613095F820200B4303F07E
:10B3B000070313423FF441AE90F8F03090F8F120CB
:10B3C0009B1A03F00303022B3FF437AEF53003F072
:10B3D00089FF94F8F12094F8F4300221023A84F8BD
:10B3E000F21084F8F120326843F00103012184F85F
:10B3F000F4300020117121E690F93930002BFFF66E
:10B4000071AE6B7F032B7FF46DAE90F8CD2190F879
:10B41000CC319A423FF40FAE90F8CE2102F00303F4
:10B42000022B7FF408AE95F82130C2F382010B4065
:10B4300095F820109B0043F0030301EA521243EAFF
:10B44000421313F01C0F80F8CE3102D013F0E00F3E
:10B4500005D194F8CE3103F0030384F8CE3194F88B
:10B46000CF31002243F0010384F8CF31A4F8C82083
:10B47000E1E590F93930002BBFF634AE6B7F052B38
:10B480007FF430AE95F8202095F82130134313F067
:10B49000070340F0B18790F8CC1190F8CD218A4293
:10B4A0003FF4C9AD90F8CE2102F00302022A7FF4E6
:10B4B000C2AD90F8CF2180F8CD1190F86010A0F8BF
:10B4C000C83063F3000280F8CF21084661F306100C
:10B4D00012F0040284F86000C1F3020141F06581BA
:10B4E0003368012119711046A8E500BF484E0020BD
:10B4F0006B7F032B7FF4F6AD90F93930002BC0F24F
:10B50000D78590F8CD1190F8CC21914207D090F8D2
:10B51000CE3103F00303013B022B40F2DD8694F8A9
:10B52000F03094F8F1001B1A03F00303022B00F033
:10B53000858694F8940194F89531984200F0D88665
:10B540002A2316222946204607B0BDE8F04FFEF711
:10B5500033BC90F93930002BBFF6C4AD6B7F082B9C
:10B560007FF4C0ADB5F82560438EF31A190400F1DD
:10B57000E98790F8F03090F8F1209B1A03F003036C
:10B58000022B00F0D787052205F12001F5300FF0DE
:10B59000ABFC94F8F42094F8F130A4F8FA606FF35F
:10B5A000000284F8F4200221023B012284F8F21008
:10B5B00084F8F13000202A7140E590F93930002BF1
:10B5C000BFF690AD6B7F0C2B7FF48CAD438EB5F83E
:10B5D0002910CB1A180400F1B58794F8F03094F8CC
:10B5E000F1209B1A03F00303022B00F0A387BD4B4D
:10B5F0001A68002A01F0068095F8203084F8283176
:10B60000B5F8213040F2E24202FB03F3C4F82431E2
:10B6100095F8242095F8233043EA0223A4F81C313E
:10B6200095F8262095F8253043EA0223A4F81E3128
:10B6300094F81A3195F8272095F82800A4F8F4100A
:10B6400023F00F0343F0080384F81A3194F81931FA
:10B6500042EA0022A4F82021013BD4F8142184F806
:10B6600019317A60326817603268C4F814210023F7
:10B67000336094F8942194F89531934207D094F86C
:10B68000963103F00E03042B01D184F89521002399
:10B69000A4F8C8301846D1E490F93930002BFFF6F1
:10B6A00021AD6B7F182B7FF41DAD90F8942190F89D
:10B6B00095319A423FF4BFAC90F8963103F00F03F6
:10B6C000042B7FF4B8ACB5F820C01FFA8CF3052B1F
:10B6D00040F206866F8CB9B2B1F5486F00F2008671
:10B6E0008B4200F2FD85AE8CB3B2B3F5FA7F80F0E9
:10B6F000F785E88C1FFA80FEAEF10A0240F6764824
:10B7000092B2424500F2EC8501339BB201FB03F398
:10B71000B3EB8E0F80F0E48595F828209142C0F0BD
:10B72000DF8584F8A02194F89621A4F898C101231C
:10B7300063F303020023A4F89A71A4F89C61A4F8AF
:10B740009E01A4F8C83095F82A1095F8293043EAEC
:10B750000123A4F8A23195F82C1095F82B3043EA78
:10B760000123A4F8A43195F82E1095F82D3043EA62
:10B770000123A4F8A63195F8301095F82F3043EA4C
:10B780000123A4F8A83195F8321095F8313043EA36
:10B790000123A4F8AA3195F8341095F8333043EA20
:10B7A0000123A4F8AC3195F8353095F8361084F8BB
:10B7B000962143EA0123A4F8AE313CE46B7F182BB9
:10B7C0007FF490AC47480368002B00F0A4829C42B1
:10B7D00000F0A18220230F22B4E690F93930002B2B
:10B7E000FFF680AC6B7F092B7FF47CAC29462046AA
:10B7F00007B0BDE8F04FFEF7D7BB6B7F022B7FF49D
:10B8000071AC94F8F01094F8F1308B4204D094F8B5
:10B81000F230032B00F0DD8594F8CC1194F8CD3193
:10B820008B4200F01C8495F8202085F82120232AE3
:10B8300012D084F8CD1194F8CF1194F860306FF3E2
:10B84000000184F8CF110021A4F8C810C3F302014D
:10B8500061F3061384F8603094F8CF315B077FF50D
:10B86000EAAB1D232B712A7794F86030C3F30203EF
:10B870006B7794F86130C3F302030020AB77FFF7D6
:10B88000DDBB6E7F062E7FF42DAC90F84A31D807D1
:10B8900040F1DF8413F002037FF4CDAB94F848212C
:10B8A00084F84921A4F8C83095F8203084F84B3149
:10B8B00095F8221095F8212094F84A3142EA0122A5
:10B8C000A4F84C2195F8232095F8241043F00203A6
:10B8D00042EA0122A4F84E2184F84A310020FFF701
:10B8E000ADBB00BF204D002090F93930002BBFF6D2
:10B8F000F9AB6E7F012E7FF4F5ABD448F8F7D6FC98
:10B90000002800F0E08194F8762122F0050242F050
:10B91000050284F8762194F87A206FF3C30284F844
:10B920007A20027946710B21C171D4F8D41142F00A
:10B9300003020271002900F0178294F8762197071C
:10B9400000F1128294F8CF21D60700F10D82D4F8CD
:10B95000E021914200F01A87D4F8D821002A00F0A3
:10B960009887D4F8DC21116801601060C4F8DC010C
:10B970000268002A7FF45FABFFF7EEBB6B7F092BF9
:10B980007FF4B0AB2A6AB2496B6A1143D0F8382110
:10B990000A40C0F8382103F0FF03D0F83C2143F0FF
:10B9A00010031340C0F83C312E6A6D6AFCF728FA88
:10B9B00005F0FF0343F01003A54AC4F8443194F89E
:10B9C000E430324343F00103024084F8E43094F859
:10B9D000303184F8313102F0FF0226F0FF031A43C0
:10B9E00042F00762002342F40322C4F84021A4F885
:10B9F000C8301846FFF722BB6F7F012F7FF472AB70
:10BA000090F8E40010F0020640F01F848F48F8F729
:10BA10004DFC0146002800F0568194F8E43043F0D4
:10BA2000020384F8E4300B794F7143F003030B7188
:10BA300013232046CB71FEF725FA2F713046FFF70E
:10BA4000FDBA6A7F012A7FF44DAB0023A0F8C8300D
:10BA500018462A71FFF7F2BA90F93930002BFFF639
:10BA6000C1AEFFF73FBB6B7F022B7FF43BAB94F87B
:10BA7000941194F8950195F82030884202D00F2B4C
:10BA800000F0998394F8BC2194F8BD11914202D042
:10BA9000142B00F00B8494F8CC1194F8CD218A4239
:10BAA00002D0162B00F07184122B04BF01232B71DE
:10BAB000EDE594F8F03094F8F1209A423FF412AB9F
:10BAC00094F8F220032A7FF40DAB6F7F012F7FF4EF
:10BAD00009AB94F93920002AC0F2488594F8762100
:10BAE00084F8F130002122F0030284F87621A4F8D2
:10BAF000C81053077FF5A1AA33686FF382021A2199
:10BB000084F8762100201971FFF798BA90F939303E
:10BB1000002BBFF6D1ABFFF7E5BA90F93930002B17
:10BB2000FFF6E0AA94F8F02094F8F1309A423FF43E
:10BB3000D9AA94F8F230032B7FF4D4AA6B7F012B9F
:10BB40007FF4D0AA94F800216FF3010284F8002159
:10BB500000202B71FFF772BA6B7F012B7FF4C2AA12
:10BB600090F93930002BC0F2C9803848F8F79EFBB5
:10BB7000002800F0A88094F8761194F87A2041F01B
:10BB8000010122F0180284F87611012184F87A204C
:10BB900002794171C7E694F8BC2194F8BD31934213
:10BBA0003FF449AA0023092184F8BD21A4F8C83034
:10BBB0006977B4F85A20B4F858002A841521B4F8EB
:10BBC0005C20E977B4F85E106984A884EA8418469A
:10BBD000FFF734BA94F8943194F8951199423FF4F0
:10BBE0002AAA94F9390095F821100028C0F22A8673
:10BBF0001A2900F0E28694F8961101F00F0004284B
:10BC000006D1144884F8953100230360A4F8C830A5
:10BC1000CF067FF510AA1923D6072B7100F1FE84F9
:10BC200095F821302B77628DB4F8C230A18D29842C
:10BC30007D2002FB03F300FB03F3EA834FF47A70E9
:10BC4000B3FBF0F300206B84FFF7F8B9484E0020F7
:10BC5000D0307808204D002094F8F01094F8F1309E
:10BC60008B423FF4E8A994F8F230032B7FF4E3A968
:10BC700094F8762184F8F110002322F0030284F86E
:10BC80007621A4F8C83095F8212085F820200D21D0
:10BC9000E9771846FFF7D2B994F8CC1194F8CD3172
:10BCA0008B423FF4C8A995F82120232A7FF4C1AD27
:10BCB000D2E50260C4E97500C4F8DC01002A7FF413
:10BCC000BAA9FFF749BA6FF06800FFF7B7B9136870
:10BCD000C4F8E031D4F8D831002B7FF432AA1368CD
:10BCE000036010600268C4E97600002A7FF4A3A90B
:10BCF000FFF732BA6B7F012B7FF4F4A994F87A3006
:10BD00006FF3041384F87A30FFF795B96B7F012B3A
:10BD10007FF4E8A929E794F9396094F8942194F81C
:10BD20009511002EC0F20C818A420AD094F8962117
:10BD300012F00B0F00F0CD8202F00F02062A00F085
:10BD4000C88294F8F02094F8F160921B02F003028C
:10BD5000022A00F06A8494F8CC6194F8CD219642CE
:10BD600000F08A842A2336E5D4F8D821002A7FF40B
:10BD7000F8AD0160C4E97500C4F8DC01F8E5137999
:10BD800003F00303032B00F08982C4F8D821FFF7E6
:10BD9000DAB9D4F8D821002A7FF44FAA3360C4E975
:10BDA0007566C4F8DC61FFF74FBA90F8E430990784
:10BDB0003FF541A9BC48F8F779FA0346002882D03C
:10BDC00094F8E42094F8BC11B4F85A00B4F8588000
:10BDD000B4F85E90B4F85CA0029042F0020284F8DD
:10BDE000E42094F8BD21914240F0DF852A8C1A2A84
:10BDF00040F2C582B4F8D2C0944528BF9446AA8CBC
:10BE000002981B2A94F8E42034BF86464FF01B0E9C
:10BE1000D20740F1B082D4F8382112F4006F02F456
:10BE2000006000F09983B4F8D420B2F5296F28BFE0
:10BE30004FF42962B2F5A47F4FF4296038BF4FF464
:10BE4000A4720190B5F822B0E88CBBF5A47FC0F0D5
:10BE50009A82934528BF934694F86020CDF80CB0A1
:10BE600002F0070B520700F174830BF12802D20095
:10BE70004FEA6B0B22FA0BFB039A5A4538BF5A461E
:10BE800092B2B0F5A47F8346C0F07B820198B0F5F2
:10BE9000A47F38BF4FF4A470834528BF834694F82D
:10BEA0006100CDF804B000F0070B400700F14E83AD
:10BEB0000BF12800C0004FEA6B0B20FA0BFB019836
:10BEC000584538BF584680B2DDF808B0DE4500F06E
:10BED0000B83013984F8BD11A4F8C0E1A4F8C2C1F4
:10BEE000A4F8C401A4F8C621002B00F0B38394F891
:10BEF000BE11052565F3020184F8BE11D4F81411B2
:10BF0000796031680F603168C4F814110021316024
:10BF1000002B3FF492A8DA811A79588142F003028B
:10BF200020461A7109241522A3F808E0A3F80CC0D2
:10BF300019465C71DA71FDF7A5FF0020FFF77EB8A6
:10BF40008A4205D094F8962112F00B0F7FF473A863
:10BF5000B5F820A01FFA8AF2052A7DD9B5F82290FB
:10BF60001FFA89F6B6F5486F76D8B24274D8B5F89C
:10BF700024801FFA88FCBCF5FA7F6DD2B5F826E064
:10BF80001FFA8EF2A2F10A0740F6764BBFB25F4568
:10BF900062D80CF10107BFB206FB07F7B7EB820FBF
:10BFA0005AD295F828B05E4556D3A4F898A1A4F8C3
:10BFB0009A91A4F89C81A4F89EE184F8A0B195F828
:10BFC0002AE095F8297047EA0E27A4F8A27195F89F
:10BFD0002CE095F82B7047EA0E27A4F8A47195F889
:10BFE0002EE095F82D7047EA0E27A4F8A67195F873
:10BFF00030E095F82F7047EA0E27A4F8A87195F85D
:10C0000032E095F8317047EA0E27A4F8AA7195F846
:10C0100034E095F8337047EA0E27A4F8AC7195F830
:10C02000357095F836E047EA0E27A4F8AE71678DB3
:10C03000BE4200F04E8494F89621032565F3030276
:10C0400084F89621013984F89511002B7EF4F5AF20
:10C0500004601846FEF7F2BF1E23FFF7BCBB94F83E
:10C06000941194F895318B423FF495AD95F82030BA
:10C0700085F8213094F939000028C0F2B9831A2BD1
:10C0800000F09B8494F8963103F00F00042806D149
:10C09000064884F8951100210160A4F8C810D9065B
:10C0A0007EF5C9AFB7E500BF484E0020204D002007
:10C0B00090F8E47017F002077EF4BDAFCC48F8F7B3
:10C0C000F5F8024600283FF4FEAD94F8CE1194F83E
:10C0D000E43094F8CDE1022060F3010143F0020363
:10C0E00084F8CE1194F8CC1184F8E43094F8D0316F
:10C0F0007145C3F3020603F0070CC3F3C20014D169
:10C10000013994F8CF3184F8CD1194F8CE1167F34A
:10C1100082036CF3840160F3471184F8CF31B4F8E3
:10C12000C63084F8CE11A4F8C83094F8CE1195F832
:10C13000213095F82070C1F3820C03EA0C0307EA62
:10C1400051179B0001F0030143EA47130B4384F8A6
:10C15000CE310323537111795072D4F8D401167281
:10C16000172341F00301D371D4F8D831117100289D
:10C1700000F0A68094F876118E0700F1A18094F863
:10C18000CF11C90700F19C80D4F8E011884200F07B
:10C190000584002B00F0D283D4F8DC3119681160DB
:10C1A0001A60C4F8DC211368002B7EF444AFC4F895
:10C1B000E421FEF740BF94F8963143F0200384F861
:10C1C000963194F93930002BC0F20C8294F8182182
:10C1D00094F819319A4206D0864841F60941F6F79B
:10C1E00069FB94F8193194F89621062161F3030252
:10C1F000013B012184F8193184F82811356884F84D
:10C200009621C2F3001394F81A21DB0022F00F02EA
:10C210000B43134384F81A31B4F89C31B4F89A21D3
:10C22000A4F81E310020B4F89E31A4F81C21A4F813
:10C230002031C4F824012971FEF700BF94F8F230D0
:10C24000032B7FF47DA9FFF774B92F710020FEF74F
:10C25000F5BE6748F8F72AF8014600283FF433ADE9
:10C2600094F84A3143F0010384F84A310379467166
:10C270000C22C271027243F003036FF00E020371CD
:10C2800042724FF0FF330522C3720373827220465D
:10C29000FDF7F8FD01232B71FFF706BBD379032BC4
:10C2A0003FF41DAD0A2B7FF470AD18E594F8BE3154
:10C2B00084F8BD2143F0080384F8BE31FFF7E7B9E5
:10C2C000002B7FF469AF1060C4E97522C4F8DC214B
:10C2D00069E72323FFF77FBA23231622FFF732B93A
:10C2E0001E231022FFF72EB9C4F8E461FEF7B0BF99
:10C2F00094F8CE31914243F0030384F8CE3111D14A
:10C30000B4F8CE2194F8D0014B1E22F49F6284F839
:10C31000CD3140F2FC4322F0040203EA80031343D0
:10C32000A4F8CE3194F8CE3195F82010C3F38200F2
:10C3300001EA531103F0030295F8213003409B00FA
:10C3400043EA4113134313F01C0F84F8CE3102D09B
:10C3500013F0E00F05D194F8CE3103F0030384F815
:10C36000CE3194F8CF310122134384F8CF3100202D
:10C370002A71FEF763BE4FF4A472019262E5C446CF
:10C380003DE54846A0E552467BE594F8602094F8E8
:10C39000CF3184F8CD1123F00903114643F008038F
:10C3A00062F3061184F8601013F0040F84F8CF31A3
:10C3B000C2F30202336800F028811D2119710023A5
:10C3C0002B776A7794F86130C3F30203AB77FFF7FA
:10C3D0005EB994F8762184F8F110002322F003026C
:10C3E00084F87621A4F8C8301846FEF727BE00BFAF
:10C3F000484E0020BCD4010001210DF117008DF83A
:10C400001720F8F729F9012800F2038195F8213067
:10C410008DF817300DF117000121F8F71DF90128EB
:10C4200000F2F7806A8C638ED31A1B0400F13A8203
:10C4300094F8F11094F8F0305B1A03F00303022B28
:10C4400000F0428294F8CC0194F8CD31834218D0A8
:10C4500094F8CE3103F00303022B12D194F8CF31BC
:10C4600084F8CD016FF3000394F8F40084F8CF3121
:10C47000C3F3800363F34100002384F8F400A4F8BD
:10C48000C83095F8213095F82000A4F8F6209B00DC
:10C4900094F8F42003F01C0343EA401302F0020274
:10C4A000134384F8F430D4F814317B6033681F6090
:10C4B0003268C4F814210023336094F8F420062075
:10C4C000023984F8F20012F01C0084F8F1103EF4F6
:10C4D000B5AD94F86010C2F3820262F3061184F8DD
:10C4E00060101846FEF7AABD0027C44584F8BD11A8
:10C4F000A4F8C87000F07181A4F85E00002B00F071
:10C50000BD81013984F8BD1194F8BE11A4F8C0E1D1
:10C51000032666F30201A4F8C2C1A4F8C401A4F87A
:10C52000C62184F8BE11A5F820E0A5F824C06884CF
:10C53000EA84EDE401232B712A2384F8533100208F
:10C54000FEF77CBD01232B712823F6E74FF4296BFE
:10C55000B5E44FF4296B8FE402F4807202434FF488
:10C56000A47200F08680A82001906BE4D348F7F70E
:10C570009DFE034600283FF4A6AB94F87A2042F0D3
:10C58000100284F87A20062102794771C171D4F82B
:10C59000D41142F00302027194F87621002900F0D0
:10C5A0001181950700F10E8194F8CF01C00700F1C9
:10C5B0000981D4F8E0018142D4F8D80100F0AA81C1
:10C5C000002800F0B381D4F8DC11086818600B6013
:10C5D000C4F8DC31196800297FF48BAAC4F8E4316F
:10C5E000FFF787BAB64B84F895110021196094F8CB
:10C5F000963113F0100340F0038101222A7118468E
:10C60000FEF71CBD1C60FEF7F7BF01221A71FFF791
:10C610003EB8336801221A711E238EE7A94841F201
:10C62000F441F6F747F9FFF7FBBA94F8F220032A32
:10C630007FF498ABFFF78FBB94F8E530023284F8B3
:10C64000F120002B40F0148194F8F23084F8E530AA
:10C65000FEF7B6BD94F8BE11A4F858C0042565F3E2
:10C660000201A4F85C2084F8BE1147E40023FEF721
:10C6700076BE0192FFF7E6BBB5F820901FFA89F26B
:10C68000052A7FF6E9ACB5F822801FFA88FEBEF5D0
:10C69000486F3FF6E1AC72453FF6DEACAF8CBEB200
:10C6A000B6F5FA7FBFF4D8ACEA8CADF8042092B2AC
:10C6B000A2F10A0A40F6764B1FFA8AFADA453FF6EB
:10C6C000CBAC06F1010A1FFA8AFA0EFB0AFABAEBA2
:10C6D000820FBFF4C1AC95F828B0DE45FFF4BCACC6
:10C6E000A4F89C71BDF80470A4F89891A4F89A81FC
:10C6F000A4F89E7184F8A0B195F82A8095F8297065
:10C7000047EA0827A4F8A27195F82C8095F82B70B9
:10C7100047EA0827A4F8A47195F82E8095F82D70A3
:10C7200047EA0827A4F8A67195F8308095F82F708D
:10C7300047EA0827A4F8A87195F8328095F8317077
:10C7400047EA0827A4F8AA7195F8348095F8337061
:10C7500047EA0827A4F8AC7195F8357095F836804B
:10C7600047EA0827A4F8AE71678DBE4500F0EE8059
:10C770001CF0020F94F896213FF45FAC022666F39A
:10C78000030284F8962101222A715BE40A68C4F846
:10C79000E021D4F8D821002A7FF4E3A80A680260D7
:10C7A0000860C4E97600FFF7E3B832681D20107115
:10C7B0002B77697794F861201846C2F30203AB77B0
:10C7C000FEF73CBCD4F8D80100287FF4FCAE196019
:10C7D000C4E97533C4F8DC31FCE652457FF48CAE15
:10C7E00048457FF489AE316801250D71FFF790BB94
:10C7F000232B3FF447ACD4F8B831C4F8EC3041E413
:10C800001923D0072B713ED41A232B77628DB4F8ED
:10C81000C230A18DEA8302FB03F37D2202FB03F306
:10C8200029844FF47A72B3FBF2F36B84FEF72FBFC7
:10C830001A7902F00302032A00F0F580C4E9763386
:10C84000FEF7FBBC23293FF4D6A9D4F8B811C4F8ED
:10C85000EC10FFF7D0B91968C4F8E011002A7EF493
:10C86000ECAC1A6832601E60C4E97666FEF7ECBC78
:10C87000144841F6C111F6F71DF8E5E6A4F858C0D2
:10C88000A4F85C204FE60F4841F63641F6F712F85F
:10C89000BAE70A7902F00302032A08D0C4E9761144
:10C8A000FFF75FB8336801221A71282345E6CA7979
:10C8B000032A3FF473AF0A2AF0D16FE7484E0020F5
:10C8C000204D0020BCD40100336801221A712A23B4
:10C8D00033E6A78D67457FF4AEAB40F2E24707FB36
:10C8E00006F642F2107707FB0262013AB2FBF6F25B
:10C8F000B4F8C26092B296427FF49DABB4F8962130
:10C9000002F0E00242F00102A4F8962101222A710D
:10C91000FFF798BB0D68C4F8E05100287FF453AED0
:10C92000086818600B60C4E9763353E6087900F0B4
:10C930000300032821D0C4E9761144E6037903F00B
:10C940000303032B1FD0C4E9760025E4B4F82CE0E0
:10C95000B6457FF40DAF40F2E24607FB06F642F221
:10C96000107707FB0262013AB2FBF6F2B4F8C2603C
:10C9700092B296427FF4FCAEC0E7C8790328CFD0CC
:10C980000A28D8D1CCE7C379032B01D00A2BDAD1FE
:10C99000036813600260C4E9762204E40168C4F805
:10C9A000E011002BF4D0FFF7F7BB94F8BE2112F092
:10C9B000060F3FF41BAAFEF7CBBC94F8182194F89D
:10C9C00019319A4206D01C4841F2C341F5F772FF73
:10C9D00094F8193194F89621062161F30302013B82
:10C9E00084F8193184F89621C2F3001394F81A21BF
:10C9F0000121DB000B4322F00F02134384F82811BE
:10CA0000B4F89C21B4F89A1184F81A310020B4F8D3
:10CA10009E31C4F82401A4F81C11A4F81E21A4F826
:10CA20002031FEF708BBDA79032A3FF41AAF0A2A4D
:10CA30007FF404AF15E700BFBCD401002DE9F84333
:10CA4000044690F8F10094F8F03098420D461646EE
:10CA500000F088801B1A03F00303022B11D094F915
:10CA600039209446BCF1000F6ADB94F8503194F8F9
:10CA700051219B1ADBB2012B00F09F800020BDE802
:10CA8000F88394F8BD2194F8BC319A4206D094F80A
:10CA9000BE3103F00603042B00F02F8294F8F270ED
:10CAA0007B1E052B00F21B82DFE813F07C00B9012E
:10CAB0002A011902EF00E400037943F00303037134
:10CAC00094F8E430DA0740F1D185D4F838315B07C7
:10CAD00040F1CC851123C371032380F809800372D0
:10CAE00089F80570002384F80131D4F8D431002B83
:10CAF00000F0AF8594F87621970700F1AA8594F8A5
:10CB0000CF21D00700F1A585D4F8E0219342D4F8D5
:10CB1000D82100F0A587002A01F05780D4F8DC3135
:10CB20001A68C9F80020C3F80090D9F80030C4F89A
:10CB3000DC91002B00F0858694F8F03084F8F13019
:10CB400094F8E530002B90D0022B00F09F81062B4B
:10CB50007ED0012B00F08580CA4840F20551F5F7E0
:10CB6000A9FE82E794F93920002A9446C0F2BF81D9
:10CB700094F8767117F001087FF474AF94F8199166
:10CB800094F818E1CE4500F0C8820122831E84F893
:10CB9000F22084F8F13094F8BD2194F8BC319A4227
:10CBA0007FF475AF2A4631462046F4F729F800286D
:10CBB00040F09A816FF08B0061E7B348F7F776FB9E
:10CBC000002838D094F85131013B84F85131037971
:10CBD0000222427143F003030371C271D4F8D431CD
:10CBE00094F85221D4F8D8110272B3B194F8762196
:10CBF000950712D494F8CF21D2070ED4D4F8E021AF
:10CC0000934200F0078559B91A7902F00302032A0A
:10CC100000F02586C4F8D83104E0002900F0D18264
:10CC2000D4F8DC311A68026018600368C4F8DC01CB
:10CC3000002B00F06681B4F8C80000287FF41EAF16
:10CC4000B4F8C230012B40F2B882A4F8C83015E71E
:10CC5000E18D628E0A443244204691B2FDF724FBF6
:10CC600003E72A4631462046F3F7CAFF00287FF43F
:10CC7000FCAE9FE7618EE38D1944314489B22046B2
:10CC8000FDF712FB94F939C0ECE67F48F7F70EFB8D
:10CC9000002800F0298194F8F03084F8F13003790D
:10CCA00043F003030371012343711223C371D4E9D9
:10CCB0007532002B00F08E8294F876118F0700F108
:10CCC000898294F8CF11C90700F18482D4F8E01169
:10CCD0008B4200F0A585002A00F0C985D4F8DC312C
:10CCE0001A68026018600368C4F8DC01002B00F0C9
:10CCF0000684B4F8C63094F939C0A4F8C830B1E657
:10CD000094F8003113F0030840F0EE805E48F7F726
:10CD1000CDFA8146002800F0E78094F93930002BE5
:10CD200080F28C8194F80181B8F1000F7FF4C4AED9
:10CD300004F17B073B46424604F5817104F2811001
:10CD400006F040F93946102204F19C000EF0CCF8B0
:10CD5000082204F1940104F1B5000EF0C5F894F82E
:10CD6000933084F88B8043F0010384F8933094F877
:10CD7000B43084F88C8068F3000384F8B43094F8FD
:10CD80007A3084F88D8043F0080384F87A3099F87B
:10CD9000043084F88E8043F00303C4E92B8884F8C0
:10CDA0008F8084F8908084F8918084F8928089F84C
:10CDB0000430012389F80530052389F80730D4F8B9
:10CDC000D431002B00F0488294F87621910700F1CD
:10CDD000438294F8CF21D20700F13E82D4F8E011CB
:10CDE000D4F8D8218B4200F08881002A00F07185A8
:10CDF000D4F8DC311A68C9F80020C3F80090D9F8DB
:10CE00000030C4F8DC91002B00F0148494F8003159
:10CE100094F939C043F0030384F8003122E6E28D2F
:10CE2000638E134494F8F420334412F001029FB24D
:10CE30006AD1B4F8FA3094F939C0FB1A1F043FF5EF
:10CE400011AEBCF1000FC0F2528394F8F03084F8B8
:10CE5000F13004F13407052204F1F50138460EF0F3
:10CE600043F805213846F7F7F7FB94F839C001235A
:10CE700060F3050C84F839C084F8E8314FFA8CFC73
:10CE8000F0E500BFBCD40100484E0020628EE18D69
:10CE900094F8F4300A44324413F0010396B240F09F
:10CEA0008280B4F8FA20B61A36043FF5DEAD04F1FC
:10CEB0003405052284F8E53004F1F50128460EF02A
:10CEC00013F805212846F7F7C7FB94F839300122FB
:10CED00060F3050384F8393084F8E821C5E5C248D9
:10CEE00040F2D441F5F7E6FC94F939C0BAE594F87C
:10CEF000E51000297FF4B6AD3AE62046FDF7D6F8F6
:10CF0000CCE5C4F8E40196E6B848F7F7CFF98046D7
:10CF10000028E9D0A38D94F8F42006333B44A4F80C
:10CF2000FA3003796FF3000243F0030384F8F4202E
:10CF30000371082343710123C371052204F1F50134
:10CF400008300DF0D1FFB4F8FA30A8F80D30D4F85D
:10CF5000D431002B00F0D78294F87621910700F1AC
:10CF6000D28294F8CF21D20700F1CD82D4F8E0111B
:10CF7000D4F8D8218B4200F08384002A00F0C384C7
:10CF8000D4F8DC311A68C8F80020C3F80080D8F85B
:10CF90000030C4F8DC8194F939C0002B7FF462AD15
:10CFA000C4F8E4815EE59148F7F780F9054600286A
:10CFB0003FF45BADA28D94F8F410037906326FF361
:10CFC0000001324484F8F410A4F8FA2043F003037B
:10CFD0000821012203714171C27104F1F50105229A
:10CFE00008300DF081FFD4F8D431B4F8FA20A5F858
:10CFF0000D20002B00F0938294F87621920700F127
:10D000008E8294F8CF21D70700F18982D4F8E011FD
:10D01000D4F8D8218B4200F04484002A00F0168511
:10D02000D4F8DC311A682A601D602B68C4F8DC5122
:10D03000002B7FF41AADC4F8E45116E504F17B0728
:10D040003B46424604F5817104F2811005F0BAFFB7
:10D050003946102204F19C000DF046FF082204F12D
:10D06000940104F1B5000DF03FFF94F87A3084F894
:10D070008B8023F0180343F0180384F87A3094F877
:10D08000933084F88C8068F3000384F8933094F82C
:10D09000B43084F88D8043F0010384F8B430012368
:10D0A000C4E92B8884F88E8084F88F8084F890807F
:10D0B00084F8918084F8928099F8042089F80530EA
:10D0C000062389F80730D4F8D43142F0030289F8F6
:10D0D0000420002B00F0C08094F87621900700F126
:10D0E000BB8094F8CF21D10700F1B680D4F8E021BD
:10D0F0009342D4F8D8217FF478AE1968C4F8E011CF
:10D10000002A7FF475AE1A68C9F80020C3F80090B1
:10D11000D9F80030C4E9769975E694F8311194F89D
:10D1200030E1714564D0A1EB0E01C9077FF59AACDF
:10D1300094F8E43013F0010700F0FC81FBF792FA59
:10D140000746002800F09E8094F8303184F8313191
:10D15000037F228DC28043F00303037709234377C3
:10D16000C377032303714146082220300DF0C7FE28
:10D17000D4E95023110C87F82020C2F3072287F846
:10D1800021201A0C87F8243087F82210C3F30723D4
:10D19000090A87F82620120A87F8231087F8253015
:10D1A00087F8272039460868FBF72CFAFBF734FA92
:10D1B00094F8F03094F8F1004CE40133A4F8C8304E
:10D1C0005DE40360C4E97500C4F8DC01002B7FF462
:10D1D00032AD96E6002A7FF481AD0360C4E97500A4
:10D1E000C4F8DC0182E500BFBCD40100484E002039
:10D1F00094F8491194F848E1714549D0A1EB0E012A
:10D20000C8077FF52FAC94F84A31D90740F19E82C8
:10D21000980740F1E282FBF725FA014690B394F8B3
:10D22000483184F84931238DC38003230371037F80
:10D2300043F003030377062343770C23C37794F863
:10D240004B3180F82030B4F84C31A0F82130B4F8DC
:10D250004E31A0F82330A6E7D4F8D821002A7FF475
:10D26000C7ADC9F80030C4E97599C4F8DC91CAE5C6
:10D2700094F8BD1194F8BC31994200F0FF8120462A
:10D28000FCF714FF94F8F03094F8F100FFF7E2BBDC
:10D2900094F895E194F894118E45E9D0DFF8648311
:10D2A000D8F80010002900F09E828C427FF4DAAB9F
:10D2B00094F8961101F00F01082900F24F850FF242
:10D2C000080E5EF821F000BF2FD40000A9D30000A3
:10D2D0005BD3000055CA000055CA000055CA0000C3
:10D2E00055CA000055CA0000EDD20000E28D638EE1
:10D2F000D4F8B0E11344334494F896212EF8023C5C
:10D30000042363F3030284F89621D4E97532AEF165
:10D310001301002B00F0D382BF0700F1D08294F8F4
:10D32000CF01C00700F1CB82D4F8E001834200F0C6
:10D330009184002A00F07D84D4F8DC311A684EF81C
:10D34000132C1960C4F8DC115EF8133C002B7FF439
:10D3500089ABC4F8E411FFF785BBBB073FF582AB8F
:10D36000FBF780F9014600288CD094F896010B7FDA
:10D37000032243F0030362F30300182784F89601A5
:10D38000208D0A710B774F77B4F898310B84B4F87D
:10D390009A314B84B4F89C318B84B4F89E31CB84A1
:10D3A0000F23C880CB77FEE694F89731002B40F02E
:10D3B000BA82002AC0F2658394F89621C4F8243119
:10D3C000062161F3030294F8A01184F8962101204C
:10D3D000B4F89A2184F82801002900F0C283B2FB36
:10D3E000F1F313FB01F3B4F898119BB2994298BF83
:10D3F0001A46A4F81C2194F8963194F81A21B4F82E
:10D400009C11A4F81E11C3F30013DB0022F00F02DD
:10D4100043F00203134309F1FF39B4F89E21A4F845
:10D42000202184F81A3184F81991FFF71EBB764841
:10D43000F6F73CFF024600283FF424AF0379C8F812
:10D44000004043F003030371182343710F23C3719A
:10D45000B4F898310381B4F89A314381B4F89C311F
:10D460008381B4F89E31C38100230374C3740375B0
:10D470004FF0FF3343758375C37503764376837628
:10D48000C376037743778377B4F8C630A4F8C830FF
:10D4900094F89631C4F8B451072161F3030384F87A
:10D4A0009631A368002B0ADAE768606823F000432E
:10D4B00087422CBFE9192918CB1AC4F8B4311332AA
:10D4C000524BC4F8B0210122022110469C60F6F7AD
:10D4D000C5FF00283FF4D6AE4D4840F60A71F5F777
:10D4E000E9F994F8F03094F8F100FFF7B3BA94F842
:10D4F000E530002B3FF4A9AC84F8E520A9E4C4F89A
:10D50000E401FFF7F6BBD4F8D821002A7FF438AD48
:10D51000C8F80030C4E97588C4F8DC813BE5D4F86C
:10D52000D821002A7FF47CAD2B60C4E97555C4F87E
:10D53000DC517DE53448F6F7B9FE804600283FF41B
:10D54000A1AE94F83131013B84F8313109234371A4
:10D5500094F93930002B037943F0030303714FF042
:10D560000802ACBF08230E23C371394610440DF0E6
:10D57000C6FCD4E94E23110C88F80820C2F3072218
:10D5800088F809201A0C88F80C3088F80A10C3F3C0
:10D59000072388F80E20090A120A88F80B1088F869
:10D5A0000D3088F80F20D4F8D431002B46D094F8F1
:10D5B0007621920742D494F8CF21D7073ED4D4F8ED
:10D5C000E011D4F8D8218B4200F08D81002A00F0C0
:10D5D000CB82D4F8DC311A68C8F80020C3F8008088
:10D5E000D8F80030C4F8DC81002B00F02781B4F8B3
:10D5F000C62094F8F03094F8F100A4F8C820FFF7A2
:10D6000029BA00BF204D0020484E0020BC07002052
:10D61000BCD401001A68C4F8E02100297FF400ABF3
:10D620001A68026018600368C4E97600002B7FF472
:10D6300002AB66E4C4F8E491FFF7E8BBD4F8D82164
:10D64000002AC6D1C8F80030C4E97588C4F8DC8166
:10D65000CAE7D4F8D821002A7FF460AAC9F80030BC
:10D66000C4E97599C4F8DC91FFF763BA0D2389F812
:10D670000880022789F80730FFF732BA94F8CC11F6
:10D6800094F8CD318B423FF4EDA994F8CE3103F0FC
:10D690000307032F00F09881002F7FF4E2A9C84808
:10D6A000F6F704FE034600283FF4ECAD94F8CE21D3
:10D6B00094F8CF01012161F3010294F8D01184F8AC
:10D6C000CE21C2F3820767F3020194F86070C0F3C1
:10D6D000400060F3C307C2F3421060F3C50184F851
:10D6E000D011C2F38201032284F86070197258725B
:10D6F0005A711621D4F8D421D971197941F0030156
:10D700001971D4F8D811002A00F0518194F87601EB
:10D71000870700F14C8194F8CF01C00700F14781E1
:10D72000D4F8E001824200F0A382002900F08A824E
:10D73000D4F8DC21116819601360C4F8DC311A6870
:10D74000002A7FF454AFC4F8E43150E79C48F6F760
:10D75000ADFD00283FF496AD94F84931013B84F8C3
:10D76000493194F84A3143F0010384F84A3103798E
:10D7700043F003030371062343710C23C371037247
:10D780006FF00E034372052383724FF0FF33C372B1
:10D790000373D4F8D431002B57D094F87621920734
:10D7A00053D494F8CF21D7074FD4D4F8E021934233
:10D7B000D4F8D82100F0F481002A00F06B82D4F86C
:10D7C000DC311A6802601860C4F8DC010368002BC1
:10D7D0007FF40DAFC4F8E40109E77A4840F6B5617B
:10D7E000F5F768F84EE594F8963103F00F03082B2F
:10D7F00000F2B48201A151F823F000BF2FD4000041
:10D80000A9D300005BD3000065CA000065CA000010
:10D8100065CA000065CA000065CA0000EDD20000BC
:10D820001968C4F8E011002A7FF458AA1A68026047
:10D8300018600368C4E97600FFF758BAC4F8E481B9
:10D84000D5E6C4F8E491FFF777B9D4F8D821002AD7
:10D85000B5D10360C4E97500C4F8DC01B6E7DA7934
:10D86000032A3FF4DDAE0A2A7FF4D4A9D8E61A7958
:10D8700002F00302032A50D0C4E97633FFF72EBA30
:10D880001968C4F8E011002A7FF47AAB1A68C8F866
:10D890000020C3F80080D8F80030C4E97688FFF78C
:10D8A0007ABB1968C4F8E011002A7FF4B9AB1A6892
:10D8B0002A601D602B68C4E97655FFF7B9BB002AC2
:10D8C0007FF43AAD4EF8133CC4E97511C4F8DC118D
:10D8D0003AE51A7902F00302032A00F06D81C4E9E7
:10D8E0007633FFF785BA1968C4F8E011002A7FF48F
:10D8F00070AE1A68C8F80020C3F80080D8F800306D
:10D90000C4E9768870E61A7902F00302032A00F06F
:10D910002081C4E97633FFF733BBDA79032A85D057
:10D920000A2AA9D182E72648F6F7C0FC00283FF46E
:10D93000A9AC027942F0030202711122C2710322E2
:10D9400042710F22027294F897214272D4F8D421C6
:10D95000002A00F01A8194F87611890700F11581E8
:10D9600094F8CF11CB0700F11081D4F8E0118A426E
:10D97000D4F8D81100F0AE81002900F0A381D4F8CA
:10D98000DC21116801601060C4F8DC010268002A23
:10D9900000F0958194F8943184F895310023C8F80B
:10D9A000003094F8F10094F8F030FFF753B80029F4
:10D9B0007FF4BEAE1A60C4E97533C4F8DC31BEE64C
:10D9C000484E0020BCD4010084F8CD111907C3F3E0
:10D9D000820240F10B81022262F3840384F8CE318B
:10D9E00094F8CE3159064FEA531240F1C580022215
:10D9F00062F3471384F8CE31831E94F8CE2194F855
:10DA0000607094F8610084F8F13094F8CF31C2F37B
:10DA1000820107F0070700F00700C3F380038F427D
:10DA200008BF00215B00B0EB521F43F001034FEA37
:10DA3000521208BF002243EA421343EA810306223E
:10DA400084F8F43084F8F220FFF728B81A7902F04D
:10DA50000302032A00F0C280C4E97633FFF7E0BA7C
:10DA60001968C4F8E011002A7FF458A81A68C9F8A8
:10DA70000020C3F80090D9F80030C4E97699FFF788
:10DA800058B8B548F6F712FC00283FF4FBAB027912
:10DA900042F003020271182242711022C271B4F8DE
:10DAA00098210281B4F89A214281B4F89C218281A4
:10DAB000B4F89E21C28194F8A0210274B4F8A22186
:10DAC000A0F81120B4F8A421A0F81320B4F8A621DE
:10DAD000A0F81520B4F8A821A0F81720B4F8AA21BE
:10DAE000A0F81920B4F8AC21A0F81B20B4F8AE219E
:10DAF000A0F81D20D4F8D421002A00F0828094F8E8
:10DB000076118F077DD494F8CF11C90779D4D4F852
:10DB1000E0118A42D4F8D81100F00281002900F007
:10DB2000F780D4F8DC21116801601060C4F8DC01D2
:10DB30000268002A00F0E98094F8962194F8F10038
:10DB4000052363F3030284F8962194F8F030FEF77E
:10DB500081BFDA79032A3FF499AE0A2A7FF4D9AE5D
:10DB600094E6A4F81C2146E41A7902F00302032A81
:10DB700058D0C4E976332CE5D70740F1B7800122AD
:10DB800062F3471384F8CE3136E7D4F8D811002970
:10DB90007FF4F5AE0260C4E97500C4F8DC01F5E677
:10DBA0001968C4F8E011002A7FF409AE1A6802600F
:10DBB0001860C4E9760009E6DA79032A3FF4A3AADB
:10DBC0000A2A7FF48CAEFFF79EBA1A7902F003029C
:10DBD000032A20D0C4E97633FEF7A0BFDA79032AFE
:10DBE0003FF465AE0A2A7FF437AF60E6D70794F8B2
:10DBF000CE3140F1A180012262F3840384F8CE315A
:10DC0000EEE6D4F8D81100298BD10260C4E9750082
:10DC1000C4F8DC018CE7DA79032A3FF427AF0A2A3B
:10DC2000D8D123E7DA79032A3FF463AE0A2AA0D1D8
:10DC30005FE61A7902F00302032A25D0C4E976339D
:10DC4000FFF77ABB117901F0030103292AD0C4E957
:10DC500076226DE51868C4F8E001002A7FF46CAB09
:10DC60001A684EF8132C1960C4E97611FFF76CBBE3
:10DC70001068C4F8E00100297FF45AAD11681960FA
:10DC80001360C4E976335AE5DA79032AE8D00A2A20
:10DC9000D4D1E5E71A7902F00302032A08D0C4E9D7
:10DCA00076338CE5D1790329E8D00A29CFD1E5E78D
:10DCB000DA79032A3FF47AAF0A2AF0D176E7C4F87A
:10DCC000E40167E6117901F00301032917D0C4E9E3
:10DCD000762254E61368C4F8E03100297FF44FAE91
:10DCE000116801601060C4E976004FE612F004028A
:10DCF00018BF042262F3471384F8CE317CE6D17951
:10DD00000329EDD00A29E2D1EAE7C4F8E40113E7D8
:10DD1000117901F00301032917D0C4E9762200E745
:10DD20001368C4F8E03100297FF4FBAE116801608C
:10DD30001060C4E97600FBE612F0040218BF04226A
:10DD400062F3840384F8CE314AE6D1790329EDD019
:10DD50000A29E2D1EAE700BF484E0020054840F614
:10DD6000F571F4F7A7FD94F8F03094F8F100FEF7A0
:10DD700071BE00BFBCD401002DE9F8433C4C3D4FBF
:10DD80006279054604F108062EE042464FF4F87128
:10DD90003846F6F7BDFA028D9045034631D1D9F8E1
:10DDA00004100A79487902F00302022A34D00028CC
:10DDB00033D1D3F8E02100200860002A43D0D3F803
:10DDC000E42102B11160C3F8E41162792379A178EA
:10DDD0009A4205D00133DBB2994208BF0023237178
:10DDE000013D15F0FF0537D023792178934233D0D8
:10DDF00013FB01F306EB030936F80380B8F10F0FAC
:10DE0000C3D9D9F804100B796FF301034FF6FF70F3
:10DE10000B71FAF73DFCD8E700B393F8D00110F08E
:10DE2000400FC6D06FF38610012A83F8D001C0D10D
:10DE30000A79022060F301020A71D3F8E021002080
:10DE40000860002ABBD1D3F8D421C3F8E011002A1E
:10DE5000B5D1C3F8D411B6E7BDE8F88393F8D02163
:10DE600042F04002404683F8D021FAF711FCACE7BB
:10DE700024070020E00C00202DE9F043D0F81441E5
:10DE800083B0064644B101252068214644680D71DF
:10DE9000FAF7B8FB002CF7D1D6F8D41131B3DFF87C
:10DEA0008080DFF8809006F1680707E029463A464F
:10DEB0002046F6F75FFAD6F8D411B9B13046FBF731
:10DEC00005FF05464046F6F7F1F904460028EDD176
:10DED00040F672114846F4F7EDFC29463A462046D2
:10DEE000F6F748FAD6F8D4110029E7D1328D0E4B57
:10DEF00000960532D2B201210020F7F7B5FD30F0CF
:10DF0000020304D0074840F63711F4F7D3FC4FF66C
:10DF1000FF73FF20338503B0BDE8F043FFF72CBF4C
:10DF20004C590020BCD40100C19B0000F0B5C4696D
:10DF3000228D4FF6FF739A428BB000F0848090F8E8
:10DF40002730012B054600F00281022B7DD0002BEB
:10DF500000F0E38094F85331002B79D1278ECDE97E
:10DF60000833AB8C7E1CB6B2002B00F0A38094F972
:10DF70003930002BC0F21D8195F826300022DB07D6
:10DF8000A4F8C02040F1E9800025A4F8C450B4F8FA
:10DF9000C8302BB1B34240F248819B1BA4F8C83073
:10DFA000B4F8D0302BB1B34240F20F819B1BA4F8E0
:10DFB000D030B4F8CC2094F8F03094F8F1105AB185
:10DFC000B24200F2DA80B4F8C8200020A4F8CC00F5
:10DFD00012B9994200F037815B1A03F00303022B58
:10DFE00000F0D48094F8182194F819319A4200F086
:10DFF000008100222286DDE9086315B9BA4200F0EB
:10E00000D280013291B213B9002E00F0AF80228D80
:10E01000E46904950020A24D03910532CDE9010089
:10E0200006940096D2B201210595F7F705FD30F070
:10E03000020308D0FAF786FB844204D099484FF4D3
:10E04000D861F4F737FC0BB0F0BD3D2384F85331B1
:10E0500094F9391000291ADB94F8501194F8510101
:10E06000091AC9B2032912D094F8E41011F004007F
:10E070000DD13D2B0BD0278EAB8C7E1CCDE908003B
:10E08000B6B2BBB141F0040184F8E41074E78649EC
:10E09000A4F85A21086884F87031844204BF002033
:10E0A00008601821204684F858110BB0BDE8F040F4
:10E0B000FFF7E2BE95F8263013F001037FF464AF5A
:10E0C000B4F8C010002948D0B14240F2C380891B87
:10E0D000B4F8C450A4F8C010002D3FF458AFAE42BD
:10E0E00080F08F80AD1BABB2062B4FF00005A4F87B
:10E0F000C43025867BD994F93930AB42BFF647AF9F
:10E10000002F74D1D4F8E8506B0815F0010518BF42
:10E1100043F00043C4F8E83039E794F87A30180740
:10E120003BD5A08DB4F8CE10831D9942C4BF8B1F80
:10E130001B1AB4F8CA00CCBF9BB20B4698425AD007
:10E14000A4F8CA30A4F8CC30A4F8D01002E7002319
:10E15000A4F8D030A4F8CC30FCE6B4F8C450002DBC
:10E16000BDD1B4F8C250A4F8C450B5E700297FF47B
:10E170004EAF002D7FF44BAF65E75B1A03F003034E
:10E18000921B022BA4F8CC207FF42CAF94F8F23031
:10E19000013B012B3FF626AF2BE794F87631D907E8
:10E1A0007FF5D8AEBDE713B9002E3FF44CAF29463A
:10E1B0002DE708AA09A92846F2F712F9D4F8D431B4
:10E1C000002B58D000232386D6E6FAF74BFA0146F7
:10E1D000002834D0238D0022A4F8D020C3801B2334
:10E1E00003710068FAF70EFAFAF716FAE1E601256C
:10E1F000CDE6228EFFE6B4F8D00000287FF4AAAE68
:10E20000A0E7294B218D1A68944204BF00221A60AE
:10E2100018220823A4F85A1184F8582184F8703180
:10E220002046FFF729FE0BB0F0BD1F4B218D1A6869
:10E23000944204BF00221A6018222223EAE7012335
:10E24000A4F8D030B5E605228B1E84F8F22084F8BD
:10E25000F130C7E61449A4F85A210868844208BF7F
:10E260000B6018213E2384F8581184F87031204641
:10E27000FFF702FEE7E6FF20FFF77EFDD4F8D4218A
:10E28000002A9FD1D4E91901F6F77EF8002899D128
:10E2900094F83C305A077FF56FAEA38D23866BE66A
:10E2A000A19C0000BCD40100204D0020D0F8D43146
:10E2B000002B00F0DE8001392DE9F047DFF8B48152
:10E2C000DFF8B4910446CDB24FF0010A11E04046A8
:10E2D000F5F7ECFF0746002866D004F168023146E6
:10E2E0003846F6F747F8D4F8D431013DEDB2002BAB
:10E2F0007AD094F8CF21D10703D494F876219207ED
:10E3000058D5D4F8D82193426ED1FF2D6CD0D4F8D3
:10E31000D4112046FBF7DAFC037903F00303032B47
:10E320000646D4D1C379033B142BD0D801A252F8AE
:10E3300023F000BF91E3000091E30000CFE2000072
:10E34000CFE20000CFE20000CFE20000CFE2000009
:10E3500091E3000089E30000CFE20000CFE200007B
:10E36000CFE20000CFE20000CFE20000CFE20000E9
:10E37000CFE20000CFE20000CFE20000CFE20000D9
:10E38000EDE30000EDE3000094F93930002B9EDA54
:10E3900094F8763143F0020384F876314046F5F77D
:10E3A00085FF0746002898D140F225714846F4F7CA
:10E3B00081FA92E71A7902F00302032AA5D1DA79E9
:10E3C000032A01D00A2AA0D194F8F11094F8F02081
:10E3D0008A4212D094F8F220032A96D01A681AB111
:10E3E000D4F8D8118A4233D0BDE8F08794F8CF3101
:10E3F00043F0010384F8CF3169E794F8310194F8D0
:10E4000030118842EAD194F8490194F848118842C1
:10E41000E4D194F8950194F894118842DED194F8EF
:10E42000BD0194F8BC118842D8D194F8CD0194F87C
:10E43000CC118842D2D194F800316AF30103023A38
:10E4400084F80031032384F8F12084F8F2305CE78B
:10E45000C4F8D421D4F8DC21D4F8E401116819609F
:10E460001360C4F8E03100287FF44FAFC4F8E43102
:10E470004BE770474C590020BCD4010010B504464E
:10E480000120FFF779FC20460121BDE81040FFF78D
:10E490000DBF00BF0149F5F723BF00BF4C59002055
:10E4A000014B5879704700BFDC04002010B50C4BBD
:10E4B00093F804C093F805E01C78F4450DD01CFBDC
:10E4C00004FC083303EB0C0480F800E033F80C0084
:10E4D000636808801360186810BD002010BD00BF7D
:10E4E000DC04002000B50B4B93F804C093F800E067
:10E4F00084450DD008331CFB0EFC03EB0C0E33F8E7
:10E500000C00DEF804300880136018685DF804FB26
:10E510000020FBE7DC040020094B19795A791878B0
:10E5200093F802C08A4209D04A1CD2B201FB0031E2
:10E53000944508BF002288681A7170470020704710
:10E54000DC04002038B5114A92F805C0947892F89E
:10E5500004E015780CF10103DBB29C4208BF0023F4
:10E560009E450AD01CFB05FC02F1080E2EF80C009B
:10E57000F444CCF80410537138BD054840F275716D
:10E58000F4F798F900231B80FFDE00BFDC040020B5
:10E59000BCD40100F0B5537983B0144605460E464D
:10E5A0003BB3237903F00302032A0DD04FF6FF7229
:10E5B000954204BF6FF3010323712146284603B03F
:10E5C000BDE8F040FAF764B84FF6FF739D4216D1EC
:10E5D000306884423DD00028EFD0C74840F29F7198
:10E5E000F4F768F92146284603B0BDE8F040FAF791
:10E5F0004FB8C14840F28271F4F75CF9D1E7BF48E7
:10E600002A464FF4F871F5F783FEE379023B07469B
:10E61000162B2ED8DFE813F0D800C5003A003300DF
:10E62000A20026002D00260091004B002D00410085
:10E630002D002D002D0023002D0026004001130188
:10E640000101E400B400AC4840F29171F4F732F9F2
:10E650000020AB4903B0BDE8F040F5F741BE237A96
:10E66000032B1AD097F8E4306FF3410387F8E430B6
:10E67000AEE73068A042ECD00028AED19DE797F815
:10E68000003143F0030387F80031A1E797F87631B2
:10E6900043F0020387F876319AE797F8763123F052
:10E6A000030387F876310023A7F8C83090E790F984
:10E6B0003930002BEADB2379172243F0030323715F
:10E6C00062710323082200F27911E371A0180CF0A3
:10E6D0000BFC97F87731237497F8783163740C2129
:10E6E00004F1120002F04CF9D7F8D431002B00F0FD
:10E6F000E38097F87621910700F1DE8097F8CF212B
:10E70000D20700F1D980D7F8E011D7F8D8218B4291
:10E7100000F0FA80002A00F00481D7F8DC311A6892
:10E7200022601C602368C7F8DC413268002B00F0CF
:10E73000C080002A87D003B0F0BD90F8763123F076
:10E74000060343F0060387F87631B7F8C630A7F81A
:10E75000C83097F8743187F8753139E790F9393056
:10E76000002B8CDA90F8763123F0030380F87631B1
:10E770000023A0F8C83090F8F03080F8F13027E797
:10E7800090F8F43090F86020C3F3820363F306122C
:10E7900087F8602097F8CF316FF3000387F8CF3107
:10E7A00016E7082204F1120100F581700CF09CFBC1
:10E7B000042204F11A0107F194000CF095FB97F87C
:10E7C000763143F00203BEE7237A132B08BF1623EA
:10E7D00080F8533190F85131013B80F85131F7E620
:10E7E00090F93930002BD5DA90F8E420454B6FF3DF
:10E7F000410280F8E42093E8030002AB03E9030040
:10E8000097F8CE3197F8602042EA930303F00703AC
:10E8100002A90B4413F8083CB8E790F8CE31022265
:10E8200062F3010380F8CE3190F93930002BB1DA70
:10E83000344B93E8030002AB03E90300E0E790F8F0
:10E84000E43090F8BC116FF3410380F8E43090F8A5
:10E85000BD318B423FF4BCAE90F8BE2102F00703FD
:10E86000032B05D0033303F00703012B3FF601AF61
:10E87000B7F8C231A7F85830B7F8C631A7F85C30FE
:10E8800002F00703052B22D0B7F8C8312BBB87F85D
:10E89000BD11A7F8C8309BE690F8BE3103F007021F
:10E8A000012A7FF495AE022262F3020380F8BE31A2
:10E8B0008EE6C7F8E4413CE7D7F8D821002A7FF478
:10E8C0002CAF2360C7E97544C7F8DC412DE704236A
:10E8D00063F3020287F8BE217AE6A7F8C23100236B
:10E8E00063F30202A7F8C831B7F8CA3187F8BE212E
:10E8F000A7F8C6316CE600BFBCD40100E00C0020D4
:10E90000484E0020FCD401001968C7F8E011002A25
:10E910007FF403AF1A6822601C602368C7E976445D
:10E9200003E71A7902F00302032A02D0C7E976331B
:10E93000F3E6DA79032AEDD00A2AF7D1EAE700BF35
:10E9400090F8F13090F8F020934203BF013380F843
:10E95000F03000200C20704790F84410B0F84030A0
:10E96000C1F30212022A0FD0042A11D0DB080A3B9D
:10E970009BB290F85E20808FD20644BF043B9BB2CE
:10E98000984228BF184670479B080B3B9BB2F0E7A4
:10E9900009074BBFA3F51473A3F5D7739B111B1184
:10E9A000023B9BB2E5E700BF704700BF10B50C46C5
:10E9B00030B994F8E4306FF3820384F8E43010BD8A
:10E9C000054840F2AF21F3F775FF94F8E4306FF398
:10E9D000820384F8E43010BD08D5010000B9704707
:10E9E000024840F2A721F3F765BF00BF08D5010038
:10E9F000012800D0704710B50C46F9F7A3FE8442F9
:10EA000006D0BDE81040034840F29F21F3F752BF03
:10EA100010BD00BF08D501002DE9F041079C9DF80D
:10EA20001880218D1D464FF6FF73994226D0064669
:10EA3000174601462A462046FEF700F8F0B923782B
:10EA40000133DBB223700BB31349144B0D8104F176
:10EA50001C000022C860C1E9006781F80A80996043
:10EA600001201146F5F7FAFC50B9FF20FFF784F9B1
:10EA70002046FF21BDE8F041FFF718BCBDE8F0815A
:10EA8000074840F22A21F3F715FFEEE7044840F269
:10EA90001D21F3F70FFFD7E7AC5B0020CC07002068
:10EAA00008D50100038E23B190F8E42012F004038E
:10EAB00000D0704710B542F0040288B00E4C80F8C8
:10EAC000E42005310122CDE90232CDE90434CDE95B
:10EAD00000330690CAB218460321F6F7ADFF30F0B6
:10EAE000020307D0054840F2E31108B0BDE810402A
:10EAF000F3F7E0BE08B010BDADE9000008D5010095
:10EB000070B50E461546FBF7CDFD002840D00446F3
:10EB10005EB990F8F02090F8F1309A4203D090F866
:10EB2000F230032B26D00C2070BD90F8760110F047
:10EB3000040012D194F8F02094F8F1309A42F2D007
:10EB400094F8F230032BEED194F8003184F801618F
:10EB500060F3010384F8003170BD94F8502194F8FB
:10EB600051319342DFD1013384F8526184F850313E
:10EB7000002070BD1022294600F281100CF0B4F97B
:10EB8000B4F8003103F0FC03A4F80031304670BD46
:10EB9000022070BD704700BF00B97047024840F2C4
:10EBA000B141F3F787BE00BF50D501002DE9F04118
:10EBB000079C9DF81880218D1D464FF6FF739942E2
:10EBC0002DD00646174601462A462046FDF736FF59
:10EBD00028BB23780133DBB2237043B30220FFF755
:10EBE000CBF802212046FFF761FB1449144B0D813D
:10EBF00004F11C000022C860C1E9006781F80A80A6
:10EC0000996001201146F5F729FC50B9FF20FFF764
:10EC1000B3F82046FF21BDE8F041FFF747BBBDE850
:10EC2000F081084840F25141F3F744FEEEE7054811
:10EC300040F23E41F3F73EFED0E700BFC45B002048
:10EC4000DC07002050D501002DE9F041064682B0D6
:10EC50000020FAF7A5FE60B3036A04464BB393F8AD
:10EC6000202042F0020283F82020076A0FB30146F9
:10EC70000020FAF765FE0546B8B93F68D7F8543169
:10EC800007F5AA78D3B11846F9F7AAFC172387F835
:10EC900058314FF6FF73A7F85A311C340223C7F8D6
:10ECA0005C4187F87031C6F80080284602B0BDE8A4
:10ECB000F0810C25284602B0BDE8F081034801939D
:10ECC00040F25F21F3F7F6FD019BDCE750D5010030
:10ECD0002DE9F8430746884691461E46FBF7E2FCBD
:10ECE00000286AD090F8742190F875319A42044651
:10ECF00042D190F8F02090F8F1309A4203D090F889
:10ED0000F230032B38D0FBF7E1FC0546A0B304300A
:10ED1000FFF74AFE3146102204F281100CF0E4F8AD
:10ED200094F87A3013F0180329D0182B21D1082237
:10ED3000414604F279100CF0D7F899F8003084F8C5
:10ED4000773199F8013084F878312B7943F0030357
:10ED500001222B710A236A71EB7129463846FBF7B1
:10ED6000C1FC30B994F87431013384F87431BDE8D2
:10ED7000F8832846FBF7B0FC0C20BDE8F8832B791C
:10ED800043F003032B71172308226B7103234146C1
:10ED9000EB71A8180CF0A8F899F800302B7499F8CA
:10EDA00001306B74082105F1120001F0DBFD042134
:10EDB00005F11A0001F0D6FDCFE70220BDE8F88387
:10EDC00030B583B001A8FFF73FFF044610B12046DD
:10EDD00003B030BDFAF7E4FD054650B195F8443074
:10EDE00000226FF30003204685F844302A6203B006
:10EDF00030BD034840F2ED21F3F75CFDEEE700BFC4
:10EE000050D50100836870B51D682C6ADCB1A36D14
:10EE100000222A6223B1124840F20931F3F74AFD79
:10EE200004F14C0104F14800F5F79AFA064680B166
:10EE30002068A665FBF720FC95F844306FF30003CB
:10EE400085F8443070BD064840F20631F3F732FDD4
:10EE5000DDE703484FF44371F3F72CFDE8E700BF0B
:10EE600050D50100F8B50F2502274FF6FF7628464A
:10EE7000FBF718FC0446C0B190F93930002B14DBC5
:10EE8000FFF75EFD034604F1F5009BB900F02AFA96
:10EE900094F8F42094F8F03084F8F27042F0010213
:10EEA000013384F8F42084F8F030013DADB2B5426E
:10EEB000DDD100231846F8BD086070472DE9F04FFA
:10EEC00091B0CDE90912069390F9393002691A9F81
:10EED000DDF86C800790002B0B9202DA1346143396
:10EEE0000B9300264FF0FF09CDE90D66DFF830B235
:10EEF0008DF833903446CDF81490B24604963546DA
:10EF00003DE09DF83300FF2855D0B9F1FF0F09D03F
:10EF10000E9B534506D0584640F29D11F3F7CAFCAC
:10EF20009DF83300831E122B26D8042878D9059B20
:10EF3000FF2B71D1053880B2FBF7ACFB079B8342F6
:10EF40001AD0099A90F93930002A40F08280002BBB
:10EF500012DB0369DDF83490DDF824A02833089330
:10EF60000A9B1B684B45C0F08380089BDDF838A0E6
:10EF700004934D469DF833903B78A34254D90FAB90
:10EF80000293684B01930DAB009302210EAB0DF180
:10EF9000330200200F91F6F7A9FD02284ED00F9BF7
:10EFA000002BAED058464FF4CA71F3F783FC9DF89E
:10EFB0003300FF28A9D10A9B1B689D4238BF1D461C
:10EFC0003B78A34226D9049B574906982B44A1FBC2
:10EFD0000323C3F34F1290424FEA531340F297803A
:10EFE000049EDDF818C002E0944540F2908008EBE2
:10EFF000440008F81430120A427038780134283579
:10F00000E4B27319A1FB0323A042C3F34F124FEAEA
:10F010005313E9D80A9B1D603C7011B0BDE8F08F16
:10F020003B780590A342AAD89DF83330FF2BF3D14B
:10F030000A9B1B689D4238BF1D46EBE70F9B022BC6
:10F04000ADD102210020F6F797FD0F9B022BF8D0DF
:10F05000A5E7002B0169DDF834904CDA01F13C039F
:10F0600008930A9B1B684B454FF0140ABFF47DAF11
:10F070009D4238BF1D463B78A34231D9049B0B9A71
:10F08000CDF86C8013449A44B0462E465546DDF8C0
:10F090006CA013E0069AC3F34F18904506F12806BA
:10F0A0004FEA18204FEA531335D20AF814308CF87F
:10F0B00001003B785FFA8EF4A34222D931464846DC
:10F0C000F6F774FD049B184A3344A8420AEB440C3B
:10F0D000A2FB032304F1010EDCD235464646D0469E
:10F0E0000A9B1D60069BB3423FF63FAF9DF833304D
:10F0F000FF2B91D15FE701F1280308934FF0000A3D
:10F100002EE70A9B35461D604646D0462DE70A9BF2
:10F1100000251D6080E70A9B0025D0461D60E5E7BD
:10F1200094D50100B9EE0000CDCCCCCC2DE9F04F48
:10F130008DB0FF2507930B1D06930023044616464A
:10F140008DF827500A939A469B460DF12C090DF134
:10F15000280802272B4BCDF80890CDE900830DF14C
:10F1600027023346214600200B97F6F7BFFC022802
:10F170003DD00B9B33BB9DF82700FF282BD00538D3
:10F18000C3B20F2BE6D880B2FBF784FA0028E1D097
:10F1900090F93930002BDDDBFF2D02690A9B0CD082
:10F1A0005946184605920493F6F700FD069B03EBBB
:10F1B0000A018842DDE904320FD89DF827509246B3
:10F1C0009B46C7E7104840F26B21F3F773FB9DF8AD
:10F1D0002700FF28D3D1FF2D05D0079BC3F800B02F
:10F1E000169BC3F800A028460DB0BDE8F08F0B9B1E
:10F1F000022BBED121460020F6F7BEFC0B9B022B52
:10F20000F8D0B6E7B9EE000094D50100C3680268F3
:10F21000596858680968C08909691033F2F714BE43
:10F2200010B50446D0F8FC20016900F59273408DBA
:10F23000F2F70AFED4F824310849D4F8F820A1FBEB
:10F2400003139B0AC3F307211370517094F81A310A
:10F25000042262F3020384F81A3110BD5917B7D1A2
:10F2600010B590F93930002184B08B42BCBFD0F882
:10F27000EC30C0F8B8314FF0060204468DF80B2090
:10F28000B8BF00F5DC72D0F8B00103910DF10B01AD
:10F29000B4F89A31A8BF03AACDE900100021204696
:10F2A000FFF70CFE94F89631082262F3030384F80A
:10F2B000963104B010BD00BF10B5084C05220146C0
:10F2C00020460BF011FE05212046F5F7C5F9044B49
:10F2D0001870FFF7C7FD002010BD00BFEC0700202D
:10F2E000E909002008B5034905220BF0FDFD024B9A
:10F2F000187808BDEC070020E909002030B502FBB2
:10F30000011C02781C499DF80C50944481FB0C218F
:10F310006144491101EBC10E01EB8E010446ACEBD7
:10F320000101C8B22070C40801F0070113F804C03D
:10F330004CFA01F111F001011DD1B0FBF5F205FB12
:10F340001202D2B203F1FF3E1C1D084600F1080C68
:10F350001EF8013F5FFA8CFC13F0010F00F1010170
:10F360004FEA530302D032B1013AD2B2C8B2844557
:10F37000F2D1A645EAD130BDA7C867DD4288008832
:10F3800050407047F0B52F4D2F4C48404FF0030CC4
:10F39000070AC0B207EB872700EB802E05EA470675
:10F3A00005EA4E0004EA471704EA4E1E3E4340EACF
:10F3B0000E0000EB002706EB062E06EB0E2600EBF8
:10F3C0000720360CC0F3074040EA062000EB00108F
:10F3D0000CF1FF3C08441CF0FF0C80B2D8D1414036
:10F3E0001A48A0FB01400C1A00EB5400400900EB46
:10F3F000C00400EB8400081AC0F3C40400F0070541
:10F40000145D2C41E407C0B21AD401FB03F3561E6D
:10F41000C3F307430432604600F1080516F8011FE4
:10F42000EDB211F0010F00F101044FEA510102D0D9
:10F4300033B1013BDBB2E0B2A842F2D1B242EBD130
:10F44000F0BD00BF10210200408408004D91CFBAEA
:10F450002DE9F843184D194E002406F1FF39AF1E6F
:10F460004FF0010806E00134082C05F1060506F10D
:10F4700028061ED004EB840319F83330DA07F2D5DE
:10F4800039787A78C3F3801308FA04FCA34041EA80
:10F490000C0C1343314628460622013487F800C07D
:10F4A0007B700BF021FD082C05F1060506F12806FE
:10F4B000E0D1BDE8F88300BF425E0020015D00207E
:10F4C0002DE9F047204E214DDFF88480DFF884904D
:10F4D0000024A5F1020AB71E1AF834304FF0010CCF
:10F4E00013F0010F30460CFA04FC294606F106061B
:10F4F0004FF0060221D098F8003063B115F8013CB6
:10F50000072B03EB830E06D819F83E3013F0040FD7
:10F5100001D0DB0611D51AF8343097F800E0C3F3B8
:10F5200040034EEA0C0C97F801E087F800C0A340B6
:10F530004EEA03037B700BF0D7FC0134082C05F175
:10F540000805C9D1BDE8F087165C0020D65B002015
:10F55000D86D0020005D00200820704710B5002005
:10F56000FAF726F8F0B9FAF74DFA10F0010019D1C0
:10F570000D4A0E4C02EBC0035B78072B03EB8301B3
:10F5800005D814F831306FF3451304F8313012F810
:10F5900030306FF3000302F8303001300828E9D131
:10F5A000002010BD0C2010BDD45B0020005D0020A9
:10F5B0002DE9F04F074683B00020F9F7F9FF002846
:10F5C0006FD1FAF71FFA10F001046AD197F800A082
:10F5D000BAF1FF0F69D0414E07F1010B0AF0010AA1
:10F5E0004FF0FF092546A6F1020809E0B9F1FF0F27
:10F5F00001D15FFA85F90135082D06F1080617D00B
:10F6000018F83530D807C3F34002EFD55245F2D190
:10F610000622304659460BF03EFC00283ED018F832
:10F620003530D907E2D50135082D06F10806E7D1B6
:10F63000B9F1070F3DD83A7818F83930284E022032
:10F6400062F3410315FB090008F8393040440622F3
:10F6500059460BF049FC3B78771E03F0010304EB9D
:10F6600084055FFA84FA17F83520C2F38011D207B7
:10F6700004F101044FEAC50501D599421BD0082CBD
:10F6800006F12806EBD108EBC903FF225A7018F8DF
:10F69000393043F0010308F83930002003B0BDE8E9
:10F6A000F08F0C2003B0BDE8F08F204603B0BDE81A
:10F6B000F08F0720F2E730460622594601930BF0FF
:10F6C000EAFB019B0028DAD17B5D43F020037B55E8
:10F6D00008EBC90383F801A0D9E700BFD65B00207F
:10F6E000015D00202DE9F04106460020F9F760FF9A
:10F6F000F0B9FAF787F910F0010419D196F80080F3
:10F70000B8F1FF0F35D01C4D0136AF1E08F00108CF
:10F7100017F83430C3F34002DB0701D542450AD065
:10F720000134082C05F10805F2D10220BDE8F08172
:10F730000C20BDE8F0810622284631460BF0ABFBD9
:10F740000028EDD107EBC4035B78072B08D80B4AE0
:10F7500003EB830312F8331060F3451102F8331002
:10F7600017F834306FF3000307F834300020BDE899
:10F77000F0812046BDE8F081D65B0020005D0020CE
:10F7800007282DE9F04104460E46904617D8124D41
:10F7900004EB8403A70015F83330DB0715D52744A5
:10F7A000282115F83730C3F3801301FB045133705F
:10F7B00040460622BDE8F04101310BF095BB0748F9
:10F7C0004FF48971F3F776F8E1E7044840F213113A
:10F7D000F3F770F8E3E700BF005D0020D8D5010023
:10F7E0000820704710B50020F9F7D6FE08B10C20AC
:10F7F00010BDFAF7EFF830F00100F8D1184B194CB2
:10F80000197893F82820207060F3000160F300025B
:10F81000197083F8282093F8501093F8782060F33B
:10F82000000160F3000283F8501083F8782093F809
:10F83000A01093F8C82060F3000160F3000283F881
:10F84000A01083F8C82093F8F01093F8182160F303
:10F85000000160F3000283F8F01083F8182110BD56
:10F86000005D0020D76D00202DE9F04F83B00346E6
:10F8700000200093F9F790FE18B10C2003B0BDE80A
:10F88000F08FFAF7A7F830F0010BF6D1009BDFF804
:10F89000348113F801AB5C460AF0010A08F1FF3726
:10F8A0001E4604EB840207EBC20517F83230C3F39F
:10F8B0008012DB074FEA840901D5524508D0013494
:10F8C000082C08F12808ECD1022003B0BDE8F08F25
:10F8D0004046062231460BF0DEFA0028EFD12A78A6
:10F8E00052073346064635D5DFF8DCA09AF800808B
:10F8F00008F1FF3818F0FF082AD0ED7D454527D0E4
:10F900003248019300EB0811102200EB05100BF0B8
:10F91000EBFA2F48019B0BEB8B025FFA8BFC17F87D
:10F92000321011F0010F0BF1010B07EBC20204D0F2
:10F93000490702D5C17D414539D0BBF1080F00F11F
:10F940002800E8D19AF8008008F1FF385FFA88F8BB
:10F950008AF80080009A1F4D92F800A0A5F10208D5
:10F960000AF0010A9B4618F83620D107C2F340007E
:10F9700001D550450FD00136082E05F10805F2D10A
:10F980004C44002017F834306FF3000307F834308C
:10F9900003B0BDE8F08F0622284659460BF07BFAEB
:10F9A0000028E8D108EBC606FF237370E8E79AF851
:10F9B0000080D575084A08F1FF3802F805C05FFAE3
:10F9C00088F8C5E7015D0020D76D0020805C00202D
:10F9D000005D0020D65B0020785C00202DE9F04718
:10F9E0005C7904F0C004402C01D0BDE8F0871E46CD
:10F9F0000F4601B3DFF8A090002400F0010A09F1DE
:10FA0000FF3803E0082C09F12809EED004EB840349
:10FA1000254618F83320C2F38013D20704F10104FD
:10FA2000F0D55345EED14846062239460BF033FA5D
:10FA30000028E7D104E0072AD7D8DFF86080154610
:10FA400005EB8505EF0018F83530DB07CDD507F15C
:10FA50001809C1440622314648460BF045FA0024F5
:10FA600001E0102CC1D0A0B2FAF71CFE034600F151
:10FA7000DD050134062249462846002BF1D00BF063
:10FA80000AFA0028EDD1791C414428460622BDE837
:10FA9000F0470BF029BA00BF015D0020005D002097
:10FAA0002DE9F84F82461A4E1AF8018B8946002438
:10FAB00008F00108771E04EB8402D50017F83230F5
:10FAC000C3F38012DB0704F1010401D5424506D0DF
:10FAD000082C06F12806EED10220BDE8F88F30464A
:10FAE000062251460BF0D7F983460028F0D105F1E4
:10FAF0001802174406213846F4F722FC0028EBD000
:10FB00000622394648460BF0EFF95846BDE8F88F13
:10FB1000015D00202DE9F84F8146164E19F8018B42
:10FB20008A46002408F00108771E04EB840207EBE4
:10FB3000C20517F83230C3F38012DB0704F1010469
:10FB400001D5424506D0082C06F12806EDD1022049
:10FB5000BDE8F88F3046062249460BF09CF98346F3
:10FB60000028F0D1696A062250460BF0BDF95846CC
:10FB7000BDE8F88F015D002010B504460020F9F7BC
:10FB80000BFD08B10C2010BDF9F724FF30F0010087
:10FB9000F8D134B1012C02D1044B1C7010BD1220DD
:10FBA00010BD024B1C70204610BD00BFD86D002058
:10FBB000034B4FF47A7202FB00F01860704700BFED
:10FBC000745E00202DE9F047824600208846F9F750
:10FBD000E3FC10B10C20BDE8F087F9F7FBFE30F034
:10FBE0000104F7D11A4E1AF8019B771E09F001099A
:10FBF00004EB8402D50017F83230C3F38012DB0720
:10FC000004F1010401D54A4506D0082C06F1280666
:10FC1000EED10220BDE8F0873046062251460BF0B7
:10FC20003AF90028F1D1B8F1000F0BD0B8F1010F6B
:10FC300005D17B5D43F010037B55BDE8F0871220B2
:10FC4000BDE8F0877B5D68F304137B554046C2E74F
:10FC5000015D0020D0B43049304C002304EBC302D6
:10FC60005278072A02EB820C05D811F83C206FF37A
:10FC7000451201F83C2014F833206FF3000204F819
:10FC800033200133082BE9D1254A264C0023137079
:10FC90000A7863F300020A7091F8282063F30002E7
:10FCA00081F8282091F8502063F3000281F8502059
:10FCB00091F8782063F3000281F8782091F8A02071
:10FCC00063F3000281F8A02091F8C82063F30002DA
:10FCD00081F8C82091F8F02063F3000281F8F02049
:10FCE00091F8182163F3000281F818210E4A13706D
:10FCF0000E4B4FF0FF364FF0FF37C3E900670C4B58
:10FD0000236020B1D0BC0B490B480CF07ABDD0BCAD
:10FD100009480CF082BD00BF005D0020D45B0020CC
:10FD2000D86D0020745E0020D76D0020E02B0020ED
:10FD3000A0BB0D00E1FF0000E82B0020034A044BAC
:10FD400000280CBF10461846704700BF405E0020D8
:10FD5000145C0020A8B10C4A126810B54FF400439F
:10FD600040F2E7300021E2FB03014FF47A720023F6
:10FD7000F0F7C6F9BDE8104002460B46034807F00D
:10FD800019BA02480CF049BD745E0020E82B00202F
:10FD90000D4A08B50023138070B90C4B0C4A1B7830
:10FDA0000020108003B908BDF9F714FE0028FAD12D
:10FDB000BDE80840FFF74CBB1846F9F723FEC30720
:10FDC000EBD4FFF77DFBE8E7145C0020D86D002042
:10FDD000405E00200E4A08B500231380C2070ED4EF
:10FDE0000C4B0D4A1B780020108003B908BDF9F7B1
:10FDF000D3FB0028FAD1BDE80840FFF729BB18461D
:10FE0000F9F7D6FB0028EBD1FFF75AFBE8E700BF74
:10FE1000145C0020D86D0020405E00202DE9F04FDA
:10FE2000824687B00CF062FE4B014201121A43EA8F
:10FE3000D06363EB01039B004FEA820818EB0008D4
:10FE400043EA927341EB0301CB0043EA5873D90BA9
:10FE5000C8F3103848EA43480191BAF1000F17D1AE
:10FE6000594AD2E90032B2F1FF3F08BFB3F1FF3F78
:10FE70000ED0B8EB030361EB0202544909688B42D0
:10FE800072F10003ACBF4FF001094FF0000901E02F
:10FE90004FF001094E4EDFF83CB10024A6F11E07D9
:10FEA00004EB8403A50017F83330DA0715D5B9F150
:10FEB000000F01D1980710D42B1917F833305907C8
:10FEC00060D42B1917F833301A074AD4254417F891
:10FED000353043F0020307F835300134082C0BF1BC
:10FEE000060B06F12806DBD1B9F1000F04D0364B22
:10FEF000019AC3F800805A60BAF1000F08D00020C0
:10FF0000F9F73CFB044618B194F86A305B0702D459
:10FF100007B0BDE8F08F94F82630072BF8D8FF2300
:10FF20008DF8083094F8293004EB830302A9DE6AC7
:10FF300004F1280001F056F9727805460232314684
:10FF40000AF0D2FF002DE3D029462046F9F740FB06
:10FF50009DF80830FF2BDBD084F8293007B0BDE8CE
:10FF6000F08F02A9A6F117000BF031F830BB02ABFD
:10FF7000C6F806300622194658460AF0B5FFC6F8FC
:10FF800006B0A3E7144B16F8072C03EB02120F324E
:10FF90000DF107030DF1170012F8011903F8011F05
:10FFA0008342F9D1314602A80BF011F8002888D01D
:10FFB0000A4840F2EB21F2F77DFC82E707484FF454
:10FFC0003E71F2F777FCD2E7E02B0020745E002050
:10FFD0001E5D0020485C0020805C0020D8D5010018
:10FFE00010B50120FFF71AFF0A4A12684FF40043C8
:10FFF00040F2E7300021E2FB03014FF47A72002364
:020000021000EC
:10000000F0F77EF8BDE8104002460B46024807F0C4
:10001000D1B800BF745E0020E82B0020072813D859
:1000200070B500EB80030C4D15F833301A07044609
:100030004FEA8006C3F3C00005D59B0706D53444BC
:1000400005EBC405686A70BD00207047034840F2A4
:100050001F31F2F72FFCF2E7005D0020D8D5010038
:1000600007280BD800EB8003054A12F833104B0722
:1000700004D5282303FB00201E3070470020704762
:10008000005D00202DE9F84F8B4617460AB1FF238B
:1000900013701B4D002400F0010A05F1FF3906E042
:1000A00052451FD00134082C05F1280515D004EB6A
:1000B00084065FFA84F819F83630D907C3F3801242
:1000C000EED4002FEED03B780134FF2B08BF87F829
:1000D0000080082C05F12805E9D14FF0FF084046C3
:1000E000BDE8F88F2846062259460AF0D4FE0028BB
:1000F000F5D0002FD6D019F83630DB07D2D4E2E79E
:10010000015D00202DE9F04F804685B000200E46AD
:100110009146F9F741FA18B10C2005B0BDE8F08F0F
:100120000446F9F757FC30F00103F5D1C2460DF152
:100130000F021AF8010B5146FFF7A4FF072840F2FF
:10014000B1809DF80F70072F00F2A88007EB870B96
:10015000564D4FEACB03581C0622514628440093C3
:100160000AF0C2FE98F8003015F83B105A464FEAE4
:10017000CB0B63F3861105F80B1005EBC2031021BE
:1001800030460193F4F7DCF815F80B20102160F3EA
:100190008202484605F80B20F4F7D2F815F80B2038
:1001A00000F0010060F3C30205F80B2052074FEA8C
:1001B000870B4BD4002863D100983D4E183006229F
:1001C000002128440AF09BFE0BEB070215F83210C1
:1001D00021F0120105F8321098F80090A6F10208FB
:1001E00009F0010918F83420D307C2F3400101D502
:1001F000494518D00134082C06F10806F2D10BEB62
:10020000070215F832106FF3451105F832100BEBA9
:100210000703002015F8332042F0010205F83320CF
:1002200005B0BDE8F08F0622304651460AF033FE95
:100230000028DFD10BEB070208EBC40415F83210DD
:10024000677041F0200105F83210E0E7194B1A4AB7
:100250001978DDF804C05754184A8CF8171002EBCF
:10026000011C013106F10F0219700CF1FF3C013E37
:1002700012F801190CF8011F9642F9D100289BD001
:10028000009BD81D4946102228440AF02DFE0BEB96
:10029000070205EBC202002151628DE7072005B07D
:1002A000BDE8F08F122005B0BDE8F08F005D0020A2
:1002B000D65B0020D76D0020785C0020805C002099
:1002C000072807D8044B00EB800013F83000C0F378
:1002D000C000704700207047005D0020072812D83A
:1002E00000EB8000094A12F8303013F0080F4FEA93
:1002F000C001C3F3C00007D0C3F340009B0703D580
:100300000A44506A70470020704700BF005D00201B
:10031000024B1B7803700248704700BFD76D002066
:10032000805C002038B50C4650B107291AD81A4D08
:1003300015F83430DA071FD505EBC404607838BDF2
:10034000072922D8154B04EB840213F83230DB075F
:1003500001D5204638BD124840F26631F2F7AAFABC
:10036000204638BD0C4D0E484FF45871F2F7A2FAF2
:1003700015F83430DA07DFD405EBC404084840F23E
:100380006131F2F797FA6078D9E705484FF459716F
:10039000F2F790FAD6E700BFD45B0020005D0020A2
:1003A000D8D5010010B5144B1B78834204460CD9F4
:1003B000124B1C5D072C11D8114B04EB840213F86F
:1003C0003230DB0710D5204610BD0E484FF45C716B
:1003D000F2F770FA094B1C5D072CEDD9094840F281
:1003E0007231F2F767FAE7E7064840F27331F2F745
:1003F00061FA204610BD00BFD76D0020785C002058
:10040000005D0020D8D5010007281BD870B500EB8F
:1004100080030D4E16F83330DB0704464FEA8005A3
:1004200005D52C4416F83400C0F3401070BD2C44A0
:10043000064840F27E31F2F73DFA16F83400C0F378
:10044000401070BD00207047005D0020D8D501002D
:10045000104B1B789BB1072970B50C460DD860B9BD
:100460000D4E01EB81038D0016F83330DA070BD502
:100470002C4416F83400430703D4012070BD01203A
:100480007047C0F3001070BD044840F29731F2F796
:1004900011FAEDE7D86D0020005D0020D8D50100ED
:1004A0001378FF2B1BD12DE9F04F194D0446AE46B2
:1004B000002303EB830CDFB215F83CC01CF00100F5
:1004C0004FEA830603D0CCF3801CA44509D0013346
:1004D000082B0EF1280EECD10120BDE8F08F012091
:1004E000704701F1FF38F4460EF1060B1CF801AF1E
:1004F00018F8019FCA45EAD1DC45F7D1334417709B
:1005000015F833305A07E8D5C3F30010E5E700BF0C
:10051000005D002010B40E4B1C787CB1072A0DD86A
:100520000C4C02EB820C14F83CC01CF0080F05D0F8
:1005300020B14B7903F0C003402B02D0002010BC47
:100540007047282000FB0240073010BC0AF02CBD89
:10055000D86D0020005D0020024B1878003818BFCD
:1005600001207047D86D0020684620F007018D46B5
:1005700001B502F049FDF3F7ABF9F3F793FABDE8E3
:1005800001408546704700BF08B5094BD3F84021AC
:100590003AB90120F3F7BAFFBDE808400220F3F7AB
:1005A000B5BF0020C3F84001F5F766F9F1E700BFD9
:1005B00000B000400020F3F7A9BF00BF10B50A4B00
:1005C0000A4C1A7823789A4206D00949094A0978D0
:1005D00011700133237010BD074840F20231F2F769
:1005E00069F92378F1E700BFDE6D0020DD6D0020A2
:1005F000D96D0020DA6D00201CD6010038B5B8B9DD
:10060000124B134D1A782B789A4217D0114A124C7C
:1006100012782178013391422B70D3B205D00F4864
:100620004FF44471F2F746F923780133237038BD53
:100630000A4840F20B31F2F73DF9E1E7074840F292
:100640000D31F2F737F92B78E0E700BFDC6D0020C1
:10065000DB6D0020D96D0020DA6D00201CD6010072
:1006600002F086BE10B51349134A0B7812789A42ED
:1006700082B01AD1114B124A1B7812789A4214D0C8
:100680000878104B01300022C0B200920870114669
:100690001046F5F7E9F9044638B1022806D00A48B1
:1006A00040F26331F2F706F900E00024204602B080
:1006B00010BD00BFDE6D0020DD6D0020D96D002073
:1006C000DA6D0020BD0501001CD601002DE9F047C0
:1006D000CB68D1F800801A682A4B2B4FD6680D469C
:1006E000044619789068536898422CBFC6EB000600
:1006F000C6EB03063B7899428AB008EB060933D073
:10070000002C3AD0237F9B0737D4DFF880A0DAF89B
:100710000000A9EB000010F4000022D0FFF7A2FFB8
:10072000237FE168CAF8009043F002032377204654
:10073000A3699847164B3C780096CDE90735154BD1
:10074000CAF8009000220134CDE90535E4B2CDE9C4
:100750000322CDE901224346114610463C70F5F7CD
:10076000F9F80AB0BDE8F0870B4B0C4A1B781278F9
:100770009A42C5D1DFF814A0DCE700200AB0BDE83A
:10078000F08700BFDB6D0020DC6D0020905E002054
:10079000FD050100A9080100D96D0020DA6D0020D7
:1007A000F0B53F4EB36889B0B3B13368A3B1FF234E
:1007B00005460DF10A008DF80A30F8F7FFF80146FA
:1007C00050B10B7F13F003040DF10A0006D0F8F7C7
:1007D000F5F801460028F4D109B0F0BD8D421ED1D4
:1007E00073683168E86803AA9847074670B1B36830
:1007F00031682046984717F10B0F1CD08C37EBD08F
:10080000284840F2D131F2F755F8E5E72B7FAA6985
:10081000E96843F002032B7728469047DCE720463F
:10082000FFF754FF30F00203D6D01E4840F29D314E
:10083000F2F740F8D0E7FF240DF10B008DF80B40E4
:10084000F8F7BCF828B913E00DF10B00F8F7B6F88B
:1008500070B1037F9A07F7D4C26831689142F3D12F
:1008600043F002030377836998478DF80B40EBE769
:100870000021306806910123CDE90411009307900F
:100880003160039BD6E9010104AAF8F757F8002864
:10089000A2D1044840F2CF31F2F70CF89CE700BF38
:1008A0007C5E00201CD6010038B5104A104C12782E
:1008B0002378059D9A4213D021780E4B0131C9B29D
:1008C00000222170012011469D60F3F7C7FD00B999
:1008D00038BDBDE83840084840F27731F1F7EABF4B
:1008E000054840F27131F1F7E5FFE5E7DA6D0020E8
:1008F000D96D0020F40700201CD6010010B5164861
:1009000005F0AAFF154B186010B3154B00249C602E
:1009100000F08EFA00281ADB214601202246F2F769
:10092000BFFF22460B200121F2F7BAFF22462146E3
:100930001820F2F7B5FF0120F2F780FF0B20F2F745
:100940007DFF1820F2F77AFF02F08EFB204610BDE3
:100950006FF0120010BD00BF64D60100785E002069
:100960007C5E0020054A10B4034610688468246841
:100970008AB21946234610BC184700BF785E002093
:10098000084B30B41D68AB685C683CB10A46A446AD
:10099000014692B22846002330BC60476FF08500C4
:1009A00030BC7047785E0020084B30B41D68AB68DF
:1009B0005C683CB10A46A446014692B22846002330
:1009C00030BC60476FF0850030BC7047785E002017
:1009D0000020704730B5044683B078B31F4B1A68C7
:1009E000824225D0FF250DF107008DF80750F7F75B
:1009F000E5FF38B91AE08C420AD00DF10700F7F78D
:100A0000DDFF98B1037F9B07F7D4C168002CF2D1BA
:100A1000037F826943F00203037790470DF10700DB
:100A20008DF80750F7F7CAFF0028EBD103B030BDAF
:100A30009B686BB1214600209847D3E7074A93682B
:100A4000002BCFD011680029CCD000209847C9E7EF
:100A50000348FD21F1F72EFFC4E700BF7C5E0020B4
:100A60001CD601000020704738B50446F7F798FF00
:100A700054B1D0B124680020F7F7C0FF2046F8F742
:100A800015F858B1002038BD0E4DAB689BB12C68ED
:100A90000023AB602B60002CECD1ECE70A4840F25D
:100AA0006D11F1F707FF002038BD074840F23711FC
:100AB000F1F700FFDEE7044840F23D11F1F7FAFEDE
:100AC000E5E700BF7C5E00201CD60100054A1368E4
:100AD00092681B1A18BF0123B2FA82F00B7040090A
:100AE000704700BF7C5E00206FF08B00704700BF36
:100AF000D0E90132002A04DB9A4238BF1A46104678
:100B00007047C068984238BF1846704710B5144601
:100B1000F5F74AF8001B030205D40330092894BFF7
:100B20000020012010BD002010BD00BF262810B5F8
:100B300004461CD0272812D0252808D00A281ED900
:100B4000272821D80330400002F06CFB02E002208D
:100B500002F068FB2046BDE8104002F069BB50205F
:100B600002F060FB2046BDE8104002F061BB1A2095
:100B700002F058FB2046BDE8104002F059BB02309D
:100B8000400002F04FFBE5E7024840F2DF11F1F7C9
:100B900091FEDFE71CD6010002F0AEBB02F0B8BB4D
:100BA00008B502F0E5FBBDE8084002F059BE00BF01
:100BB00008B502F0DDFB02F053FEBDE8084002F08C
:100BC000FBBD00BF08B502F0D3FB02F049FE02F006
:100BD0002FFE03F071F8BDE8084002F0EDBD00BF44
:100BE00008B50146134802F01FFA02F0E3FB60B1BA
:100BF00002F012FF02F080FA00F076F900280EDB16
:100C0000BDE808400020FFF72FBF02F09DFB02F077
:100C100003FF02F071FA00F067F90028F0DA0648E5
:100C200040F24321F1F746FEBDE808400020FFF7FF
:100C30001BBF00BF610601001CD6010010B50446B1
:100C400002F096FB02F00CFE02F0F2FD03F034F825
:100C500002F0B2FD2046BDE81040FFF7C1BF00BF63
:100C600008B501460F4802F0DFF902F0A3FB40B1DE
:100C700000F03AF900280ADBBDE808400020FFF741
:100C8000F3BE02F061FB00F02FF90028F4DA064809
:100C900040F25221F1F70EFEBDE808400020FFF7B8
:100CA000E3BE00BF610601001CD601002DE9F0473C
:100CB00084B006461D460DF10F00FF239DF83090CD
:100CC0008DF80F300F469046F7F778FE044620B9AE
:100CD0002AE0F7F773FE044630B394F81CC01CF00A
:100CE000030F0DF10F00F4D1DFF8E0A0DAF80830BF
:100CF00003BBB9F1000F37D0CDF8009043462A4628
:100D000039463046F7F71AFE40B9314840F28E2195
:100D1000F1F7D0FD0020B9F1000F18D06FF0760484
:100D2000204604B0BDE8F087DFF8A0A0DAF808306C
:100D30000BB30024CDF8009043462A46394630468E
:100D4000F7F7FCFD0028E0D0B9F1000FE6D101462D
:100D50002046FFF7BBFC30F00203DFD01C4840F216
:100D60009921F1F7A7FDD9E7AC4204D0184840F229
:100D7000BF21F1F79FFDEB68CAF80030CAE90167AF
:100D80002846C0470446FFF76DFC30F0020316D139
:100D90000DF10F00F7F712FE0028C1D0037F13F00A
:100DA0000303F5D101461846FFF790FC30F002032B
:100DB000B6D0074840F2D921F1F77CFDB0E70448EE
:100DC0004FF43371F1F776FDE2E700BF7C5E00205F
:100DD0001CD6010001F1100006F056B870B50546AA
:100DE0008AB00C460122002104A80BF068FC0F4BCE
:100DF000019300260323694628460396029309F0CF
:100E000062FD002810DB4FF40043314640F2E7302A
:100E1000E4FB03014FF47A720023EFF771F9024605
:100E20000B4604A806F056F80AB070BDD50D0100B7
:100E300010B5012003F004FB0449002301248C6059
:100E40004B60BDE81040CB6009F03DBD985E0020CE
:100E50000C4B1A780AB10020704710B501201870A9
:100E600003F0EEFA4FF4FA710446FFF7B7FF38B912
:100E7000204609F071FD02280CBF00206FF004002D
:100E800010BD00BFDF6D002008B50A4BBFF35B8FBC
:100E900053E8002F511C43E800100028F8D1BFF39D
:100EA0005B8F002A01DD002008BD03F0D1FA00208D
:100EB00008BD00BF945E002008B5002003F0C0FA12
:100EC000BFF35B8F074B53E8002F013243E800214B
:100ED0000029F8D1BFF35B8F0221BDE80840FFF77E
:100EE0007DBF00BF945E002008B50D4B1A68002A34
:100EF00012DDBFF35B8F53E8002F511E43E8001053
:100F00000028F8D1BFF35B8F012A01DD002008BD66
:100F100003F0B4FA002008BD6FF0770008BD00BFF1
:100F2000945E00200520704732207047014B33F853
:100F30001000704768D6010010B50446FFF742FE66
:100F400002F06CFC2046BDE81040FFF749BE00BF30
:100F500030B583B00546FFF723FE962002F090FCE3
:100F6000002318461A46194602F0D2FB0120F7F773
:100F700097FC044600283DD004F11C0002F0B0F9B3
:100F800002F004FAF0B91E48294602F04DF8FFF7C6
:100F9000E3FA20BB02F094FD00210446084602F06B
:100FA000B9F900210546084602F0B0F92C44C334D3
:100FB000201A02F03DFD02F075FD03B0BDE830409F
:100FC00002F0EABB0F4840F27D41F1F773FC0C4898
:100FD000294602F029F8FFF7BFFA0028DAD00DF110
:100FE0000700FFF795F9002201469DF8070002F07F
:100FF00023FECFE7034840F27941F1F75BFCBBE702
:101000008516010078D60100814208B50ED00B7A12
:10101000DB0702D46FF08B0008BD0F4B1360FFF7A6
:1010200033FF00280FDB6FF00A0008BD0B7B01EBDC
:1010300083010B691B7803F00F03012B14BF6FF0C2
:101040008B00002008BD054840F23241F1F732FC28
:101050006FF00A0008BD00BFC914010078D6010076
:1010600010B598B10C46FFF73FFF002804DB20467F
:10107000BDE81040FFF7F8BC08484FF48B61F1F76A
:1010800019FC2046BDE81040FFF7EEBC044801F013
:10109000CBFFBDE8104002F057B900BF78D6010081
:1010A000390F0100084B042210B598182821F3F7D6
:1010B000CDF8064B00249C800222214604480BF008
:1010C000FEFA204610BD00BFA85E002004080020E4
:1010D0004C5F0020084B042210B598182821F3F724
:1010E000B5F8064B00249C800222214604480BF0F0
:1010F000E6FA204610BD00BFA85E002004080020CC
:101100004C5F002010B504460548F3F7CFF820B136
:10111000034600205870636010BD6FF00B0010BDD7
:10112000A85E002003460020187058709860704731
:1011300038B5284C227961792378914203D002FB9B
:1011400003439D6835B92448F3F7B0F80546A0B1CC
:10115000284638BD21480022002305F0BBFE38BBDD
:1011600023796279A1789A42F2D00133DBB29942B5
:1011700008BF00232371284638BD18484FF0FF32BE
:101180004FF0FF3305F0A6FEF0B92379617922789C
:10119000A078994212D003FB024201339268DBB27D
:1011A000984208BF0023237142B11546284638BD36
:1011B0000B484FF4CD71F1F77DFBD1E708484FF4B0
:1011C000D871F1F777FBC3E7054840F2AD11F1F7AD
:1011D00071FBDAE704080020A85E00204C5F0020C5
:1011E00078D6010010B5027843789A4214D0D4B270
:1011F00044700278944204D05A1C4370D3B2022B3C
:101200000ED01C4600EB84040B70606800B110BD6A
:10121000FFF78EFF606010BD0133DBB2022BF0D10F
:1012200000242346EEE700BFF8B504460378407873
:10123000984228D0164A0E46517992F802C0DDB283
:101240004B1CDBB29C4508BF002392F804C004EBA2
:1012500085079C45786809D092F800C00CFB0121F5
:10126000886053710B4805F00FFE00206B1CDBB249
:10127000022B786004BF002003464FF00102237068
:1012800018BF1846327004EB80046068F8BD00BFD8
:10129000040800204C5F0020037A70B5C3F30213EA
:1012A000002B044693FAA3F0B0FA80F008BF4FF089
:1012B000FF30451C82B041D0217A5A1E134063F39F
:1012C000061105F124002172FFF730FC00230DF117
:1012D000070104F10C008DF80730FFF7A5FF054664
:1012E000A8B3284602F002F82B7803F00F03022B74
:1012F0001CD00DF1070104F11800FFF795FF064619
:1013000058B39DF807305BB92146174801F08CFEB1
:10131000962002F0B5FA002002F0E6F902B070BDA6
:101320000622A91CB01C09F0DFFDEDE70F4821469D
:1013300001F07AFE02F018FA02B070BD0C4840F2DB
:101340006F51F1F7B7FA237AC3F30213B4E70848F1
:101350004FF4AF61F1F7AEFAC3E7054840F28251AE
:10136000F1F7A8FACDE700BF510F01007513010096
:1013700078D6010010B50446FFF724FC237A03F069
:101380007102012A05D1C3F3420262F306132372EC
:10139000DBB213F0700F05D0636853B193F82030BF
:1013A0009B0706D502F03AFA2046BDE81040FFF749
:1013B00017BC2046FFF770FF01F0C0FFBDE81040EA
:1013C00002F070BBF0B5C468636883B00546002BBB
:1013D00065D101F06BFE002001F0E6FE0021084619
:1013E00001F08CFE00222521082001F04BFF314B3B
:1013F000019301A801F02EFF2F4940F25B6001F03C
:10140000E3FF237AC3F3420262F3061320462372FA
:10141000FFF742FFFFF7A0F898BB637A9B0727D13D
:1014200027682E683846FFF763FB06446A6806F1B2
:101430000901012002F030FA02F034FB2046F8F7EF
:101440008FF8811C3246C9B23846FFF75FFB30B9CE
:101450002046FFF707FBD0B9002003B0F0BD1748C6
:10146000214601F0E1FD01F06FFF002003B0F0BD67
:101470000120FEF763FC4178821C007802F0AEF98F
:10148000CEE7607A10F0030018BF0120F1E70C48A6
:1014900040F20941F1F70EFA002003B0F0BD93F8D5
:1014A00020309A0795D00748214601F0BDFD01F094
:1014B0004BFFD1E7D6BE898E55555500390F010037
:1014C00078D60100610C0100C36870B51E6804463F
:1014D000F4F76AFB05463046FFF70AFB00232D1A96
:1014E000C4E9005323812046BDE87040FFF76ABF7E
:1014F00010B582B00446FFF7C7FC002813DB0D4A85
:101500000D490E4800940023F7F798FC08B1773096
:1015100001D102B010BD0A484FF4287102B0BDE8F5
:101520001040F1F7C7B9064840F29D21F1F7C2F922
:10153000E5E700BFC51301006110010009100100BB
:1015400078D601002DE9F04190F809C09DF8188087
:101550001CF0010F0F4616461D4609D0B8F1000FCA
:1015600016D03B78B6EBD31F19D00020BDE8F08130
:10157000044611F8020B079AC0F38010FEF790FFA3
:101580000028EED1637ADB07EFD5B8F1000FE8D180
:10159000079B1878FEF738FF0028E2D1E5E706221E
:1015A00007F10801284609F076FCB0FA80F04009FE
:1015B000BDE8F0812DE9F0471F46099B9DF820907A
:1015C0009DF8286005460C469046FBB9437A9A0779
:1015D00007D5A6B12378B8EBD31F3AD00020BDE8D9
:1015E000F08711F8020B0B9AC0F38010FEF758FF3A
:1015F0000028EFD16B7A9B07F0D5002EEAD10B9B28
:101600001878FEF701FF0028E4D1E7E78A460B9A35
:101610001AF8020BC0F380105146FEF741FF002874
:10162000DCD02378B8EBD31FD8D13846062204F19A
:10163000080109F030FC0028D0D10B9B1878FF2856
:1016400011D0AB7AFF2B0ED0C01AB0FA80F040094F
:10165000C5E7062204F10801384609F01CFCB0FA7F
:1016600080F04009BBE72378C3F380134B45B5D125
:1016700009980622514609F00EFCB0FA80F04009A4
:10168000ADE700BF2DE9F0478AB0044601F088FEBF
:10169000C0B250B9FFF796FA7548214601F0C4FC74
:1016A0000AB0BDE8F04701F04FBE01F099FE0546D3
:1016B00002F0C6F8074602F0CDF802F013FB8246AE
:1016C00002F0F4FA814602F07FF8EDB28046FFF7AF
:1016D00079FA002DE0D01AF0FF0A7FD1FF208DF8B3
:1016E00027000120F7F7DCF80546002800F0A3806A
:1016F000237B04EB830305F11C0118690346FFB249
:1017000013F8026B06F00F0CBCF1010F08BF00F1DB
:101710000809287F00F00F0018BF4FF000090328C8
:10172000C6F380124FEAD6165FD00528B4D1687F81
:101730002228B1D160680028AED090F82000800740
:10174000AAD40DF127000390CDE901970096204619
:10175000FFF730FF00289FD00420F7F7A1F80028FA
:101760009AD04448214601F05FFC01F0EDFD01F004
:101770000DFE002859D15FFA88F000284FD1626829
:1017800092F8203043F0010382F82030F7F7A8F8F0
:1017900017224FF6FF730271C3808460054602F082
:1017A00035F9286102F086F900210446084601F067
:1017B000B1FD241A6C61BAF1000F14D09DF82730E6
:1017C0006B76F7F78DF8034629462868EB60F7F744
:1017D0009DF8F7F7ABF80AB0BDE8F0875FFA89F03B
:1017E000FEF7E0FD7BE7FF23EAE7687F0C287FF444
:1017F00053AFB9F1000F7FF44FAF0DF12700019007
:1018000000972046CDE906230591FFF79BFEC0B95E
:10181000287F079BDDE9051200F00F0085E701F046
:10182000C5FF626882F8A100AAE7134840F212617E
:10183000F1F740F89FE7104840F2B251F1F73AF85B
:1018400056E721460A4801F0EFFB01F08DFF237EA9
:1018500004EB8304E06901F049FD01F097FD0028E5
:10186000B9D0054840F2CB51F1F724F8B3E700BFF7
:1018700075130100390F010078D601002DE9F04100
:10188000C46894F91630002B8CB0C0F2EE80636807
:1018900005460F46002B40F0DD80A37D6FF300036B
:1018A000A37501F003FC002001F07EFC0021084636
:1018B00001F024FC00222521082001F0E3FC012096
:1018C000F6F7EEFF0646002800F0BE8006F11C0089
:1018D00001F006FD6A4B0B930BA801F0BBFC6949B4
:1018E00040F25B6001F070FDA07DC0F34100253047
:1018F000FFF71CF96448214601F096FBA37D9B0687
:1019000003D46368002B00F08180962001F0B8FFBB
:1019100000231A461946184601F0FAFEFEF71CFE8F
:10192000002835D1A37D13F0180F52D1D4F80080D0
:101930002E684046FFF7DCF806446A6806F10901A4
:10194000002001F0A9FF02F0ADF801F025FF2046CC
:10195000F8F718F8011DC9B240463246FFF7D6F82D
:1019600068BB17B9636A002B53D1636843B1474B17
:101970000122022100209D60F2F770FD00283AD17B
:101980002046FFF76FF868BB00200CB0BDE8F0817F
:10199000A07DC0F3C000FEF7D1F906460DF12B0083
:1019A000FEF7B6FC71788046B21C307801F016FF65
:1019B0009DF82B000022414602F03EF9B6E734487C
:1019C000214601F031FB01F0BFFC00200CB0BDE866
:1019D000F0810120FEF7B2F94178821C007801F015
:1019E000FDFEA3E72B4840F21521F0F763FF00202E
:1019F0000CB0BDE8F08127484FF40471F0F75AFFAE
:101A00002046FFF72FF80028BED0EBE701F0ACFE30
:101A100084E7214A0792214A059240F2FB12009383
:101A200008923346CDE90377CDE90177069439462C
:101A30000322F3F78FFF30F0020396D015484FF4DE
:101A4000FE71F0F737FF90E712484FF4C771F0F7D7
:101A500031FF3BE7636893F82030D90705D463680A
:101A600093F820309A077FF518AF0D48214601F012
:101A7000DBFA01F069FC00200CB0BDE8F08100BF8A
:101A8000D6BE898E55555500392100002808002002
:101A9000351B0100C4D60100291C01009D1C01005A
:101AA000610C01000021FFF7E9BE00BF30B504461C
:101AB00083B0FFF787F8A37D6FF30003A3759B0640
:101AC00001D4636873B3962001F0DAFE00231A464E
:101AD0001946184601F01CFE0120F6F7E1FE054606
:101AE000D0B105F11C0001F0FBFBFEF735FD40B95C
:101AF00001F052FE0D48214603B0BDE8304001F030
:101B000093BA0DF10700FEF703FC002201469DF891
:101B1000070002F091F8EBE7054840F25631F0F784
:101B2000C9FEDEE701F020FED6E700BF3921000044
:101B3000C4D6010010B50446FFF744F801F06EFE6C
:101B40002046BDE81040FFF74BB800BF08B5FFF7CF
:101B5000ADFF01F0EDFBBDE8084001F0A3BF00BF01
:101B600070B582B00546FFF71BF801F0FDFD0120BE
:101B7000F6F796FE0446B8B304F11C0001F0B0FB82
:101B800001F004FCE0B9FEF7E7FC10BB01F098FFA0
:101B900000210446084601F0BDFB00210646084628
:101BA00001F0B4FB3444C334201A01F041FF01F0CA
:101BB000F3FD1048294602B0BDE8704001F034BA88
:101BC0000D484FF44571F0F775FEFEF7C5FC00288F
:101BD000DCD00DF10700FEF79BFB002201469DF8CB
:101BE000070002F029F8D1E703484FF44471F0F7F9
:101BF00061FEC1E739210000C4D60100C36870B599
:101C00001E680446F3F7D0FF05463046FEF770FF26
